:020000040000FA
:10000000407F040001000000B0010000B0010000CA
:10001000B0010000B0010000B0010000B00100001C
:10002000B0010000B001000056610100B001000005
:10003000B0010000B0010000B0010000B0010000FC
:10004000445F0100B0010000B00100001C6D010020
:100050005C6C010054210100B0010000B0010000FF
:10006000D6450100B0010000B0010000B001000061
:10007000B0010000B0010000B00100001A6E0100E4
:10008000E0660100B00100005E6D0100BC6C010083
:10009000B0010000B0010000B0010000B00100009C
:1000A000B0010000B0010000B0010000B00100008C
:1000B000B0010000B0010000B0010000B00100007C
:1000C000B0010000B0010000B0010000706B010041
:1000D000B0010000B0010000B0010000B00100005C
:1000E000B0010000B0010000B0010000B00100004C
:1000F000B0010000B0010000B0010000B00100003C
:10010000FFFFFF00FFFFFF00B0010000B001000093
:10011000B0010000B0010000B0010000B00100001B
:10012000B0010000B001000056610100B001000004
:10013000B0010000B0010000B0010000B0010000FB
:10014000445F0100B0010000B00100001C6D01001F
:100150005C6C010054210100B0010000B0010000FE
:10016000D6450100B0010000B0010000B001000060
:10017000B0010000B0010000B00100001A6E0100E3
:10018000E0660100B00100005E6D0100BC6C010082
:10019000B0010000B0010000B0010000B00100009B
:1001A000B0010000B0010000B0010000B00100008B
:1001B000B0010000B0010000B0010000B00100007B
:1001C000B0010000B0010000B0010000706B010040
:1001D000B0010000B0010000B0010000B00100005B
:1001E000B0010000B0010000B0010000B00100004B
:1001F000B0010000B0010000B0010000B00100003B
:100200002F4E22000E7F22000E0188000000000009
:100210000C000700006723001100200011000700F8
:10022000000020000000E000020032000000020098
:100230000000000050090200010000000040DA0048
:100240000000FE004440A90080FA20000000E00009
:100250000300320000002000A00188004440A800F4
:100260000000060091018800800078000000EB008B
:1002700015003700E280400032A0B4009101BA00BE
:10028000E280400032A0B4009102BA00E280400057
:1002900032A0B4000002EB00472BDE00F507B200ED
:1002A000602CE10004003A000059EB008301E900F2
:1002B000FDFF3E00040037006128E100010032002C
:1002C0000082EB00040007001101BA000200E00008
:1002D000E8FF3A00000006003159BA008301E90046
:1002E0000C0032002159BA008301E90008003200F5
:1002F0000400E00003003A00E280400032A0B400B5
:10030000F5FF370011D9BA008301E900FAFF3A007E
:100310008100E800E180400032A0B4000000060047
:100320003C17040001000000D45404000100000048
:10033000B416040001000000BA52040001000000DD
:1003400098610400010000003E1404000100000058
:1003500076490400010000005E4A0400010000002C
:100360000040DA000000FE00800078001106B100B5
:10037000030035009101B10001003C000050A100D4
:10038000000006001004B100030035009001B10028
:1003900001003C001000050000000500800078000E
:1003A0001104B100030035009101B10001003C00CF
:1003B0000050A000000006001004B1000700350046
:1003C0009001B100040034007000B100030035005A
:1003D0009001B10001003C00100005000000050084
:1003E0006900E100040035006D00E1000300340005
:1003F0000002B100010032000000050010000500FD
:10040000889FBE0080047800F02281000000E00098
:1004100003003A009A0007000000E0000A003500DF
:10042000F02281000900E00002003A000004780098
:100430000600370000047800090040009000070023
:100440000000E00001003D000084EB00080078009F
:100450004F04BE00000006000C02E20004003D0054
:100460000F42AB00020032000F02AB00FEFF320071
:100470000040DA00FEFF37000A00FA008001780031
:10048000E20F500028003E0000238100E10F5000E1
:1004900008003200E02120000000E00005003200EA
:1004A0006421200085212000A62120008001780001
:1004B00004003700C4202000E52020000621200091
:1004C00043212000144090000004E00004003500A7
:1004D0008009EB00144090000074A00010429800C6
:1004E000154090000028A30003003A00154090003A
:1004F0000024A000904298008001EB000700370024
:10050000154090000008A300FDFF320063C0780092
:100510000000FB00000B78008301E800828F51008F
:10052000F7FF3A000800370030002000B0BF9F00FE
:10053000C3BF9F00D1BF9F00E2BF9F006A805700EA
:1005400000C0DA006FB99700020078000080FA005E
:10055000000006000A00FA0011002000B1BF9F0051
:10056000C0BF9F006A80570000C0DA004FB89700F4
:100570000080FA00000006000A00FA005100200086
:10058000B1BF9F00C0BF9F006A80570000C0DA0063
:100590005FB897000080FA00000006000A00FA0029
:1005A000881F7800800178000000E00029003A00F0
:1005B00000238100E10F500008003200E0212000FC
:1005C0000000E000050032006421200085212000A9
:1005D000C72120008001780004003700C4202000DB
:1005E000E520200027212000432120001440900016
:1005F0000004E000040035008009EB001440900086
:100600000074A000104298000002EB000C003700BC
:10061000130A2000154478006140640002003A008B
:100620008301E900FBFF3A000402E80095417800ED
:1006300061C0610005003200170078008058780022
:1006400004035100820F5200F1FF3A0006005100EE
:100650000800370020002000A0BF9F00B3BF9F000C
:10066000C1BF9F00D2BF9F006C80570000C0DA005E
:100670005FB897004F0478000080FA000000060081
:10068000800078000000E00004003A0020462200CC
:10069000F022890001017800060037000081EB009C
:1006A000204E2200808F500002003E00F12289007F
:1006B0000001EB000200780000000600020AB90009
:1006C000001BB9000200B800810042008100430015
:1006D00000000600889FBE008A9FBE0001057800CA
:1006E0000100E0000400350008003C000000E000CC
:1006F000200032000500370060001000E080180084
:1007000002003B0001F02C001A0037000004BE007C
:100710006011B8006B0920000982CF000200390087
:100720000882CF000441B000694252000E0032003E
:1007300008003B0082817100610164008904D100DE
:100740000884D3008B05E8000442E800F9FF3A0072
:10075000050037000804440089844C008B05E9003B
:100760000442E900FBFF3A00860107000AF0A700F7
:1007700001F0A0004F05BE004F04BE0000000600BF
:10078000889FBE008A9FBE008C1F7800A3010700CF
:100790001002200002003B0010458800A70137002E
:1007A0008A0062006408E10002003A0010458800F7
:1007B000AF0137006108E100FCFF32000800BE0015
:1007C000030478000B00070001F0A100AB01070053
:1007D00008F0A600040037000001BE0091042400C8
:1007E000B0FD20007900070009F0A70001F0A20089
:1007F0009B013700889FBE008A9FBE008C1F780037
:10080000860107008D01330003866C006450E1000F
:100810002E0032006420E100330032006150E1001C
:100820002F0032006120E100310032008585550043
:10083000EB07B00009002000080420000500370085
:100840000804440089844C000A0031000603430078
:1008500087834B000001530081815B00F8FF330068
:100860000203BE000800A0000804440089844C0074
:10087000F6FF3900C639DD00830173000100320044
:10088000130020008904D1000884D3000998A30034
:10089000050032000800A7000300A0008904D10071
:1008A0000884D3008B05E8008904D1000884D300B4
:1008B0000001EB000281D2003201070001F0A1002B
:1008C0000CF0A70001F0A000650137006420E100F2
:1008D000670132000801BE000200BE00F7FF3700CA
:1008E0006120E100620132006000B800F3FF3700D0
:1008F0000000200001F82700F0FF3700889FBE00AD
:100900008A9FBE008C1F7800440107004B01330012
:1009100003866C006450E100240032006420E10092
:10092000270032006150E100220032006120E10026
:10093000210032008B854200EB07B1000134B80082
:10094000003AB8000804420089844A00013AB8001D
:100950000030B8008880400009014A0004003300DC
:100960000000400081804800020149008B05E90039
:10097000C909DD008301700001003200130020006E
:10098000C814DE004814DD004709DE001200B20082
:10099000C808DE0008847000FA00070001F0A1001A
:1009A0000CF0A70001F0A0002D0137006120E1004C
:1009B0002F0132000801BE000200BE00F7FF370021
:1009C0006150E100FCFF3A002901370003F0A2006A
:1009D000889FBE008A9FBE008C1F78000F01070011
:1009E000160133006450E1004F0032006420E10042
:1009F0005200320003826C0007003B000905D00062
:100A00000306D000820F54000C065D00020039007E
:100A100002003200890178000306780085825500C3
:100A200004003D000003FD008103FD008502EA0093
:100A30008B854200840F720002003B0060001000B2
:100A4000E08018006011B8000005EB007A28E10092
:100A50000A00390006007800C75DDD00F707B20024
:100A6000878075002D003700828171000A017800AF
:100A7000610560008180D1000080D3008502E9001B
:100A8000F9FF3B00060440008784480002003B0059
:100A900060041400E0841C000988A30007003200F1
:100AA0008A81710082817100610164008904D10032
:100AB0000884D3008B05E800170037000978A300ED
:100AC00013003A000B00E000130034008B05E9002E
:100AD0000804440089844C000A4474000978A30087
:100AE0000D003A000B00E000070034008B05E90020
:100AF0000804440089844C0001003A000B002000E7
:100B00000978A300F7FF32000001EB000200370074
:100B1000828171000A0178009A0007000CF0A7009A
:100B200001F0A000CE0037006420E10002003A008E
:100B3000838F6C00CE0033000801BE000200BE00AF
:100B4000C70037000001EB0031010700040032004C
:100B50000200200003F8230001F0A7009BFF07001C
:100B6000000006000001BE00500107000470A7004D
:100B700003F0A1006509B100160032000D00350038
:100B80006828E10006003500F0FF2F00F1FF270084
:100B90000300E00013003B000100280000000500F6
:100BA00000004000818048008502E900FCFF3A0017
:100BB00008003700F88F420002003C008000EB0084
:100BC000000005008100D1000080D3008502E8000C
:100BD000FCFF3A000300E00002003B006000100050
:100BE000E0801800000006001400200044013700D7
:100BF000F4FF2F00420137000001EB005B013700DA
:100C0000839F68000100E00002003D0060001000CA
:100C1000E08018000300E00002003D0060011100C8
:100C2000E0811900B80107004F00E00002003B001E
:100C300060001000E080180000000600889FBE00E1
:100C40008A9FBE008C1F78000004BE0017010700B9
:100C50000478A30026003A006120E100250032005C
:100C600009F8A30025003A006420E10021003200C9
:100C7000F507B1000508A3000200320000004000A3
:100C8000818048006044B80003102000020020006A
:100C900000004000818048000805440089854C0020
:100CA0000A0541008B8549000A0550008B855800D4
:100CB000030033000A00BE00020474008384740041
:100CC0008301D1000281D300830F7100F0FF3A004D
:100CD0008904D1000884D3006001490082017800B2
:100CE000C1ADDE00FB07B000260007005C00370046
:100CF0000960A0000800BE00590037001202200061
:100D000012458800F0FF2F00F1FF27005400370044
:100D100004002000FA0037000001BE00E3000700D5
:100D20000470A70003F0A10003F8A30013003A0029
:100D30006509B10010003200090035006928E100A2
:100D400002003500010028000000050000004000FE
:100D5000818048008502E900FCFF3A00000006009F
:100D6000F88F4200050035008100D1000080D300DB
:100D70008502E800FCFF3A00000006008000EB005E
:100D80000000050081002000618055000B003D003F
:100D90000B00200061FE2F000100E1001D00340067
:100DA00082817100610164008904D1000884D3004C
:100DB0000000E800FAFF3A007100200061006400C2
:100DC000030070000200600009003200610444006A
:100DD000E0844C000988A500050032008B05E8007E
:100DE0006808E10002003A008904D1000884D300B9
:100DF000F20F20000258E10005003D00C75DDD0054
:100E0000F907B2008980750008007800000006002C
:100E10000BF827008B007800000005000004BE00DE
:100E2000A20007000003BE000405BE000200BE00D1
:100E30009E000700844F7500000006000200BE00FF
:100E40006450E100050036006420E1000200360035
:100E50000968A30001003A000800BE000160A0007C
:100E60004F0678004F05BE004F04BE00000006008C
:100E7000F0FF2F00F1FF2700F9FF3700889FBE0029
:100E80008A9FBE008C9FBE000004BE008700070042
:100E90000800BE00890678006420E10008003900DF
:100EA000040032000160A0001202200012458800F8
:100EB0005300370091FC2300B0FD20004E003700A6
:100EC0000006EB0009F0A10003F823000200200057
:100ED0000800BE0044FF07000600340001F82300AC
:100EE000000020000801BE0042FE07000004BE0012
:100EF0002C0020000800BE0093E82300320A2300E3
:100F000039FF0700120034000801BE00D1FD2300A4
:100F1000703D2B00AEFE07000005BE00B3F32300BA
:100F2000F27A26000800BE0074FE070003F82300D2
:100F300002002000A5FE07000801BE00A4FE070075
:100F40000A01BE002BFE07000004BE000C06E800EC
:100F50000800BE0001F0A100020020000398230059
:100F600021FF07000800BE00160035000801BE0082
:100F700062FE07000005BE0032CD2C0043FB2300BB
:100F800093FE0700809FBE001269280003D52B0046
:100F90000A00BE0059FE0700620F210013EF2B006C
:100FA0008BFE07000A01BE0054FE07004F01BE0081
:100FB00010FE07000801BE0050FE07000801BE0039
:100FC00083FE07000C00E0000B0032000C10A700AD
:100FD00001F0A200B2FD200093FC23006260E1005A
:100FE0000400320022A9200063F023000C10A700A7
:100FF00063F8230076FE07000DF0A70001F0A200C1
:101000004F06BE004F05BE004F04BE0000000600A4
:10101000889FBE008A9FBE000003BE002300070019
:101020008505780082815200020020006220E100E4
:1010300004003A00F307B100040035007718E1001E
:10104000040035000600BE00140037006000B80040
:101050000F003700F50F2000FAFF2F008502D100A6
:101060000A85D3008301E900FCFF3B008184620014
:1010700000046500890F7400F2FF32008582EA00E7
:101080000A85EA0081846200000465003DFF0700D4
:1010900007F0A70001F0A0000081EB000200E000D3
:1010A0004F05BE004F04BE0000000600C70ADE0068
:1010B000F107B200F50FB20008003200E1CF4200A4
:1010C000020032000170A00024000500810F7000B2
:1010D000010032000408050044000500810F700083
:1010E00002003A00140005008502E90000004000FB
:1010F00081C04800FCFF3B000170A00024000500F7
:10110000889FBE008A9FBE00841F780043FF0700AF
:101110004F00780011003300F0FF2F00838F6C0028
:1011200006003B00040565000A00A7000800370020
:1011300009F0A6001000200008003700820F5400BC
:10114000838F5C00030039001000200001003E0086
:101150000000200009F0A7000000EA004F05BE00D3
:101160004F04BE000000E00000000600889FBE00A3
:101170008A9FBE008C9FBE000206780001F0A70087
:101180000CF0A0000004BE00C8FF07000800BE006D
:101190006420E1000700390002003A00F1FF270057
:1011A000F0FF2F000160A00012022000124588000D
:1011B0005100370009F0A1000800BE000200200025
:1011C00003F823008AFE0700F4FF3C000800BE007D
:1011D000020020000398230083FE07000800BE00E1
:1011E000300035000200200003F0230080FE0700DD
:1011F00005003C000800BE000801BE00BFFD07005E
:101200000005BE000E0037000C10A20000002000F8
:1012100001F823000801BE00ECFD070002002000D9
:1012200003F02300B5FD07000005BE0083FE0700A4
:101230000200200003002C00B0FD07000004BE00E7
:101240000A00BE00B2D02800130B2C00E0FD0700FE
:101250000A01BE00A9FD0700020F2500330B240080
:10126000DBFD0700809FBE000A00BE005206220080
:1012700013F02B00A1FD0700B2662100F3F6230056
:10128000D3FD07000A01BE009CFD07004F01BE0010
:1012900058FD07000801BE0098FD07000801BE00C8
:1012A000CBFD07000C00A70007003700B2FD2000AF
:1012B00093FC23000C10A700C5FD07000CF0A7004D
:1012C00001F0A2000C0037000CF0A700020037006C
:1012D00001F0A20004003700B2FD200093042400B6
:1012E0000C10A60003003700B2FD200093FC230081
:1012F0000C10A700B6FD07004F06BE004F05BE004C
:101300004F04BE00000006006022B8000602200064
:101310000000D0008180D2000482D2008582D200F9
:101320000000A0000202520083825A000300310034
:101330000202420083824A000000A1000603E90085
:10134000F3FF3A0000000600881F780000047800D0
:101350005001BE004000BE000400400085804800EF
:101360000601490087814900009CBE000294BE002E
:101370000400E1000588E1000690E1000798E10023
:1013800002003100680044001008E8004F047800B3
:1013900000000600F4874700889FBE008A9FBE00B9
:1013A0008C9FBE008E1F78000205BE000004BE00A8
:1013B000D4B79F00E5B79F00F6B79F0087BF9F0097
:1013C0000000EB00C0B79F00B0B79F00A0B79F0020
:1013D00090B79F0080B79F000D042000BFB097001A
:1013E0004FB09700000140000000E0000F003D00FA
:1013F0004F08DE0000007100C0B79F009E0007008C
:1014000001003D0012002000A100070001003D0086
:1014100012002000A6000700B1000700B600070078
:101420000F004000C8FF0700220037004F08DE0011
:1014300000067100CCB79F008F00070001003D003F
:10144000120020009200070001003D001200200061
:1014500097000700A20007000FB297009FB2970005
:101460002FB39700BFB39700A900070000005200F8
:1014700081805A0002015B0083815B0080B79F007E
:1014800091B79F00A2B79F00B3B79F000007EB0082
:101490009F0007000020E10001A8E10002B0E10088
:1014A00003B8E100010031001E0020000E005600CC
:1014B000C0B79F004FB297000400E000070035005E
:1014C00010002000010020006011B8000804700026
:1014D000898470000A0571008B8571008D06E90012
:1014E000BEFF3A000400E00003003D008200070058
:1014F0000F00400094FF07004FA897000000E00095
:1015000004003A000FB497009FB497002FB59700DE
:10151000BFB59700940007004F0778004F06BE0044
:101520004F05BE004F04BE004F01B1000000060091
:10153000881F780018002000881F780095FF07009A
:101540008F87E9004F04780000000600801FEB0041
:1015500090FF07008F87E90000000600889FBE000B
:101560008A9FBE008C1F78006E00070007003D00B8
:1015700073000700E00F5B00E08F5B0007003D0099
:10158000320007000006EB000400370034000700BB
:1015900002003D002A0007001C0020007200070026
:1015A000E3FF07000203BE000002BE000C00E000E3
:1015B00001003200220007000400BE000601BE0048
:1015C0004F0678004F05BE004F04BE000000060025
:1015D000889FBE008A9FBE008C1F780051000700C4
:1015E00005003D0056000700E00F5B00E08F5B0048
:1015F00006003D00040037001900070003003D000D
:101600006000B8006011B800100007005600070025
:10161000CEFF07000203BE000002BE000C00E00087
:1016200001003200060007000400BE000601BE00F3
:101630004F0678004F05BE004F04BE0000000600B4
:101640006000B8006011B8000000370004025000CC
:101650008582580006035900878359000000060060
:101660000006EB00E00F5200E08F5A00E00F5B0035
:10167000E08F5B00000006000180400090B79F00F3
:101680000001EB008FB097000100E00000000600B1
:101690000200700090B79F000180400080B79F005B
:1016A0000001EB00FFA897000100E0000000060029
:1016B0000200700080B79F00018040006FAA970071
:1016C000CF20DE0001007000F0AF9F000402420056
:1016D000250007004F18DE0000027200000006001F
:1016E000E4AF9F000804440089844C000A054D00C3
:1016F0008B854D00000006003FB29700CFB29700E7
:101700005FB39700EFB3970000FE2F0000000600C4
:101710003FB09700CFB097005FB19700EFB197004F
:10172000000006000205BE000004BE00E00F5000ED
:10173000E08F5800E00F5900E08F590000000600CC
:101740006000B8006011B800080450008984580097
:101750000A0559008B8559001C002000E00F52003B
:10176000E08F5A00000006000800BE000A01BE001B
:10177000000006002800FA00889FBE008A9FBE0075
:101780008C9FBE0003866B000C0207000028A3009C
:1017900064003A000128A30067003A000008A30093
:1017A00062003A000108A30065003A001E009000A4
:1017B000BE08900081064000ED3FB100F480570064
:1017C000EE019000111AB8008E099000311BB8008C
:1017D0009E099000311CB800511DB800F4855700D7
:1017E00046000700FE0190003A0007008B85E800E4
:1017F0003E0007008E09900040000700EE019000B7
:10180000340007008B85E800380007008E0990003F
:10181000400007009E0990001B18B8008904400092
:101820000A854800FE019000340007008B85E8001F
:1018300038000700EE019000300007008E0990008C
:101840001B18B800890440000A8548000A98A300C4
:1018500008003A000402420085824A0006034B0059
:1018600087834B0008044C0089844C000A054D0016
:101870008D06E90084827200850273004C3ADD0017
:10188000850272000100320015002000443ADE009B
:101890001400B2004538DE00CB45DD000B007000BF
:1018A000C540DE00CB4DDD008B8070004549DE0079
:1018B000CB55DD000B017100C551DE000D03780032
:1018C000D701070003F0A1000CF0A70003F0A0006F
:1018D000CE0137001B18B80085024000068348007F
:1018E000E0834B0060044C00070037001B18B80071
:1018F0000603400087834800FAFF37001B18B80032
:101900008703400008844800E0844C0060054D00D7
:10191000000006001B18B800080440008984480035
:10192000FAFF37000108A300B5013A005800BE00D5
:101930005801BE00E3FF37000008A300B0013A00E1
:1019400009047800F9FF370081037800D7FD07000C
:101950000001BE006000B8000478A30013003A0044
:101960006220E10015003E000D0039008301D10026
:101970000281D3008180D3008301D1000281D30092
:101980008180D3008301D1000281D3008180D30004
:101990000538B000C42ADD00F300B2008381720074
:1019A00007F0A70003F0A00000000600F3FF2700E7
:1019B000F2FF2F006110B900FBFF370003FF270083
:1019C000F7FF37008F1FD100C10107008F87E900A3
:1019D0000000E00000000600801FEB00BC010700D3
:1019E0008F87E9000000E000000006001400FA0004
:1019F000889FBE008A9FBE008C9FBE000005BE006F
:101A00000206BE00680047000C90BE000A90BE00AF
:101A1000D80107006400E1001A00320016003E0001
:101A20006100E1001A0032006E049000FE04900094
:101A30000E0B90009E0B90006011B8009E05900068
:101A40000B38B100D5012000828171006101640072
:101A50008703D1000683D3008984D3000884D30090
:101A60008502E900F8FF3A00C6FC07000DF0A70068
:101A700001F0A00065013700F1FF2700F0FF2F0003
:101A80006201370001F8270000002000F7FF37004F
:101A90006000B800F5FF3700DD0107000509780098
:101AA00000000600809FEB00890107008F87E90096
:101AB0000000E000000006002800FA00889FBE0039
:101AC0008A9FBE008C9FBE0007067800878669004B
:101AD0000C003B00030478008704780008F0A100A4
:101AE00009F0A100840F5000858F5800860F59001F
:101AF000890F5C00030033000CF0A20001003A00E3
:101B00000CF0A1002D0107006400E1005F0032002D
:101B1000780147006408E100610032006C01470071
:101B2000748557003200BE001201BE003A04BE00A8
:101B30001A05BE001E039000BE0A900085035300E4
:101B400006003D000004FD008104FD000205FD00CB
:101B50008305FD008703EA00050378000DF8A30064
:101B60000400320060041400E0841C0060051D00C5
:101B7000E0851D006022B8007D0320000D38E100E3
:101B80008006EB000B0039004433DD00F300B200A7
:101B90008301730039003700848272000D027800DF
:101BA000E10664008B85D1000A85D3008984D300C7
:101BB0000884D3008703E900F7FF3B0008004000DA
:101BC000898048000A0149008B81490004003B00DC
:101BD00060001000E080180060011900E081190029
:101BE0000358A300090032008D82720084827200C3
:101BF000610260008301D1000281D3008180D300A3
:101C00000080D3000603E8001B0037000348A30050
:101C100017003A000600E000170034000603E90050
:101C20000D00A30000004800818048000201490027
:101C3000838149000348A3000F003A000600E0003A
:101C4000090034000603E9000000400081804800DC
:101C5000020149008381490001003A000003EB00C2
:101C60000348A300F5FF32006022B80002003700ED
:101C70008482720061826600E900070003F0A1001F
:101C80000CF0A70003F0A000E0003700640147005B
:101C90006408E10002003A000DF8A300D8003A0001
:101CA0003200BE001201BE00D80037001400FA0056
:101CB000889FBE008A9FBE008C9FBE000004BE00AD
:101CC0000205BE00680047000A90BE000890BE00F2
:101CD000280107000070A7000BF0A1000BF8A3007B
:101CE00020003A009E0990000E099000FE0090002E
:101CF0006E0090009E0290003443200084825200C7
:101D0000C20032000A003C00B4FC2F000428E100AD
:101D1000140034008301D1000281D3008180D300FC
:101D20000080D3008502E800FAFF3A00B7003700D0
:101D3000B40020000428E10007003C00000040003F
:101D40008180480002014900838149008502E90041
:101D5000FAFF3A00AD00370003002800020020001F
:101D6000010037006011B8006000B800A70037001C
:101D70002800FA00889FBE008A9FBE008C9FBE008C
:101D800003866B008D0007006400E1004400320010
:101D90006408E1004A0032006100E10046003200C0
:101DA0006108E10049003200EC0647006000B8001D
:101DB0003D02BE003D03BE00F48657006011B8002E
:101DC0003D04BE003D05BE007D0320000B00370032
:101DD0000000A0008D06E90013003200040242005A
:101DE00085824A0006034B0087834B0000004000B9
:101DF00081804800020149008381490008025200A5
:101E000089825A000A035B008B835B00F0FF3B0072
:101E10000802420089824A000A034B008B834B0070
:101E20008D06E900EDFF3A0084827200868272001E
:101E3000F707B2008782720001003200150020000F
:101E40001E0490003E0B900006035400E63FB000D5
:101E50000368A300070032000000A7000500A000EF
:101E60008301D1000281D3008180D3000080D300A0
:101E70000603E8008301D1000281D3008180D300F2
:101E80000080D3000002EB000482D200640007004F
:101E900003F0A1000CF0A70003F0A0005B003700E6
:101EA000640247006408E100550032003400BE00BF
:101EB0003401BE00F6FF37006108E1005000320037
:101EC0006011B8006000B800F1FF370003FF270081
:101ED00002002000FBFF3700889FBE0083047800CB
:101EE0000300E0002C00350003003C00008270007D
:101EF000040271002600320036432000C500200095
:101F00008383CF000A0039000541B1008283CF00EE
:101F1000070039000541B1008183CF00040039007A
:101F20000541B1008083CF00010039000541B100B7
:101F300085C353006022B800120032000A003B0043
:101F400084827200610260008301D1000281D300AB
:101F50008180D3000080D3000603E8008743E800B7
:101F6000F7FF3A000700370000004000818048007A
:101F700002014900838149000603E9008743E90023
:101F8000F9FF3A002600070009F0A70003F0A000BF
:101F90004F04BE000000060060001000E080180042
:101FA00060011900E0811900D3FF3B00033E2C00C3
:101FB000F7FF370007F0A200BFFE370068044700B4
:101FC0000294BE000094BE00FC0447008694BE004C
:101FD0008494BE00090078006600070008007800BD
:101FE0006400070099007800814F70000B003B00EF
:101FF0000800BE00930007004F00B1000300370047
:10200000F3FF2700F2FF2F006110B9004F06BE005A
:102010004F05BE004F04BE000080FA00000006001D
:102020001800200057002000080453000D003D0058
:102030000600200097FC2F000740E1001E0034003E
:1020400084827200610260008301D1000281D300AA
:102050008180D3000080D3000804E800F8FF3A0034
:10206000470020006104600005047400040464005B
:102070000D00320061004000E0804800600149002E
:10208000E081490003B8A500070032000603E8001C
:102090006538E10004003A008301D1000281D300D9
:1020A0008180D3000080D300F87F20000830E10059
:1020B00003003500080378006000B8006011B80024
:1020C0004433DD00F300B20083017300000006001A
:1020D000889FBE008A9FBE008C9FBE000404BE0085
:1020E0000605BE00809FBE00829FBE006300070001
:1020F000040678000800BE000A01BE005F00070069
:10210000840678004F03BE004F02BE008D4F76005C
:102110007FB0970013003300F0FF2F008B8F6B0010
:1021200006003B000D0666000C00A7000A00370001
:1021300007F0A600100020000A003700880F5200A8
:10214000898F5A008A0F5B008B8F5B000300390078
:102150001000200001003E000000200007F0A70052
:102160000000EA004F06BE004F05BE004F04BE004F
:1021700000000600800078005002BE005003BE0040
:102180004439DE00F700B200F37F20000301610054
:10219000090032000218E10016003A0085017200C1
:1021A00083017300838173000008200015003A004A
:1021B0004000200013003700850172008301730086
:1021C0008381730005003A0004A8BE0006A8BE0083
:1021D000100020000B0037000201E9000402420059
:1021E00085824A0006034B0087834B000748A30003
:1021F000F9FF32000740A00004A8BE0006A8BE00F8
:102200002000200080009800920098000000060046
:102210000003BE00A5FB07006220E10002003200BF
:102220000600BE0005000500E507B100F107B20099
:1022300004F023008480700007F0A70001F0A000E4
:1022400024000500E48240001078A300070032005B
:10225000640240001178A3003400BE001401BE00E7
:10226000040032000330A700000006003500BE0065
:102270001501BE000330A0000000060005FF270086
:1022800005826100070032000428E10001003200ED
:10229000240005000600070001003A004400050084
:1022A0000408050002000700F9FF3A0014000500C9
:1022B0006F826100810270008502710085027200E8
:1022C00000000600800078003004E000FEFF3A00C5
:1022D000010050000000E900000006000C00FA00B8
:1022E000A0BF9F00C0BF9F00F6FF0700B0BF9F00C8
:1022F000F0BF9F00100C2000D0BF9F0074815700DA
:10230000EFB097006C805700470107000080FA008B
:10231000000006008001EB000200370081717800A8
:102320008301E800828F5100FCFF3A0000000600A4
:102330000C00FA00A0BF9F00C0BF9F00E1FF070094
:10234000B0BF9F00F0BF9F00100C2000D0BF9F00C7
:1023500074815700EFB097006C8057007F02070030
:102360000080FA00000006000001780000C2B300FF
:10237000010037000201E8009240780080CF500051
:10238000FCFF3200E9CF5000FAFF3200D0C2B300A8
:1023900080CF500003003A000201E80014C0B300EF
:1023A000050037000042EB00B0C2B30080CF500000
:1023B00001003A000201E8008000EB0005FD2F005B
:1023C000040037006A08B900008041008500400021
:1023D0000201E8009201FB0005804100E90F500076
:1023E000F8FF36000404E000010032008100EA003A
:1023F0000100780000000600889FBE008A9FBE0092
:102400008C9FBE0000017800A13F22001100E00077
:102410000B003A00E03F2200D01F8900B01F890066
:10242000F11F8900C11F8900214090000004A00015
:10243000A0409800614090000004A000E040980097
:10244000E7004100C208DE00C20CDD00C41F8100AD
:102450002D462200204E22000D05500022002000B3
:10246000811F7800110009000205D80000067800DD
:10247000CF007800C308DD00E48540008001EB0058
:1024800026462200A53F2200010037000102780005
:10249000244090000008A300020032000A00370028
:1024A000110A780094007800214090000008A300F1
:1024B000FBFF320009014200828F50000200390008
:1024C000840F51004600310094007800848F500042
:1024D000EEFF3E00868F500002003900858F5000CD
:1024E000EAFF3900B01F8100800F52004F003A0010
:1024F000858F50004D003A008301E800E18F5100C4
:10250000E2FF36008C8F5400040036008A8F54009E
:10251000020031000B04780012003700614AB80055
:102520006151B900B0FF2F000100200002005000EF
:1025300083805800800F5200818F5A0002003500BE
:1025400009047800070037000D805400524E220025
:1025500002004000110009000A80D8000A80B9007A
:102560000004780008007800A5F7070080017800D3
:10257000E10F40002D003200B01F810003087800F9
:10258000B21F810064004100A2409000808F510082
:10259000020032000104A000010037000104A10084
:1025A00021419800088041006400500080097800B3
:1025B000B01F8900A23F220002087800B11F8100ED
:1025C000214090000004A000A0409800234090000B
:1025D0000004A100A041980002027800A7FF370084
:1025E000C21F8900828F50000900360092007800D7
:1025F000403F2200A241900003487800911F8900CB
:10260000140978008040EB00C01F81002140980031
:10261000C01F8100000A7800244090000004A00040
:102620002042980064004200010037000000EB00E7
:102630004F06BE004F05BE004F04BE00000006005E
:1026400064005000C01F8900A04090000104A10058
:102650002140980000000600889FBE008A9FBE00AF
:1026600000057800E401500013001000C285DE0070
:10267000234090000008A30004003200C31F89001B
:10268000234090000004A100A041980001007800C0
:1026900059FF0700000478000000E0001700320036
:1026A0008A0F50001500320060B8970008005000F3
:1026B000C284DE00898F550001003600890578004C
:1026C0004259DD008A00780008007800C402070043
:1026D0008A0F5400090031004248DD000000440028
:1026E0008A0F5000050036000A0050000000440028
:1026F000921F8100A31F81000288BE00080078009D
:102700004F05BE004F04BE00000006000004780024
:10271000BA020700080078004FF707000C00FA0023
:10272000889FBE0000047800CFB09700F0FF27001C
:10273000D0BF9F008004EB0099BF9F0088BF9F001F
:10274000A8BF9F00200C2000B0BF9F0078815700D9
:10275000708057000E0307000FB8970009487800F3
:102760000FB8970008045000080078004F04BE001E
:102770000080FA0000000600889FBE000004780078
:102780008144780000FD2F0000004400E90F500054
:1027900002003E00000178000D00370008007800BC
:1027A000F8F607000000E00003003200080078009F
:1027B000FAF607000004780008007800FEF607002B
:1027C0000000E0000700320090FA2F0000014400F2
:1027D0000980FB00800F510002003D000280FB00D9
:1027E00001003700F00F20004F04BE00000006007B
:1027F000881F7800A02281002A08070000047800C2
:10280000F7F607000000E000FAFF3A00E10F44008D
:1028100003003200A122810008007800550807005B
:102820004F04780000000600EC874700889FBE0038
:102830008A9FBE008C9FBE008E1F780081BF9F00C4
:1028400002077800A02289008046EB0004013700CF
:102850008884FB0009007800E1F60700800078001A
:102860000000E00002003200E1FF0700FC0037003A
:1028700050C2B300804F5400F0003A000FBD9700E3
:1028800020C0B300C0EF9F00D1EF9F0081EF9F00F9
:102890000300370040C0B300C0EF9F000FBD97009A
:1028A0000FB99700B240780082BF9F008184FB007F
:1028B00090C6B30080CF50003500320017003E00B4
:1028C0006640500080CF5000620032000C003E0095
:1028D0007740500080CF50002800320006003E00B4
:1028E0000104E0009B003200A0C2B30080CF500082
:1028F0006E003A001D00370080C5B3001600370097
:1029000040C6B30080CF5000210032006440400038
:1029100080CF500065003A001200370030C7B30086
:1029200080CF50001E00320007003E00674050007C
:1029300080CF5000110032006340400080CF500033
:102940005A003A001400370050C7B30080CF50003F
:102950000F0032006340400080CF500053003A0027
:102960006500370020C0B300CBFF3700DFE89700D9
:102970008140E800D1EF9F00C8FF37004FE9970082
:1029800080C0B300E24F5100C3FF3A00C1FF3700DF
:10299000ACC0B300590037008CC0B30057003700FB
:1029A00093FF0700DFE897000104E00002003A000F
:1029B0004E017800D2B79F00A0228100B90707001E
:1029C00000047800E10F4000A20032008FEC970075
:1029D000120037000A85E8008ABF9F001600370002
:1029E0008FB897001100FB00800F5400F9FF3200F0
:1029F0005FE997000204E00003003A005FB097002F
:102A000008587800D0B79F008944E9000A003200D6
:102A1000A0228100A3070700000478000800E80056
:102A2000E10F500004003600080078006CF6070043
:102A30000000E000EAFF3200DFE897000104E00058
:102A400087003A008D46E8005FB1970001497800A1
:102A5000830037005FE897000004E00003003A00BD
:102A60008D46E800CE007800D1B79F00A0228100FB
:102A70008C070700E10F4000760032005FE9970005
:102A80000204E00003003A00DFB0970080587800AD
:102A9000D1B79F000FE997000241E90082EF9F0044
:102AA0004240A9006E003400F0FF37000180FB00B7
:102AB00008FD2F0008004000E90F50005F003E00B5
:102AC0000A00780028FE070080EF9F008800780049
:102AD000030037000FB897000000E80080BF9F0098
:102AE0000FB997001200FB0001004000E90F5000F1
:102AF000F8FF360069FF37000CC1B3003CFF070048
:102B0000A022810067070700000578000040EB0065
:102B1000E0EF9F00D0022000800F550005003A0032
:102B2000A02281005F0707000005780011C0B300F4
:102B3000E1EF9F008C4078000A0078000EFF07004C
:102B4000E14F40000A003A00A12281000A0078000B
:102B5000880707000D04E0004B003A00A022810026
:102B6000300090000048A3004300320048003700C6
:102B70008FED97006044B8000C81FB00030020003B
:102B80000800BE00CDF607000004BE008C407800AF
:102B90000A007800F8FE07000080FB00010020001A
:102BA00008044000898448008B45E9000700320092
:102BB000A02281003B070700000578008C407800C8
:102BC000EDFE0700E14F4000EBFF3A008C4078003B
:102BD0000A007800E8FE0700E14F400003003A00D9
:102BE000A12281000A007800620707006FE99700C0
:102BF0000204E0000200320060041400E0841C00C3
:102C00005FE897000004E00015003A008D46E800F8
:102C1000CFE89700E4CF500003003A004E00780060
:102C20000888BE000E0037000E81E9000207780018
:102C3000120078000808780009003700A0228100FF
:102C400018070700808F540005003200E10F400094
:102C50000B003A000D04E0000D0032000A003700BE
:102C60008FB897003144780081BF9F000804E000CE
:102C7000F7FE3A00040037000000EB0005003700C3
:102C8000A12281003B0707000D80FB0001003700F7
:102C90000080EB004F0778004F06BE004F05BE00D6
:102CA0004F04BE00CF00B10000000600889FBE00A8
:102CB000000478008144780000FD2F0000004400EB
:102CC000E90F500002003E00000178000D003700BF
:102CD00008007800ABF507000000E00003003200B8
:102CE00008007800ADF507000004780008007800BF
:102CF000B1F507000000E0000700320090FA2F0055
:102D0000000144000980FB00800F510002003D00DB
:102D10000280FB0001003700F00F20004F04BE00CE
:102D200000000600881F7800B0228100DD06070041
:102D300000047800AAF507000000E000FAFF3A005E
:102D4000E10F440003003200B12281000800780046
:102D5000080707004F04780000000600EC874700D2
:102D6000889FBE008A9FBE008C9FBE008E1F780089
:102D700081BF9F0002077800B02289008046EB00E7
:102D8000040137008884FB000900780094F50700EF
:102D9000800078000000E00002003200E1FF070040
:102DA000FC00370050C2B300804F5400F0003A00DE
:102DB0000FBD970020C0B300C0EF9F00D1EF9F0070
:102DC00081EF9F000300370040C0B300C0EF9F00B9
:102DD0000FBD97000FB99700B240780082BF9F00E7
:102DE0008184FB0090C6B30080CF500035003200D4
:102DF00017003E006640500080CF50006200320055
:102E00000C003E007740500080CF50002800320078
:102E100006003E000104E0009B003200A0C2B300A7
:102E200080CF50006E003A001D00370080C5B3000F
:102E30001600370040C6B30080CF5000210032009A
:102E40006440400080CF500065003A001200370017
:102E500030C7B30080CF50001E00320007003E0094
:102E60006740500080CF50001100320063404000A6
:102E700080CF50005A003A001400370050C7B3000A
:102E800080CF50000F0032006340400080CF5000E0
:102E900053003A006500370020C0B300CBFF370075
:102EA000DFE897008140E800D1EF9F00C8FF3700BE
:102EB0004FE9970080C0B300E24F5100C3FF3A00D2
:102EC000C1FF3700ACC0B300590037008CC0B3005D
:102ED0005700370093FF0700DFE897000104E00088
:102EE00002003A004E017800D2B79F00B022810064
:102EF0006C06070000047800E10F4000A2003200D9
:102F00008FEC9700120037000A85E8008ABF9F0007
:102F1000160037008FB897001100FB00800F540097
:102F2000F9FF32005FE997000204E00003003A0075
:102F30005FB0970008587800D0B79F008944E90037
:102F40000A003200B0228100560607000004780013
:102F50000800E800E10F5000040036000800780087
:102F60001FF507000000E000EAFF3200DFE89700ED
:102F70000104E00087003A008D46E8005FB1970049
:102F800001497800830037005FE897000004E00003
:102F900003003A008D46E800CE007800D1B79F00CC
:102FA000B02281003F060700E10F400076003200AA
:102FB0005FE997000204E00003003A00DFB09700E9
:102FC00080587800D1B79F000FE997000241E900CF
:102FD00082EF9F004240A9006E003400F0FF3700EE
:102FE0000180FB0008FD2F0008004000E90F5000A1
:102FF0005F003E000A007800DBFC070080EF9F00C6
:1030000088007800030037000FB897000000E80040
:1030100080BF9F000FB997001200FB000100400025
:10302000E90F5000F8FF360069FF37000CC1B3000C
:103030003CFF0700B02281001A0607000005780057
:103040000040EB00E0EF9F00D0022000800F550011
:1030500005003A00B0228100120607000005780042
:1030600011C0B300E1EF9F008C4078000A007800A7
:103070000EFF0700E14F40000A003A00B122810034
:103080000A0078003B0607000D04E0004B003A0000
:10309000B0228100300090000048A30043003200BD
:1030A000480037008FED97006044B8000C81FB00AA
:1030B000030020000800BE0080F507000004BE00E9
:1030C0008C4078000A007800F8FE07000080FB00C2
:1030D0000100200008044000898448008B45E90075
:1030E00007003200B0228100EE05070000057800DD
:1030F0008C407800EDFE0700E14F4000EBFF3A0006
:103100008C4078000A007800E8FE0700E14F40009C
:1031100003003A00B12281000A007800150607007A
:103120006FE997000204E00002003200600414001E
:10313000E0841C005FE897000004E00015003A00FE
:103140008D46E800CFE89700E4CF500003003A0036
:103150004E0078000888BE000E0037000E81E9009E
:10316000020778001200780008087800090037008C
:10317000B0228100CB050700808F5400050032008B
:10318000E10F40000B003A000D04E0000D0032009A
:103190000A0037008FB897003144780081BF9F0044
:1031A0000804E000F7FE3A00040037000000EB00DE
:1031B00005003700B1228100EE0507000D80FB00FD
:1031C000010037000080EB004F0778004F06BE007B
:1031D0004F05BE004F04BE00CF00B1000000060046
:1031E0008001EB000200370061F079008301E80004
:1031F000828F5100FCFF3A0000000600881F780013
:10320000C02281000000E000010032000000010047
:10321000C835220008007800F30507006C0444005C
:1032200000382200800F5400FAFF3A004F04780063
:1032300000000600889FBE008A1F7800804078004A
:103240000004E00021003D008040EA00D0C6B30049
:1032500080CF5000090034008104FB0042062000AA
:10326000110009008204D8000001780001007800F4
:103270004311DD00EAE421001F0037000100FB00DC
:10328000E3E4210039003700A2002000110009000A
:103290000200D80000017800010078004311DD0031
:1032A000030141004300DD00030040003002BE0086
:1032B0002003BE0042209000D2209000F221900016
:1032C000622190002BF907002E003700D0C6B30012
:1032D00080CF5000230034008104FB004206200010
:1032E000110009008204D800000178000100780074
:1032F0004311DD00EAEF21000A014100A80020008F
:10330000110009000800D8004300DD000A00400059
:1033100040229000D022900060239000F023900083
:103320000288900092889000B289900022899000D3
:1033300010F90700801F78000102780011000900D1
:103340008804D8000102FD004F0078000402FB0051
:103350004322DD000A0242005403BE004402BE00C4
:10336000D8FF37000100FB00E3EF2100EACF500057
:10337000C5FF3C004300DD00030040005001BE00DB
:103380004000BE004F0578004F04BE00000006005C
:103390008F03B000889FBE008A9FBE008C9FBE0036
:1033A0008E1F7800E0B79F00F1B79F0082BF9F009B
:1033B0000000EB00A0B79F00E60437008001EB009F
:1033C00050C2B30080CF5000090032000100FB0062
:1033D000EFB09700EC040700E10F4000DD0432007D
:1033E000AFB097008100E800A1B79F00D904370073
:1033F0007FB1970092407800D0C2B30080CF5000D8
:103400000C00320007003C006D40500080CF50009F
:103410000D0032006B40400080CF500019003A0090
:103420000E00370000C3B30080CF500015003A00F3
:103430000F0037000330A0007FB297000402E800BD
:10344000F4B79F00EAFF37000300A000FFB2970027
:103450008502E800F5B79F00E5FF37000310A000E4
:103460007FB697000C06E800FCB79F00E0FF37002E
:103470000320A0007FB097000000E800F0B79F0095
:10348000DBFF37000318A300010032000300A10096
:103490000338A300010032000320A1000100FB005B
:1034A00002FD2F0002004000E90F500010003E0016
:1034B0008000EB00C1B79F00020278004FB1970077
:1034C0006A10B900FFB297001501FB00000141002E
:1034D00004014100C2B79F005500FB00F5B79F00F3
:1034E00004004000E90F50000D003E00F3FF3700DC
:1034F0000006EB00CCB79F00A0C2B30080CF500005
:1035000007003A000FB89700C000780080BF9F0006
:10351000C1B79F007FB197000201E800F2B79F009A
:10352000E0C2B3007FB29700944F100021003A0030
:10353000830678000DE0A0008400E800644050009D
:10354000914F100004003200F1B79F008002EB00A1
:10355000B5B79F00100037000FBE97004C007800F1
:103560008CBF9F00B0B79F00FFB097008180E8003C
:10357000F1B79F00130037003FB297006A20B900EF
:103580000000410003004000B0B79F00FFB2970069
:103590008502E800F5B79F007FB697001C01FB008D
:1035A00003FD2F0003004100E90F5000F2FF360039
:1035B00004003700830678000DC0A0000000EB0077
:1035C000B0B79F007FB19700B2407800F2B79F007C
:1035D000C17F9F00C0C6B30080CF500027003200DB
:1035E00014003C006840500080CF50009D00320025
:1035F00009003C006C40500080CF50002900320090
:103600006B40400080CF5000720032000104E000A7
:10361000560432008E00370060C6B30080CF5000E1
:103620001C0032006340400080CF500088003A0008
:103630008C00370030C7B30080CF50001C00320030
:1036400007003C006440500080CF5000130032005F
:103650000040E80080CF50007D003A0011003700A4
:1036600050C7B30080CF50007D003200634040005F
:1036700080CF500076003A000B0037000000280091
:103680000D48A30001003A0000012000808676006A
:10369000CCFF37000DA0A000720037000D60A00025
:1036A000700037000D50A0000D70A0006D003700B5
:1036B0008FB997004300780083BF9F000004780013
:1036C0000000E00001003A00083322008004EB0013
:1036D000010037008104E800890078000880440078
:1036E0001004E000FBFF3A003FB297000400E00046
:1036F00003003200890F5200010031008404780079
:103700000007EB00CFB29700898F5200010036000E
:10371000098752004368DE00E106600019003A00A4
:103720000D06780009003700EFB097000002200076
:1037300015040700E10F4000030032002FB097008E
:103740000000E800A0B79F000C06E8008E0F5600AE
:10375000F5FF3A000087EB000A0037008800780088
:103760003100FB0001047800EFB097000604070069
:10377000E10F400003003200AFB097008100E80085
:10378000A1B79F000900E90080047800E10F400024
:10379000F2FF3A000006EB000D00E0000A003A00DC
:1037A000EC033700EFB0970000022000F60307009B
:1037B000E10F4000030032002FB197000201E80042
:1037C000A2B79F000C06E8008E0F5600F5FF3A00E6
:1037D000E00337008FB997004300780083BF9F0054
:1037E000CF80DE0001017800820178000205BE0072
:1037F0000004BE000203BE000002BE004822DE003C
:10380000482EDD0004027600C47F9F000D48A3000F
:103810000A0032000404E00008003200E14F4200D8
:1038200006003200D1FB2F000180470004487800D9
:10383000184098002900200002003700D07F9F0028
:1038400019002000D2FB2F0002844700A6FF37009A
:10385000C3FB2F000384470019002000A2FF37009C
:103860000D0CB300007020000082660027023200B9
:103870000DC8A3000200320064002000B4B79F000E
:103880000D48A300050032000FBA97004401BE00A6
:103890004400BE0084BF9F00040037008FBA970029
:1038A0004500BE0085BF9F0027F80700E0AF9F00DE
:1038B000F1AF9F0082B79F0093B79F006022B800CE
:1038C0006033B8006FA89700FFA897000FB197006A
:1038D0009FB197003BF807000000E0000A003D00A0
:1038E0006FA89700FFA897000FB197009FB19700AE
:1038F00003F0A200E0AF9F00F1AF9F0082B79F00EE
:1039000093B79F003D00B3000000EB0080A79F002D
:103910006022B8006033B8006FA89700FFA8970036
:103920000FB197009FB197002BF807000000E0004F
:10393000340032006FA89700FFA897000FB19700DE
:103940009FB1970029F8070003FC2F00038147006F
:1039500051F807000FA097000000E9006300B900CC
:10396000A2002000110009000200D8008000FD0024
:1039700081A79F000100E00002003D000100E90076
:1039800080A79F000FA497000840EA0029FE0700C7
:103990006FAA9700FFAA97000FB397009FB39700F5
:1039A00074F70700A0AF9F00B1AF9F00C2AF9F00A8
:1039B000D3AF9F006022B8000600200007FF23005D
:1039C00000F807000000E00002003D000800E900E8
:1039D0000B0037006022B8000600200047022400D8
:1039E0002FA89700BFA897004FA99700DFA99700BD
:1039F0002CF807000000E000020035000800E80095
:103A000080A79F003FB29700F80F520057003C007C
:103A1000D0C6B300804F5200290036000485FB0059
:103A200042062000110009000285D800000178003C
:103A3000010478004311DD00EBE421000B0141009B
:103A40006022B8000600200007FE230002889000D4
:103A500092889000B28990002289900045F7070073
:103A6000A9002000809FBE00110009000984D80031
:103A7000000478004F00BE004344DD000B04440006
:103A800048229000D822900068239000F8239000EC
:103A900038F70700801F7800010278001100090044
:103AA0000985D8000102FD004F0078004322DD00A7
:103AB0000B0242005403BE004402BE001F00370048
:103AC0000480FB00E9E42100EA4F520014003600B4
:103AD000A2002000110009000280D8000001780037
:103AE000010478004311DD00090141006022B800A3
:103AF0000600200007FE230042209000D220900004
:103B0000F2219000622190001AF707004344DD0083
:103B1000090444003802BE002803BE000700370035
:103B20004300DD00090040006022B80006002000CC
:103B300007FE23005001BE004000BE000DF7070045
:103B40000002BE000203BE006FA89700FFA8970006
:103B50000FB197009FB19700D7F70700E0AF9F0024
:103B6000F1AF9F0082B79F0093B79F000FA497000B
:103B7000E90F540015003C006022B8006033B80023
:103B80006FA89700FFA897000FB197009FB197000B
:103B900091F707000000E000320032006FA89700A4
:103BA000FFA897000FB197009FB197003FF807005B
:103BB000E00F5000E08F5800E00F5900E08F5900EF
:103BC00028003A00E10F54002600340004002000D1
:103BD00005002E00B6E02200170124002FA8970050
:103BE000BFA897004FA99700DFA9970075F70700B6
:103BF0000000E00002003D007300540001003700A7
:103C00007200540080A79F000FC0970089FD070035
:103C1000A0AF9F00B1AF9F00C2AF9F00D3AF9F0086
:103C20000002BE000203BE006FA89700FFA8970025
:103C30000FB197009FB197004DF807001BF80700E0
:103C40000205BE000004BE006000B8006011B800AC
:103C5000A0A79F00B1A79F00C2A79F00D3A79F0066
:103C60002E0037006FA89700FFA897000FB19700AC
:103C70009FB197000DF807000205BE000004BE00CA
:103C8000E00F5000E08F5800E00F5900E08F59001E
:103C90000200350090F807001300370010002000E4
:103CA000010020006011B8000800600089806000F9
:103CB0000A0161008B8161008B03D1000A83D3006C
:103CC0008982D3000882D3000000720081807200D4
:103CD00002017300838173007FF807000002BE00B9
:103CE0000203BE0074F707000002BE000203BE001C
:103CF0006FA89700FFA897000FB197009FB197009A
:103D0000ACF80700A0A79F00B1A79F00C2A79F0023
:103D1000D3A79F000000EB0080A79F0014C0B30052
:103D2000651D22000B0037000400FB004300DD008E
:103D3000050040005001BE004000BE000040E10010
:103D400001C8E10002D0E10003D8E100030039001E
:103D50000442E800F44F5200F3FF3A00C47F9F0092
:103D60000400FB00BFB09700008040008FA09700C8
:103D7000010040004FB1970000075100BFB197000C
:103D80000300E000010032000E07E90063806600D6
:103D9000010032000E07E9000D28A30026003200C2
:103DA000E18066000D18A3000C003200D002200054
:103DB0000100E00001003A000080E900EFB0970048
:103DC00071020700E10F4000180032002FB2970087
:103DD0000402E800A4B79F00140037000100E000CF
:103DE00012003200EFB097000002200066020700C8
:103DF000E10F40000D003200AFB297008502E800ED
:103E0000A5B79F0009003700EFB09700000320001E
:103E10005D020700E10F4000030032002FB697005B
:103E20000C06E800ACB79F000E07E9000E00E000AA
:103E3000F5FF3C003D0037000D38A3000A003200BA
:103E40000B003700EFB09700000220004E02070081
:103E5000E10F4000030032002FB097000000E8009F
:103E6000A0B79F000E07E9000E00E000F5FF3C0040
:103E7000E18066000D18A3000C003200D002200083
:103E80000100E00001003A000080E900EFB0970077
:103E90003D020700E10F400024003200AFB0970060
:103EA0008100E800A1B79F00200037000100E0007A
:103EB0001E003200EFB0970000022000320207001F
:103EC000E10F4000190032002FB197000201E80015
:103ED000A2B79F00150037000000FB004300DD0083
:103EE000611D2200010040003002BE002003BE0020
:103EF0000800BE000A01BE008DF50700A4002000E6
:103F0000050020006033B80090F507000003B00002
:103F1000EFB097001C020700E10F400003003200E1
:103F2000AFB197008301E800A3B79F004F7A9700D5
:103F30000440E900C07F9F00E14F4000E6FF3A00E7
:103F40000B003700EFB09700000320000E020700BF
:103F5000E10F400003003200AFB297008502E80095
:103F6000A5B79F000FA097000000E90080A79F0061
:103F70000FA097000000E000F2FF3C003FB6970062
:103F800020C1B300F20F560001003C006FE0970023
:103F9000C07F9F00CF7897000100FB003FB19700E2
:103FA00000005100E0A79F000104E000080032007B
:103FB000EFB09700E0022000F3010700E10F40009E
:103FC00003003200AFB197008301E800A3B79F0060
:103FD0004F78970097FC07000002BE000203BE0066
:103FE0002FA09700BFA097004FA19700DFA19700D7
:103FF000E0F507002DF707001E0037000000FB006A
:104000004300DD006C1D22000C0040003002BE00A9
:104010002003BE000800BE000A01BE0044F50700F0
:10402000A4002000050020006033B80047F5070019
:104030000003B000EFB09700D3010700E10F40008C
:10404000030032002FB297000402E800A4B79F00DB
:10405000CF7A97000500FB004300DD000C00400014
:104060003002BE002003BE000800BE000A01BE00F0
:1040700036F507000205BE000004BE004F7E970023
:104080000C40E900C07F9F00E14F4000DBFF3A0099
:104090000006EB0009003700EFB097000003200096
:1040A000B9010700E10F4000030032002FB0970074
:1040B0000000E800A0B79F000C06E800EFA0970002
:1040C000810F5600F4FF3A000D38A300A101320021
:1040D0000E00E0009F0134000006EB00EFB09700F7
:1040E00000022000A8010700E10F40000300320099
:1040F0002FB197000201E800A2B79F000C06E8006C
:104100008E0F560093013200F4FF37000D00780047
:10411000000CB20028003A000D00E00005003D0050
:104120008FB997004305BE004304BE0083BF9F00C4
:10413000140037000D48A3000B0032000FBA97009F
:104140004400BE0084BF9F004F89DE00CF91DE0097
:104150000002BE0002037800820378000605BE005C
:104160000404BE00070037008FBA970045007800AE
:1041700085BF9F0000047800CFC4DE0009057800E9
:104180008A057800E00F5400E08F5C00E00F5D00CE
:10419000E08F5D0020003D003D00B3006000B800EE
:1041A0006011B80008045000898458000A055900BD
:1041B0008B855900180037000D00E00005003D0018
:1041C0000FBE97004C05BE004C04BE008CBF9F0084
:1041D000110037000D48A300080032008FBA970085
:1041E0004500BE0085BF9F0004017800840178006F
:1041F0000205BE000004BE00070037000FBE970096
:104200004C0078008CBF9F0000047800090020005B
:104210000A0020000B0020003FB097000000E000E3
:1042200007003A00E00F5400E08F5C00E00F5D00F3
:10423000E08F5D0002003A0011002000B1B79F003E
:104240000D0778000E0CB20000042000800F57000C
:104250002F00320003003C000E00E0000700320097
:104260003F00370000082000800F57001400320084
:10427000000C2000800F570039003A0014C0B30032
:10428000651D22000B0037000400FB004300DD0029
:10429000050040005001BE004000BE000040E100AB
:1042A00001C8E10002D0E10003D8E1002B00390091
:1042B0000442E800F44F5200F3FF3A0027003700B1
:1042C00000012000010020006011B80014C0B300FC
:1042D0000040E10001C8E10002D0E10003D8E100A4
:1042E0001E003900450020000000D0008180D2006F
:1042F0000281D2008381D2008502E900FAFF3A00F0
:104300000442E800F04F5200F1FF3A00130037007A
:1043100080002000010020006011B80014C0B3002C
:104320000040E10001C8E10002D0E10003D8E10053
:104330000A0039003C0020000000D0008180D2003B
:104340000281D2008381D2000C06E900FAFF3A0014
:104350000442E800F54F5200F1FF3A00C47F9F008D
:10436000CF7897000100FB003FB19700820F50000B
:1043700002003D00C27F9F0004003700BFB19700DC
:10438000808F510001003D00B0B79F004FB29700F1
:104390000400E00004003200638066000200320086
:1043A0000402E900C4B79F000DE8A3000B0032002F
:1043B000CFB297003FB697008C8F520003003C00AD
:1043C0000000EB00C0B79F0004003700CFB097009B
:1043D0003FB1970082805000C1B79F00CF7997000E
:1043E0000300FB000002EB0094A79F00CFB29700F0
:1043F000808F5200020034000080520090A79F007E
:104400000D28A30037003200E18066000D18A300DC
:104410000C003200D00220000100E00001003A0050
:104420000080E900EFB09700D7000700E10F4000DF
:104430000E0032002FB697000C06E800ACB79F00C4
:104440000A0037000100E00008003200EFB09700DA
:1044500000022000CC000700E10F40000300320002
:104460002FB097000000E800A0B79F009FA0970022
:104470000100E0000F0032000006EB00EFB09700F3
:1044800000032000C0000700E10F400003003200DD
:104490002FB197000201E800A2B79F000C06E800C8
:1044A0009FA19700830F5600F4FF3A000002EB0033
:1044B00094A79F00BFB29700C328DD00E01C220034
:1044C0008080400091AF9F004228DD0064005000D2
:1044D00080AF9F006328B900F0A79F0063065000DB
:1044E000820037001FA697000C00E0001100320088
:1044F000688066000F003A0000067800EFB0970071
:1045000000022000A0000700E10F4000030032007D
:104510002FB097000000E800A0B79F000C06E8004D
:104520009FA09700810F5600F4FF3A000001EB00B6
:1045300092A79F00E18066000D18A3000C003200D6
:10454000D00220000100E00001003A000080E900F4
:10455000EFB097008C000700E10F4000D5FF32005C
:10456000AFB197008301E800A3B79F00D1FF3700E8
:104570000100E000CFFF3200EFB097000002200002
:1045800081000700E10F4000CAFF32002FB2970000
:104590000402E800A4B79F00C6FF37000004200013
:1045A000800F57003000320003003C000E00E00096
:1045B000070032003D00370000082000800F570040
:1045C00011003200000C2000800F570037003A0025
:1045D0001FA897003002BE002003BE000800BE00E6
:1045E0000A01BE00D2F30700A4002000050020004D
:1045F0006033B800D5F3070004C3B30004424000A1
:10460000C47F9F002900370075332200D5B79F0073
:104610000D58A30002003A0080342200D0B79F005A
:1046200014002000050020006033B8008FA8970018
:104630008100E900050033000402D0008582D20029
:104640000683D2008783D200F9FF37000800BE003E
:104650000A01BE00B6F307006F0060005FB197006B
:104660006240780010003700140020000500200090
:104670006033B8008C0178008301E9000500330045
:104680000402D0008582D2000683D2008783D20044
:10469000F9FF37000800BE000A01BE00A4F30700BE
:1046A000674060000043B000C07F9F004F7A9700D2
:1046B0000400FB00EFB0970033000700E10F40005B
:1046C00003003200AFB297008502E800A5B79F0053
:1046D0001FA897006800500090AF9F008FA8970018
:1046E000E480500081AF9F0063065600D0FF2F008A
:1046F0003FB197000090B900FFA1970000804100F2
:1047000063005000800F5600A4FF3A000D38A3004C
:10471000100032001FA297000400E0000D003400DA
:104720000006EB00EFB09700000220001600070023
:10473000E10F400003003200AFB297008502E800AD
:10474000A5B79F000C06E8001FA09700800F560039
:10475000F4FF3A007FB19700B2407800F2B79F00B3
:10476000C17F9F000104E00014FB3A002FB09700C6
:104770004F0778004F06BE004F05BE004F04BE0035
:104780008F03B10000000600889FBE000001780082
:1047900001047800B10090000118A3003D00320030
:1047A0000198A30003003A00180090000000E00008
:1047B00038003A000190A00031049800820478008B
:1047C000F90FB200180090000000E00002003A006B
:1047D00028009000000C7800EA8F540006003A0090
:1047E000380090000078A30003003A0088007800A9
:1047F000D0002000E4FF07009800900058009000CF
:10480000808F50000B0032000100E8001004980077
:104810001800780009587800000C780011C0B30027
:104820000044220001487800EA8F5400060032005C
:10483000190037008800780009407800A2000700BE
:104840008004780014003700380090000088A3002E
:104850001100320018019000A8009000480090005C
:1048600005EF070098009000810F5000040032000F
:10487000380090000003B300300498008084EB00FF
:104880000000EB001004980028009000000C780055
:10489000010037008084EB00090078004F04BE005F
:1048A00000000600881F780000047800B000900027
:1048B0000148A30007003A000108A30005003200E8
:1048C0000198A30008003200100090000000E000F2
:1048D00005003200380090000040A000300498002D
:1048E0008080EB00200037000190A1003104980087
:1048F000180090000000E000060034000000E9000D
:104900001004980018007800B080FB00000C7800BC
:1049100006003700380090000068A300EDFF3A0061
:1049200008007800AB000700800078003800900095
:104930000078A3000C003A00FA8F500008003A00FB
:10494000280090000000E000E2FF32001800900014
:104950000000E80010049800180CE900DDFF3700A3
:10496000ED8F5000E2FF3200010078004F04780024
:104970000000060080017800E10F400017003200BF
:10498000310090000008A300140032000098A3003A
:1049900012003A00210290000400E0000F003200F3
:1049A0001101900051009000800F51000B00320067
:1049B00011007800840F500002003A008008E800DF
:1049C000020037000200E800900098001100E900A2
:1049D0008008780003487800010037008081EB00F0
:1049E0000300780000000600889FBE008A1F780040
:1049F0000004780030009000630060002400320062
:104A000008007800C10007003805900080EF2F00F3
:104A10000000650030049800280090000000E000CD
:104A200004003200E804650002003A00F0000700CC
:104A30002904980048009000C6EE0700E10F4000EE
:104A400013003200B80090000102B20010003A00DA
:104A50000AC8A30018003200E02281000000E00034
:104A6000150032000001780081047800012A20003E
:104A700012289000880F5000070032004205B00055
:104A80004905B000818F54000B003200F8FF370059
:104A90000080EB000900370002007800B6EE070046
:104AA000E0228100090040008000EB0011289800FE
:104AB00001007800010037000000EB004F0578008E
:104AC0004F04BE00000006000200FA00889FBE00EE
:104AD000A0FF9F0001047800B100900081047800DD
:104AE0000904B200020032000000FB00360037006B
:104AF0000118A30005003A000103B3003104980037
:104B0000190498000080EB002F0037005800900037
:104B10000000E00006003A0048009000120020006B
:104B2000E680570054EE070019049800240037006F
:104B3000280090000000E00008003A00C043220076
:104B400020049800000C78002000200050049800F9
:104B5000100498000130A000310498001801900062
:104B6000A80090004800900043EE07002800900045
:104B7000000C78000080EB0010049800180078000A
:104B8000AFF8970001587800000C78002FF89700D4
:104B9000EA4F50000A003A00380090000088A30055
:104BA0000700320018019000A80090004800900013
:104BB00031EE070019049800A8009000010C78005D
:104BC000AFF897000100FB004F04BE000080FA0020
:104BD000000006000200FA00889FBE008A1F7800CD
:104BE000000478000000EB001004980038009000EA
:104BF0008080EB000008A3003F0032000044220048
:104C00001004E00010003200C93522002A362200CC
:104C10001A0078006C0545002010B2002110200019
:104C2000810F500002003A000900780037000700A9
:104C3000EC84440000382200808F5400F4FF3A00D6
:104C4000004422000048EB0048009000580190000A
:104C50000200E0000D003A0012049800120020004B
:104C6000E88057004DEE0700E10F500003003A00C6
:104C70000FF897008080FB001F003700380090007D
:104C80000040A0003004980012003700A8009000F7
:104C900042EE0700100498000000E000030032001C
:104CA000E10F40000D003A0003003700380090008B
:104CB0000040A00002003700380090000003B3005D
:104CC00030049800A8009000010C78000000EB0070
:104CD000100498008080EB0007003700A8009000C7
:104CE000010C78000000E900100498000100780031
:104CF000B080FB00000C7800010078004F057800C0
:104D00004F04BE000080FA0000000600881F7800F3
:104D100000047800300090000008A3000700320073
:104D2000800078000120B20004003A0011049800CD
:104D3000A8009000010C7800170037000018A300AD
:104D4000190032000098A30017003200A80090005C
:104D50000100E00014003200180190000200E000A1
:104D60001100320048009000C3ED07009800900049
:104D7000810F500003003200380090000003B300A0
:104D8000300498000000EB00100498002800900008
:104D9000000C7800380090000058A3000200320098
:104DA0000080EB00010037000000EB004F047800AA
:104DB00000000600D12281000100E0000300320063
:104DC00011007800D0228900030037002000200065
:104DD0008BED070080007800E18F400002003A0070
:104DE000906E260010458800010078000000060043
:104DF000D122810001087800D0228900000006003D
:104E00000C070000574500004C4300004F4D0000C8
:104E100045200000746F00002074000068650000E9
:104E20002053000065720000436F00006D200000F9
:104E3000707200006F7400006F6300006F6C000000
:104E4000206F00006E200000652D000050750000EE
:104E5000636B00000D0A000074680000652000000C
:104E600045500000464C00002065000064750000BD
:104E700063610000746900006F6E00002072000022
:104E80006F6200006F7400002074000079700000F1
:104E9000652000002248000022200000666F00000C
:104EA00072200000686500006C7000000D0A0000B0
:104EB000006100002C250000642C00002564000027
:104EC0002C250000640D00000A000000612C000089
:104ED000302C0000302C0000300D00000A000000D3
:104EE000622C0000256400002028000025640000DA
:104EF00025250000290D00000A000000622C00009A
:104F0000256400000D0A0000004200002C2500006E
:104F1000640D0000006200000D0A00000063000044
:104F20002C250000640D00000A000000442C000045
:104F3000256400002C250000640D000000640000C2
:104F40000D0A0000006500002C250000642C000004
:104F5000256400000D0A0000004600002C2500001A
:104F6000640D0000006600000D0A000000670000EC
:104F700020490000522000006368000065630000C3
:104F80006B2000003A2000003078000025780000F7
:104F90002C20000061640000647200006573000052
:104FA000732000003A2000003078000025780000CF
:104FB0002C2000006461000074610000203A0000B1
:104FC0002030000078250000780D00000A00000065
:104FD000672C0000256400002C250000642C0000D4
:104FE000256400000D0A0000006700002C3000005E
:104FF0002C3000002C3000000D0A0000000A0000D8
:10500000002200004122000020200000202000009B
:105010002020000020200000202000002020000090
:10502000202000002041000063630000656C000048
:10503000657200006F6D000065740000657200000D
:105040000D0A000000220000422C00002322000074
:105050002020000020200000202000002020000050
:105060002020000020200000204200006F6400008B
:10507000792000006C65000064200000303D0000D5
:105080006F66000066200000313D00006F6E00007A
:10509000203200003D6900006E760000657200005D
:1050A000736500000D0A000000220000622200006B
:1050B00020200000202000002020000020200000F0
:1050C00020200000202000002020000020420000BE
:1050D00061740000746500007279000020760000A1
:1050E000616C0000756500000D0A000000220000E0
:1050F000622200002020000020200000202000006C
:10510000202000002020000020200000202000009F
:105110002042000061740000746500007279000094
:1051200020730000746100007465000020280000F6
:10513000313D00006F6B00002C200000303D00006E
:105140006C6F0000772900000D0A000000220000AB
:10515000432200002020000020200000202000002A
:10516000202000002020000020200000202000003F
:1051700020530000656C000065630000746F000040
:1051800072200000706F00007369000074690000F5
:105190006F6E00000D0A000000220000442C000089
:1051A000232C0000232200002020000020200000EB
:1051B00020200000202000002020000020530000BC
:1051C00065740000206D00006F7400006F720000B5
:1051D000207300007065000065640000206C000012
:1051E00065660000742C00007269000067680000AA
:1051F000740D00000A00000022450000222000007B
:10520000202000002020000020200000202000009E
:105210002020000020200000202000004765000022
:10522000742000006D6F0000746F00007220000099
:105230007370000065650000642000006C6500006C
:10524000667400002C72000069670000687400003A
:105250000D0A000000220000462C0000232200005E
:10526000202000002020000020200000202000003E
:10527000202000002020000020460000726F000067
:105280006E740000206C0000656400002030000097
:105290003D6F000066660000203100003D6F000099
:1052A0006E200000323D0000696E0000766500004F
:1052B00072730000650D00000A0000002247000024
:1052C00022200000202000002020000020200000DC
:1052D00020200000202000002020000020200000CE
:1052E00049520000207200006563000065690000FB
:1052F00076650000720D00000A00000022670000C1
:10530000222000002020000020200000202000009B
:10531000202000002020000020200000202000008D
:1053200047790000726F00000D0A000000220000A3
:105330004822000020200000202000002020000043
:10534000202000002020000020200000202000005D
:1053500020480000656C0000700D00000A0000008D
:105360002249000022200000202000002020000010
:10537000202000002020000020200000202000002D
:1053800020200000476500007420000063610000D9
:105390006D65000072610000207000006172000005
:1053A000616D000065740000657200000D0A000068
:1053B000002200004A2C0000232C0000232C0000B7
:1053C000232C0000232C0000232C000023220000AB
:1053D00020200000205300006574000020630000BE
:1053E000616D0000657200006120000070610000C6
:1053F000726100006D65000074650000722000009D
:105400006D6F0000646500002C7700006964000087
:10541000746800002C680000656900006774000073
:10542000682C00007A6F00006F6D000028310000CA
:105430002C340000206F000072200000382900008A
:105440002C780000312C0000793100000D0A00009A
:10545000002200004B22000020200000202000003D
:10546000202000002020000020200000202000003C
:105470002020000020430000616C000069620000F1
:10548000726100007465000020700000726F0000FF
:10549000786900006D6900007479000020730000D5
:1054A000656E0000736F0000727300000D0A00004B
:1054B000002200004C2C0000232C000023220000BE
:1054C00020200000202000002020000020200000DC
:1054D00020200000204C000065640000206E0000C9
:1054E000756D000062650000722C0000303D000008
:1054F0006F66000066200000313D00006F6E000006
:10550000203200003D6900006E76000065720000E8
:10551000736500000D0A0000002200004D2200000B
:10552000202000002020000020200000202000007B
:105530002020000020200000202000002046000045
:105540006C6F00006F72000020730000656E000039
:10555000736F0000727300000D0A0000002200004B
:105560004E2200002020000020200000202000000B
:10557000202000002020000020200000202000002B
:1055800020500000726F0000786900006D69000013
:10559000747900000D0A0000002200004F22000074
:1055A00020200000202000002020000020200000FB
:1055B000202000002020000020200000204C0000BF
:1055C000696700006874000020730000656E0000C9
:1055D000736F0000727300000D0A000000220000CB
:1055E000502C0000232C000023220000202000006B
:1055F00020200000202000002020000020200000AB
:105600002053000065740000206D00006F740000DE
:105610006F720000207000006F730000697400005A
:10562000696F00006E2000006C6500006674000069
:105630002C72000069670000687400000D0A000009
:105640000022000051220000202000002020000045
:10565000202000002020000020200000202000004A
:10566000202000002047000065740000206D00002D
:105670006F7400006F720000207000006F730000F4
:1056800069740000696F00006E2000006C65000006
:10569000667400002C7200006967000068740000E6
:1056A0000D0A00000022000052220000202000000D
:1056B00020200000202000002020000020200000EA
:1056C0002020000020200000205200006573000010
:1056D00065740000206500002D70000075630000F7
:1056E0006B0D00000A000000225300002220000081
:1056F00020200000202000002020000020200000AA
:105700002020000020200000202000005374000012
:105710006F700000206500002D70000075630000B0
:105720006B200000616E00006420000074750000B2
:10573000726E0000206F000066660000206C0000A2
:1057400065640000730D00000A0000002254000090
:105750002C23000022200000202000002020000038
:105760002020000020200000202000002020000039
:10577000506C000061790000207300006F7500001C
:105780006E640000203100002D350000206500000F
:105790006C73000065200000737400006F700000DF
:1057A000207300006F7500006E6400000D0A000099
:1057B00000220000742200002020000020200000B1
:1057C00020200000202000002020000020200000D9
:1057D0002020000020540000656D0000706500006E
:1057E0007261000074750000726500000D0A00000F
:1057F0000022000055220000202000002020000090
:105800002020000020200000202000002020000098
:10581000202000002047000065740000206D00007B
:1058200069630000726F0000706800006F6E000016
:1058300065200000616D0000706C0000697400005C
:1058400075640000650D00000A000000225600008B
:105850002220000020200000202000002020000046
:105860002020000020200000202000002020000038
:105870005665000072730000696F00006E20000022
:105880006F6600002053000065720000436F000047
:105890006D0D00000A0000002257000022200000C9
:1058A00020200000202000002020000020200000F8
:1058B000202000002020000020200000577200005F
:1058C0006974000065200000493200004320000098
:1058D000286D00006F6400002C72000065670000F6
:1058E0002C760000616C0000290D00000A00000009
:1058F000225900002220000020200000202000006B
:105900002020000020200000202000002020000097
:105910002020000052650000616400002049000062
:105920003243000020760000616C00003D2800003A
:105930006D6F0000642C0000726500006729000094
:105940000D0A00000022000041220000202000007B
:1059500020200000202000002041000063630000A0
:10596000656C0000657200006F6D000065740000DA
:10597000657200000D0A0000002200006222000093
:1059800020200000202000002020000020420000F5
:1059900061740000746500007279000020760000D8
:1059A000616C0000756500000D0A00000022000017
:1059B00062220000202000002020000020200000A3
:1059C00020420000617400007465000072790000DC
:1059D000207300007461000074650000202800003E
:1059E000313D00006F6B00002C200000303D0000B6
:1059F0006C6F0000772900000D0A000000220000F3
:105A00004322000020200000202000002020000071
:105A100020530000656C000065630000746F000097
:105A200072200000706F000073690000746900004C
:105A30006F6E00000D0A000000220000442C0000E0
:105A4000232C00002322000020200000205300000F
:105A500065740000206D00006F7400006F7200001C
:105A6000207300007065000065640000206C000079
:105A700065660000742C0000726900006768000011
:105A8000740D00000A0000002245000022200000E2
:105A9000202000002020000020200000476500009A
:105AA000742000006D6F0000746F00007220000011
:105AB0007370000065650000642000006C650000E4
:105AC000667400002C7200006967000068740000B2
:105AD0000D0A0000002200004722000020200000E4
:105AE000202000002020000020490000522000005B
:105AF0007265000063650000697600006572000051
:105B00000D0A0000002200004822000020200000B2
:105B1000202000002020000020480000656C0000CC
:105B2000700D00000A000000224B0000222000003F
:105B30002020000020200000202000004361000001
:105B40006C69000062720000617400006520000052
:105B5000707200006F780000696D000069740000C9
:105B600079200000736500006E7300006F72000002
:105B7000730D00000A000000224C00002C230000DE
:105B80002C23000022200000202000004C65000093
:105B9000642000006E7500006D62000065720000F8
:105BA0002C3000003D6F00006666000020310000D0
:105BB0003D6F00006E200000323D0000696E000065
:105BC0007665000072730000650D00000A00000099
:105BD000224D000022200000202000002020000094
:105BE00020200000466C00006F6F00007220000053
:105BF000736500006E7300006F720000730D00008B
:105C00000A000000224E0000222000002020000098
:105C10002020000020200000507200006F7800005B
:105C2000696D000069740000790D00000A00000031
:105C3000224F000022200000202000002020000031
:105C4000202000004C6900006768000074200000FC
:105C5000736500006E7300006F720000730D00002A
:105C60000A000000225000002C2300002C2300001A
:105C70002220000020200000536500007420000056
:105C80006D6F0000746F000072200000706F0000E4
:105C900073690000746900006F6E0000206C0000E2
:105CA00065660000742C00007269000067680000DF
:105CB000740D00000A0000002251000022200000A4
:105CC0002020000020200000202000004765000068
:105CD000742000006D6F0000746F000072200000DF
:105CE000706F000073690000746900006F6E00003F
:105CF000206C000065660000742C000072690000D2
:105D000067680000740D00000A00000022520000C5
:105D10002220000020200000202000002020000081
:105D2000526500007365000074200000652D0000BE
:105D300070750000636B00000D0A00000022000077
:105D4000532200002020000020200000202000001E
:105D500020530000746F000070200000652D0000CB
:105D600070750000636B0000206100006E6400002D
:105D700020740000757200006E2000006F66000045
:105D8000662000006C650000647300000D0A0000CE
:105D900000220000552200002020000020200000EA
:105DA000202000002047000065740000206D0000E6
:105DB00069630000726F0000706800006F6E000081
:105DC00065200000616D0000706C000069740000C7
:105DD00075640000650D00000A00000022560000F6
:105DE00022200000202000002020000020200000B1
:105DF0005665000072730000696F00006E2000009D
:105E00006F6600002053000065720000436F0000C1
:105E10006D0D00000A000000692C000025640000E0
:105E20002C250000642C0000256400002C250000B7
:105E3000642C0000256400000D0A0000004A0000E8
:105E40002C250000642C0000256400002C25000097
:105E5000642C0000256400002C250000642C000048
:105E6000256400000D0000006A0D00000A0000001B
:105E70006B2C00002053000074610000727400005D
:105E8000696E000067200000636100006C6900001B
:105E90006272000061740000696F00006E200000F3
:105EA0002D200000526500006D6F00007665000037
:105EB000206100006E790000206F0000626A00001F
:105EC0006563000074200000696E0000207300000C
:105ED000656E0000736F0000727300002072000096
:105EE000616E0000676500000D0A0000006B000095
:105EF0002C200000436100006C6900006272000009
:105F000061740000696F00006E2000006669000087
:105F10006E69000073680000656400000D0A0000EF
:105F2000004C00002C250000642C000025640000BB
:105F30000D0000006C0D00000A0000006D2C000038
:105F4000256400002C250000642C0000256400005E
:105F50002C250000642C0000256400000D0A0000C0
:105F6000006E00002C250000642C00002564000059
:105F70002C250000642C0000256400002C25000066
:105F8000642C0000256400002C250000642C000017
:105F9000256400000D0A0000006E00002C250000A2
:105FA000642C0000256400002C250000642C0000F7
:105FB000256400002C250000642C000025640000EE
:105FC0002C250000642C0000256400002C25000016
:105FD000642C0000256400000D0A0000006F000022
:105FE0002C250000642C0000256400002C250000F6
:105FF000642C0000256400002C250000642C0000A7
:10600000256400002C250000642C0000256400009D
:106010000D0A0000006F00002C250000642C000019
:10602000256400002C250000642C0000256400007D
:106030002C250000642C0000256400002C250000A5
:10604000642C0000256400002C250000642C000056
:10605000256400000D0A0000005000002C250000FF
:10606000642C0000256400000D000000700D00008D
:106070000A000000712C0000256400002C2500009F
:10608000640D00000A000000720D00000A0000000C
:10609000730D00000A000000542C0000256400006D
:1060A000007400000D0A0000007400002C250000A0
:1060B000640D00000A000000742C0000300D000088
:1060C0000A000000752C0000256400002C2500004B
:1060D000642C0000256400000D0A0000007600001A
:1060E0002C56000065720000736900006F6E00009E
:1060F000203100002E3200002E320000204100002E
:1061000075670000757300007420000032300000D5
:10611000303800002047000043740000726F000018
:106120006E690000630D00000A000000485700007F
:106130002076000065720000736900006F6E000039
:106140003A200000255800000D0A0000005700000A
:106150002C250000642C0000256400002C25000084
:10616000640D0000007700000D0A000000590000D7
:106170002C250000642C0000256400000D000000A8
:10618000792C0000256400002C250000640D00001F
:106190000A000000792C0000256400000D0A0000B0
:1061A00000250000643A000020250000640D000076
:1061B0000A0000007A2C0000436F00006D6D0000A3
:1061C000616E0000642000006E6F0000742000000B
:1061D000666F0000756E0000640D00000A0000008C
:1061E000536500006C650000637400006F7200006E
:1061F000207000006F73000020250000640D000077
:106200000A0000000C0700000A0A00000D570000F9
:10621000454C0000434F00004D4500002074000035
:106220006F2000007468000065200000707200009C
:106230006F7400006F6300006F6C0000206F00003F
:106240006E200000652D000050750000636B00009B
:10625000204200006C750000657400006F6F000044
:106260007468000020630000616C00006962000037
:1062700072610000746900006F6E0000000A000087
:106280000D5000007265000073730000204800008C
:10629000202800007265000074750000726E000016
:1062A00029200000666F0000722000006865000071
:1062B0006C700000000A00000D500000494E000004
:1062C000206300006F640000652000003D20000096
:1062D00025730000004F00002C250000730A000009
:1062E000000A00000D450000727200006F7200008D
:1062F000207700007269000074740000696E00006D
:1063000067200000504900004E0000004D2C0000A6
:10631000257300000A0000000A0D0000457200000D
:10632000726F000072200000777200006974000034
:10633000746900006E670000204E0000616D00006F
:10634000650000000A0D000046720000696500004B
:106350006E6400006C790000206E0000616D00002A
:10636000652000003D200000257300000053000060
:106370002C250000730A0000006500002D7000004D
:10638000756300006B5F000025730000000A0000C9
:106390000D5200006573000065740000206F00005E
:1063A0006B20000046690000726D000077610000FC
:1063B00072650000203D0000202500006400000000
:1063C0000A0D0000202200004622000020460000A6
:1063D00061630000746F0000727900002072000099
:1063E0006573000065740000000A00000D200000C5
:1063F000224D00002C4E0000616D0000652200005F
:10640000205700007269000074650000204E0000F3
:10641000616D000065200000666F000072200000C2
:1064200046720000696500006E6400006C7900002F
:10643000204200006C750000657400006F6F000062
:1064400074680000206E0000616D000065000000AF
:106450000A0D0000202200004E2200002052000001
:106460006561000064200000616300007475000035
:10647000616C00002046000072690000656E00003B
:10648000646C000079200000426C0000756500001B
:10649000746F00006F740000682000006E610000DF
:1064A0006D650000000A00000D200000224F000072
:1064B0002C230000222000005772000069740000A5
:1064C0006520000023200000504900004E200000FD
:1064D0006E7500006D62000065720000000A000029
:1064E0000D20000022500000222000005265000014
:1064F00061640000206100006374000075610000A9
:106500006C200000504900004E2000006E75000015
:106510006D62000065720000000A00000D2000009E
:106520002252000022200000536F00006674000019
:1065300020720000657300006574000020420000B6
:106540006C750000657400006F6F000074680000D7
:10655000206D00006F640000756C00006500000095
:106560000A0D000020220000532C0000232200000E
:1065700020570000726900007465000020230000AD
:1065800020500000494E0000206E0000756D000094
:106590006265000072200000616E0000642000004F
:1065A000736100006D65000020740000696D0000DB
:1065B00065200000652D000070750000636B000011
:1065C0005F230000000A00000D7A00002C43000049
:1065D0006F6D00006D6100006E640000206E0000B1
:1065E0006F740000206600006F7500006E6400008C
:1065F000002500006325000063250000643B0000C7
:10660000256400003B250000646D0000000C0000C4
:10661000075300007461000072740000696E00008E
:1066200067200000636100006C6900006272000076
:1066300061740000696F00006E2000002D200000D2
:10664000526500006D6F000076650000206100005B
:106650006E790000206F0000626A00006563000030
:1066600074200000696E000020730000656E000059
:10667000736F00007273000020720000616E0000F2
:10668000676500000D0A000000430000616C000017
:106690006962000072610000746900006F6E0000A2
:1066A00020660000696E00006973000068650000E4
:1066B000640D00000A0000000C0700000025000027
:1066C00063250000634800000D0A000041430000FC
:1066D000434500004C450000524F00004D4500006E
:1066E00054450000520D00000A25000063250000FB
:1066F000633200004B250000346400002C200000B1
:1067000025340000642C00002025000034640000C3
:106710000D0A00000A000000534500004C4500002F
:10672000435400004F5200000D0A00002563000092
:1067300025630000324B000025320000640D00008C
:106740000A0A000000490000520D00000A2500005E
:1067500063250000633200004B63000068650000A1
:10676000636B0000203A0000203000007825000014
:10677000782C000020610000646400007265000055
:1067800073730000203A00002030000078250000DC
:10679000782C00002064000061740000612000007B
:1067A0003A20000030780000257800000D0A000033
:1067B0000A000000505200004F580000494D0000F0
:1067C0004954000059200000534500004E5300007A
:1067D0004F520000530D00000A2500006325000001
:1067E000633200004B250000346400002C250000BB
:1067F000346400002C250000346400002C250000C7
:10680000346400002C250000346400002C250000B6
:10681000346400002C250000346400002C250000A6
:10682000346400000D0A00000A000000414D000021
:1068300042490000454E0000542000004C49000031
:106840004748000054200000534500004E5300000C
:106850004F520000530D00000A2500006325000080
:10686000633200004B250000346400002C2500003A
:10687000346400002C250000346400002C25000046
:10688000346400002C250000346400002C25000036
:10689000346400002C250000346400002C25000026
:1068A000346400000D0A00000A0000004D49000099
:1068B000435200004F500000484F00004E4500007A
:1068C0000D0A00002563000025630000324B000024
:1068D00025340000642C000025340000642C0000E6
:1068E00025340000640D00000A0A00000043000087
:1068F000414D000045520000410D00000A250000F6
:1069000063250000633200004B5200003D2500006B
:10691000336400002C200000473D000025330000B8
:10692000642C0000204200003D250000336400007C
:106930000D0A00000A0000000C0700005745000087
:106940004C4300004F4D000045200000746F0000D4
:1069500020740000686500002052000053320000DF
:1069600033320000202D0000204900003243000097
:1069700020740000726100006E7300006C61000002
:10698000746F0000722000006F6E00002065000030
:106990002D500000756300006B0D00000A20000000
:1069A0003120000062790000746500002070000052
:1069B000726F0000746F0000636F00006C200000B5
:1069C000415300004C2D000045500000464C000093
:1069D0002032000030300000360D00000A000000B8
:1069E0000C070000574500004C4300004F4D0000CD
:1069F00045200000746F00002074000068650000EE
:106A0000205200005332000033320000202D0000DD
:106A10002049000032430000207400007261000031
:106A20006E7300006C610000746F00007220000043
:106A30006F6E0000206500002D500000756300009F
:106A40006B0D00000A2000006D7500006C740000E2
:106A50006920000062790000746500002070000069
:106A6000726F0000746F0000636F00006C20000004
:106A7000415300004C2D000045540000485A0000CE
:106A80002032000030300000370D00000A00000006
:106A9000256400002C200000256400002C2000004C
:106AA000256400000D0A000000430000616C000036
:106AB0006962000072610000746900006F6E00007E
:106AC00020760000616C000075650000733A0000DC
:106AD00020250000642C000020250000642C00000C
:106AE00020250000640D00000A000000467200002E
:106AF0006565000020660000616C00006C3A0000D3
:106B0000202500006C6400002C20000028250000D7
:106B1000642C000020250000642C000020250000CB
:106B200064290000202D00003E20000028250000E0
:106B30006C640000290D00000A000000536800008A
:106B40006F6300006B3A0000202500006C640000B9
:106B50002C20000028250000642C000020250000C7
:106B6000642C00002025000064290000202D000076
:106B70003E200000282500006C640000290D000064
:106B80000A000000287800003D250000642C000069
:106B9000207900003D25000064290000202D000020
:106BA0003E200000616E0000676C0000653D000043
:106BB000256600002C2000006C650000643D00008C
:106BC000256400000D0A0000000000006C65000054
:106BD0006674000020250000752C00002072000063
:106BE000696700006874000020250000752C000013
:106BF000206C000069670000687400006573000085
:106C000074200000257500002C2000006C69000035
:106C100067680000745000006F73000020250000BA
:106C2000750D00000A000000436100006D200000A7
:106C30006C6900006768000074200000256C00008B
:106C4000750D00000A0000000A0000000A000000A4
:106C5000050000000000000000000000FBFF000035
:106C6000F6FF0000F6FF0000F6FF0000F6FF000050
:106C7000FBFF000000000000000000000500000015
:106C80000A0000000A000000256400002C2000001B
:106C900000730000657400007370000065650000FB
:106CA000642000002564000020250000640D000021
:106CB0000A0000007370000069720000616C00003F
:106CC00020250000750D00000A0000004C6F000038
:106CD0006361000074650000207300006F750000A0
:106CE0006E6400000D0A000000720000693A0000A6
:106CF000200000002533000064200000000D00008B
:106D00000A6C0000653A0000200000000D0A000037
:106D1000626100003A2000000000000025640000CD
:106D20002C20000000200000636100006C6900005E
:106D30006272000061740000696F00006E20000044
:106D4000646F00006E6500000D0A00000000000086
:106D500006000000260000001F00000012000000D6
:106D600027000000180000001C0000002D0000009B
:106D700041000000FD000000E500000032010000BD
:106D80008B0200001E0200004400000024FF0000EF
:106D9000B8FE0000BDFE00003DFF000027FF000020
:106DA0003DFE000026FE00009EFC0000DCF9000015
:106DB0003BFE0000C908000044100000D60E000091
:106DC0009405000033FB00005FF600008FF7000021
:106DD0008AFA00008AFB0000A3FA0000A1FB000071
:106DE00021010000E7080000A60D00001A0C0000B9
:106DF000BB03000046FB0000A9F80000D3F9000027
:106E000037FD00004AFF00005AFE0000C3FD0000ED
:106E1000D6FF0000F90300002C060000D801000096
:106E2000D0F8000029F80000CF030000FF0F000099
:106E30007F110000D406000014F9000088F2000061
:106E4000DDF5000006FD00007A0000009FFD000057
:106E500059FA000033FD000016060000D30D0000B3
:106E6000B20D0000EC04000025F9000007F5000059
:106E70009BF8000020FF0000150300000001000047
:106E8000ADFD0000E6FD0000A7020000270700009E
:106E90008703000013F7000027F100003DFD00000C
:106EA000BD100000B41900009E100000F7FD0000A6
:106EB000C3F00000D8F000003FF900003BFF0000E5
:106EC000B2FC000016F7000030F80000C601000018
:106ED000A20D0000211300003A0D0000A5010000E2
:106EE000ACF8000082F5000006F9000051FD00003A
:106EF00048FD000002FB0000F7FA0000C9FF000097
:106F0000D70600002E0700001AFD00004BF6000017
:106F10002DFF0000980F0000D21600009B0D00000E
:106F2000A4FB000013EF0000A5EF00005FF80000D5
:106F300010FF00009EFD000076F900007DFA0000C1
:106F400021010000390B0000B112000050100000B8
:106F50001006000049FA0000BBF20000EDF300004B
:106F600083F9000095FC000066FC0000C6FB0000F1
:106F700015FF00003005000078040000BEFC000092
:106F800022FB00003006000051130000BE13000079
:106F9000BF050000A0F40000BEEC0000CBF0000034
:106FA0003BF9000017FD00004FFA000009F900004E
:106FB0007CFC00008E030000790D0000DB12000055
:106FC000470E0000C7010000C8F40000B1EF000048
:106FD000E5F300002CFA000026FC00001DFB000079
:106FE000D7FA00005E00000017060000D401000080
:106FF00011FA0000F6FC0000120C00003617000029
:107000009511000010FF000067EE0000E5EA0000A7
:107010005EF200002AFB000032FC0000ABF800002A
:1070200087F900007BFE000027080000981300008D
:1070300000160000000D0000C8FD00004CF000002C
:1070400057ED0000C0F30000E1F90000CFFB0000A5
:1070500077FA000065FC00001D040000980600009F
:10706000EA00000094FD000044070000B414000092
:107070008D1400003204000080F0000075E800006C
:1070800049EE00001DF90000DEFD00009AFA000044
:10709000F2F9000009FE0000EC0400007A0F000085
:1070A0007C1500000D1200004C050000EBF4000000
:1070B000D3EB00000FEF000015F70000E4FB000029
:1070C000D8FB0000D8FA00008D0100005C0700002A
:1070D00079050000EF010000450600006B1100007B
:1070E000D1130000D40600006DF3000041E9000058
:1070F00040ED00005DF8000088FF000070FD00001A
:107100004BFC00005EFF0000FE020000F1090000E1
:10711000DC110000FA1500000A0F0000D5FD000088
:1071200021EE00002AEB0000E7F2000006FB000061
:10713000A4FD0000DFFA000071FE000098050000C9
:10714000CC0800008A0A0000B80B0000F50E000011
:10715000D40D0000020300002AF400008CEC0000B3
:107160009FEF000020F8000077FF0000FEFF000006
:1071700050010000CA030000EE01000010020000F0
:10718000E7090000AB160000BD180000FF08000072
:10719000DAF20000B5E7000046ED00000DF900004E
:1071A000A0FF00002CFC000085FA00008601000012
:1071B00060080000780F0000D9120000E8100000FD
:1071C000AE0A0000BFFE0000DAF2000031EE00005F
:1071D00047F2000040F8000091FD0000F3FE0000BF
:1071E000C802000089080000940500002800000083
:1071F000BF0100003A0F0000181A0000DB11000068
:107200000CFB00008EE800002AE800005FF400009C
:10721000DEFF00009BFF0000BCFA000037FE00000C
:10722000FE030000EB0A0000D31000003C13000036
:10723000EA1000000C05000059F5000042EC0000C7
:107240000FEF000001F60000C1FB000026FC00006B
:10725000D9FD000011060000B90800001108000067
:1072600034070000850A000086100000630C00004F
:10727000C9FC00000AED0000CEE90000BEF10000EC
:10728000FDFC0000530100005CFF00000102000053
:10729000AF02000067020000190700002D0F000078
:1072A000E31500001C0F000057FC0000ECEB000091
:1072B000C0E9000065F2000030FB00001DFD000089
:1072C00016FA0000C4FF00004F0700003809000054
:1072D000070B0000A90B0000E90D0000950B000052
:1072E00065FF0000EBF00000FFEA000058EF00002F
:1072F000C1F7000087FE0000B8FE00005D0200003C
:10730000B70600000A040000F7020000590600005A
:10731000CA0F0000251400003C0800002FF40000F4
:1073200050E80000D7EB0000A7F60000A7FE000021
:1073300024FD000006FC00002303000023060000DB
:10734000430700009D090000110E0000B611000067
:107350004C09000040F800004DEB000001EB00007C
:10736000C6F2000032FB000078FD000085FD000041
:10737000D4040000FF07000041070000CF08000010
:107380000E0B0000F60E00007A0A0000B5FB0000AC
:10739000D3ED0000E9EA0000FFF1000027FB000048
:1073A00001000000B6FE00002D03000008070000E9
:1073B00058030000DC020000870700005F11000096
:1073C0001014000081060000F5F20000ADE8000096
:1073D000EEEC00008BF70000F8FE000096FD0000C8
:1073E000F4FD0000C7050000D1070000E20700001F
:1073F00046090000900C000027100000C1080000A2
:1074000011F900009EEC0000D1EB0000C4F3000075
:1074100047FD0000D1000000D4FF0000300500004F
:107420001807000097040000A60500008908000066
:10743000AB0E0000810E00005902000019F300009D
:1074400026EC00008FF00000F5F90000820000003B
:10745000FEFE0000DEFF00003C0500001A040000F4
:107460002C030000BF060000330E0000891300004B
:10747000FB0B0000CFFA0000E0EC000072EB000014
:10748000C3F3000016FD00008DFF00005FFD00004B
:10749000AF020000D60700002F060000E60500003E
:1074A00039080000E00C0000640D0000DA03000061
:1074B000DAF50000DFED0000B3F0000038F900005D
:1074C0001D000000FFFE00002AFD00004102000038
:1074D0009D0300000A030000EB060000B70B00004C
:1074E0001F0F0000FB0B000066FF0000BAF2000057
:1074F00083EF00006CF40000C2FA0000A5FC00005D
:107500007BF900003BFC00008A05000096060000A5
:10751000C403000037060000310C00006D100000AD
:10752000C00A0000B8FB000080EF000016EE00006B
:10753000E0F4000092FB00004CFC0000F1F80000B9
:10754000B2FD0000C50700004C0700000A03000060
:1075500077040000540B00007D100000CC090000EF
:10756000CBFA0000F9EF000099EF00001DF60000D3
:1075700040FB000068FA00005AF700008AFD000096
:107580002E0800005808000017040000B104000095
:10759000440A0000750E0000220900002DFC0000C6
:1075A00072F10000E1EF00005BF50000CCFA000092
:1075B000A4FB00007DF90000E6FE0000D9070000F2
:1075C000E50600005602000080030000C909000023
:1075D000F30D0000DC09000001FF000081F5000050
:1075E0000DF2000028F40000A3F80000CCFA00001F
:1075F000B5F90000AEFD000075060000E6060000CB
:1076000065010000C50100003D0A00003D110000B9
:10761000BD0E0000E901000093F4000077EF0000C8
:1076200062F200005EF8000069FA0000F9F800005C
:10763000CCFB00002D070000240D00008806000090
:107640001B010000A7030000BA0800001D0C000089
:10765000650700009BFB00005EF20000DEF000000A
:1076600054F7000074FE000031FF000046FB0000EC
:107670006AFE0000C0040000EC02000087FF00006A
:1076800082040000090E0000AA120000530E000040
:10769000A5000000E8F3000011EF0000E6F1000093
:1076A000A7F7000032FA000003FA0000A0FE000075
:1076B000450A0000F90C0000DE02000024FD000075
:1076C00040040000490E0000DA1000006E080000BF
:1076D000F7F90000D3F00000A0F00000F5F600007C
:1076E000DAFC000072FD0000C0FB00005401000045
:1076F000C50A0000180800004AFE000030FD000026
:1077000026070000DE1000009D1100002907000080
:10771000A1F800007BF0000003F20000D2F80000A6
:10772000C1FB0000FAF90000F6F900007F04000038
:10773000CB0E0000F6080000B9FD000063FE00005B
:10774000EC080000F40E0000510C00007402000070
:10775000CEF70000D6F200000BF5000088FA00001A
:10776000C6FB0000BBF9000037FA00002905000045
:107770001A0E000084050000F1F9000087FD0000EA
:10778000C30C00001E150000580F00000D00000083
:10779000D0F2000083EF000057F40000C2FA0000AE
:1077A00009FB000091F80000E6FA0000E507000080
:1077B00037110000E205000067F60000EEF8000057
:1077C000740B00009A170000B6110000ECFF0000D7
:1077D00001F10000D2EE00004AF500006EFB00004F
:1077E000FFF9000037F6000076F900006C08000091
:1077F00045140000EB08000002F50000AAF30000A9
:1078000002070000D91600003A130000F80100003A
:10781000BAF20000DCF00000C8F70000EDFC000048
:10782000F1F90000E2F3000013F50000520300003C
:10783000E1120000550C00006AF700001FF2000082
:10784000180500005819000054180000B00400008A
:1078500047F0000036EB0000F0F30000BDFD000033
:107860003BFE00006FF600008BF300005AFE0000A4
:10787000171200006D140000B0FD000037EC00008E
:1078800004F7000036110000AC1B00007D0F000063
:1078900005FA0000DCED0000A2F200000AFD000085
:1078A000B3FF000072F600000DEE0000FCF30000D4
:1078B0002F090000601A0000750D0000E5F10000BE
:1078C000C6EB0000D1030000491C0000BA190000FB
:1078D0003403000013EF00003FEE000020FB000027
:1078E0002D03000042FC000031EE00006EEC0000B1
:1078F0006CFD000099160000E01A00009CFE0000DC
:1079000031E5000013EE0000BD100000E22400008D
:107910009B160000D5F9000006EA000096F1000071
:10792000290100005E030000DBF4000075E70000A1
:10793000B6EE0000BE070000881E0000CE16000054
:1079400016F300004DDF000070F40000E01A0000A4
:1079500031260000B50D000023F00000D2EA00003F
:10796000CFFC0000ED0A0000AC0100009CEA000022
:1079700069E00000DCF10000BF0F0000692000009A
:107980002F100000AFEA0000CFDC0000FDF900007E
:1079900019230000402B00007D0C0000AFEA00001E
:1079A000F3E8000021020000201100009100000017
:1079B000BAE20000EDD9000022F4000040180000F7
:1079C00038250000220E0000E2E5000034D9000056
:1079D0003BF900000A2500008C2D00008A0D0000F4
:1079E0008AEB000082EB0000DA050000F8120000CC
:1079F000E7FE000075DF00004FD800008CF40000A7
:107A00007D180000AE220000420D00004CE900008D
:107A100097DB00001FF7000094200000F22C00000C
:107A20003112000044F0000072EB00003A03000045
:107A30005B130000E902000015E30000C8D8000055
:107A4000B9F1000099150000611F0000E00A000074
:107A500086EF00008CE2000050EE00007F0A00007C
:107A600093200000261F00008D0C000032FE000055
:107A700097000000BC070000AFFF0000F0E8000026
:107A80001CDA0000B2E5000039030000E617000030
:107A90001A140000F803000004F5000015EF0000C0
:107AA00087F90000760D00008B1800004D110000D2
:107AB000BC0100006DFC0000110600004C0C000031
:107AC000ACFF000061E900000FE000008CED000059
:107AD00045050000C71100005B0C000090FF00008E
:107AE00042F300005CEF000073FC0000A9100000EE
:107AF000F9190000C01300008C080000D604000033
:107B0000F40500001B00000070F000003DE20000E2
:107B100057E4000095F60000260A00002D10000032
:107B2000550900000501000046F80000ACF2000015
:107B300099F900007B0B000051190000101600009D
:107B40003008000031000000B70200000903000007
:107B5000CBF7000005E90000E9E4000043F1000074
:107B600051040000D60D0000FD090000B3FD000027
:107B700030F10000D0F2000021060000961800004D
:107B8000D7170000C8070000B6FB0000CC000000BB
:107B9000DE0B000089080000DEF4000081E4000034
:107BA000A5E9000032FD0000140A0000F6050000FF
:107BB0002EFB000080F80000B7FA00008AFA0000EF
:107BC000F8FC000077080000D2130000DD1100006F
:107BD000D9060000750100002F070000070B000008
:107BE0004B0100004AF0000098E800007CF1000022
:107BF000E2FE000049020000CAFC000017FB000082
:107C00007B0100000E03000058F800009CF100000A
:107C1000C5000000ED170000E31A0000240A000070
:107C20005CFB0000C3FC000052080000440B000095
:107C3000D8FD0000D5EC000022EA000063F7000048
:107C400019060000F50600008BFC000048F5000056
:107C5000FEF50000FAF900007AFF00007509000047
:107C6000DE1200008211000097060000F3FF000002
:107C700041020000D902000036FB000055F200006E
:107C8000C9F200000AFE0000ED080000D60700005F
:107C9000DBFD000056F3000057F0000071FA000011
:107CA000C40900004F0E00000E0600007AFF00001D
:107CB0009A030000970B0000D609000011FB00009A
:107CC000E8EC00000BEE0000F4FB00002D090000C2
:107CD000C80B0000FA0500006AFF000026F800004B
:107CE00065F20000DCF70000B90600004612000053
:107CF000F91100005D090000B9030000DE02000078
:107D0000BEFE000081F30000C2E70000A7E700000C
:107D100080F6000001090000F60F0000230A0000B1
:107D2000A101000075F80000E9F20000EDF9000083
:107D3000C60B00006A190000E4150000F7070000F8
:107D40002B000000C6020000F20200008FF70000C6
:107D5000D8E80000FDE400008EF10000910400006E
:107D6000DE0D0000DA09000078FD000012F10000CD
:107D700000F3000080060000BE180000AB170000F2
:107D800082070000A2FB0000FF000000F40B0000CF
:107D90005808000086F400005FE40000E7E90000F6
:107DA0007DFD0000250A0000D10500000CFB00004D
:107DB00089F80000BAFA000085FA000017FD0000FB
:107DC000B0080000E8130000B8110000AE06000083
:107DD0007A0100004E070000000B000008010000BF
:107DE0000CF00000A2E80000ADF100002DFF000043
:107DF000EA020000EAFC0000DCF90000B9FF000024
:107E00004F0200007DF90000D8F300002D020000B1
:107E1000F016000018180000A50800005DFD000025
:107E20004B000000730900003E09000069FC0000DF
:107E300083EF000051EF00002EF90000BF000000AA
:107E40000CFE00001EF70000DFF700008AFE0000B5
:107E500023FF0000CFF900009BFD00007E0C000016
:107E6000851400008E0B000051FF0000A1FE0000F1
:107E7000650500002B0900005C05000036FD0000D0
:107E80001DF9000022FB000029FC0000D2F70000D1
:107E9000B1F10000CAF1000066FB0000DD04000043
:107EA000C8000000DDF60000B8FC0000AF0E0000C6
:107EB0000A1400007805000041F3000054F40000AB
:107EC000320A0000A6190000E310000047FD000080
:107ED0005FF60000BFFF0000880600001FFB0000E7
:107EE000A3E7000009E300008CF50000980B0000F8
:107EF0006C0D00000BFE000086F2000024F800006C
:107F0000520900006D100000CE00000089F2000050
:107F100028FA0000010E000044190000891000003A
:107F20006601000079FE00004D0500008D0500008F
:107F30000EF90000A9E9000072E60000C6F3000097
:107F40007103000056070000B000000032F9000085
:107F500095FA000090010000130800008C05000055
:107F600090FA000029F7000027000000680F0000C9
:107F70004C150000100E00004E040000940000009C
:107F8000E1040000F0070000670000000AF10000B3
:107F9000C7E8000091EF0000D1FC0000F0020000F3
:107FA000A5FE000037F900004BFA000055FF000065
:107FB000FE0100005C03000061020000CCFF000035
:107FC000090000005C0300000D08000086090000A5
:107FD000E0080000BB0500006A0200000704000082
:107FE000DE060000740400005AFE0000BCF9000028
:107FF00025F800008AF70000DBF5000059F40000C6
:108000001CFA0000420500001E06000005F90000F1
:1080100044F0000025FD0000E30C00005A0A0000B7
:10802000C7F80000D5F400007008000091110000AE
:1080300038060000F6FC0000D900000057080000D8
:108040000C0A0000C9050000210300000304000021
:108050004102000030FD000041F90000D2F50000AF
:1080600028F4000095F8000073FB000087FA000078
:1080700019FA00003FFB00000FFF00005F03000043
:10808000D006000036020000C1F700004DFA0000E3
:108090007F0800000F0C0000AB020000EE000000A3
:1080A000510A0000C90D0000B3080000C101000022
:1080B000EEFE00004E00000054FF0000FCFB00003C
:1080C00055FC00005F0000004AFF000035FA000088
:1080D000F7F60000F8F7000060FC0000E5FC000087
:1080E000C9FD00003400000038F9000030F700003E
:1080F000CA00000098030000EA050000B50900006E
:10810000910000005DFB00004E060000CD0D000058
:108110004E060000F7FA000082F900007B02000022
:108120007209000004040000B7FC0000F4FF000026
:10813000790500002D010000E4F8000004F90000BA
:108140000FFF000067FF000097FA00009DF9000094
:1081500021FC0000AEFD0000A9FF0000C8010000E6
:1081600041FF0000FAFB000000FD0000F8FF0000E6
:10817000F40300007B040000C3FF000013020000B2
:108180002A0800000F0800003E07000080010000E0
:1081900077FB000057000000F00400005BFD0000CA
:1081A0000CF80000AAFE00000D02000031FE0000E5
:1081B000DBF90000D0F90000C0FD0000B9FE0000AE
:1081C000BCFE000084FE000005F900004BFA000030
:1081D000AC020000D2020000700400004D08000054
:1081E000ED000000B9FC000075050000AC0B0000BC
:1081F000F6040000E0F9000004F80000F0010000BF
:1082000036090000F5010000E1F9000093FF0000CD
:108210007D070000F50100003BF800002AFC00008B
:108220009D050000E00100004FF9000078F9000012
:10823000FAFD000029FF00000100000095FF00008A
:10824000EAF70000B5F80000930300003E030000C9
:1082500094FD000039FD0000DBFD0000200300005C
:10826000950300002F01000010070000930000009C
:10827000DAF50000B2020000FD0E000020FD000053
:1082800022EF000023FD0000EE090000AB07000014
:108290004900000026FD0000600000005E030000B1
:1082A00031FF0000DEFB000065000000FF00000061
:1082B0005BFE000097FE00001BFF00000A010000AB
:1082C000470000006CFB0000C0FB0000D90000006C
:1082D000EB010000CFFE0000D2FD0000E102000033
:1082E00093030000AFFD00006CFA000050FF000097
:1082F0008306000074020000EEFD0000CCFF0000C9
:108300008E0000004101000033FF0000C8FB0000A8
:1083100069010000AB0600009EFE00003DFC00006D
:1083200048060000190A000026FE00004AF400007A
:10833000E1FD0000230B0000A6030000B0F50000E3
:108340001FFD0000100700006E03000058FF000032
:1083500020FF000017FE0000170000002C050000A1
:108360003504000088FF000016FD000063FE0000D9
:10837000AC0100003C0000001EFE00005DFF00009C
:108380006D000000C10100001B010000AC000000F6
:108390006D0200002601000089FE0000FDFE0000C5
:1083A00019FF0000BCFF0000FC02000026000000D6
:1083B00088FC000048010000AE04000067000000D7
:1083C000FAFD0000D3000000980100001700000033
:1083D000FCFB0000A0FE0000BE07000041030000FF
:1083E00077F7000041FB000063070000FF04000076
:1083F00002FC000067FF00002B030000500000009B
:10840000FAFD00000AFE000073010000F700000002
:1084100016FE0000AEFE00005FFD0000F2FC000052
:10842000550300000005000085FE00004AFD000025
:10843000B70100000802000067FF00003C000000D8
:108440005700000046FD000090FD000053010000B1
:10845000B402000037FE0000DFFC0000A0010000B5
:108460004E0200008AFE00007FFD00001C0200009A
:1084700090030000D5FC00003EFB0000CE01000090
:108480005005000097000000E6FA00003EFD0000E5
:1084900027010000610300009203000073FF000049
:1084A00026FB000065FD0000DD0300007F040000E6
:1084B0002DFE000010FC000009000000BDFF0000C0
:1084C00088FF00009FFF0000F6FF00001901000078
:1084D00002000000A9FD00002CFE00002A0200009E
:1084E0009A0100006EFE00002BFE000052FF00000B
:1084F000ABFF00007FFF000082FF0000440000008F
:108500004101000002010000A6FC000094FD0000F3
:10851000E30300000902000091FB0000FEF90000E7
:1085200045FD0000FD010000DB0200000900000025
:1085300058FF000036000000A40100005F010000A9
:10854000D8FF0000BFFC00002DFC00004CFD000027
:1085500069FD000015020000AB000000D9FC00001E
:1085600077010000C304000054020000A8FE0000D0
:108570004CFC0000E2FC00009D0000001A0000001E
:1085800053FE0000AA000000F30000009501000067
:10859000AE0100004BFC00004BFC0000000300009B
:1085A000AE010000E5FE0000E5FE000030FC00002A
:1085B000E9FE0000C50300003B010000DBFB0000FA
:1085C00098FC00005202000042040000A9FF0000D5
:1085D000C7FD00001C0200001402000075FD000031
:1085E00024FF000069030000D700000075FC0000B4
:1085F00057FD000078FF0000EA0000003402000090
:10860000DC000000020000004E000000D10000006D
:1086100036010000C4FE000062FD000024FE0000E0
:10862000BE00000017030000380200001D0000001B
:108630001DFD0000B3FE00005202000077010000A3
:1086400081FE0000B3FE000054020000B9020000E9
:108650004BFF0000C8FD00004D0100006E0300004C
:108660002DFF00007FFC0000F5FE0000640100000B
:108670007300000066FF0000A30100007D020000FF
:1086800006FF00003BFD000048020000B8030000A8
:10869000C7FD00000CFC00006FFE0000AEFE0000F5
:1086A0001AFE000005FF00003B000000430200002E
:1086B0003D030000520200005E020000D7010000EE
:1086C0001F00000092FE0000A8FE000064FE0000F3
:1086D0002AFD0000F9FE0000EF00000078FF000016
:1086E000FBFE000048010000F30100005400000000
:1086F0009C00000072000000BAFD000099FF00001D
:108700009F020000B3000000FCFD000058FF0000C5
:108710006601000097FE000011FD0000DDFF000073
:108720005302000036000000FCFC00004500000081
:108730009A0400006F020000ECFD000030FD000014
:10874000790100008A02000041FD000071FD000077
:10875000B4020000110200002DFE000073FE0000B4
:10876000F90100006C0200001AFF0000E7FF0000A2
:108770001C02000054FF000099FD000038010000B9
:108780005C02000009FE0000CCFC00007301000048
:10879000C40300009EFF00006DFD0000E701000023
:1087A000DD030000DCFC00009CF90000D3000000A9
:1087B0005C0400002FFF0000B1FD00003403000046
:1087C000D2040000A1FF000095FC0000EDFF0000B6
:1087D0000A02000033FE000000FC00003C00000024
:1087E000A5020000E7FF0000BEFE000039FF000008
:1087F0003AFF000000010000890100005BFF00005B
:108800001AFF000072000000E5000000C8FF000031
:1088100086FE000023FF00005D000000F6FF000060
:10882000A0FE0000C9FF0000F50000000E010000DE
:10883000ED00000012FF0000E5FE00004F00000008
:10884000410000007E0000007500000033FE0000C3
:1088500091FE00005D0000004CFF0000ABFE000038
:1088600066000000210100007CFF000054000000B1
:1088700004020000B200000097FE00000CFE0000A1
:10888000CCFF000097FF000026FE000045FF00001F
:10889000BA00000076FF0000EFFD0000F8010000C4
:1088A00077040000F4FF0000DDFD0000B8000000C8
:1088B0004B02000098FF0000D9FC000093FE00006E
:1088C000540000009DFF00001BFE00001AFF000086
:1088D0006C0200006D0200002B00000051FF000040
:1088E00082000000A600000010FE000034FE000020
:1088F0008C00000042FF0000E1FD0000FAFF0000D4
:108900007D01000083000000A8FE000005FF0000BC
:10891000340100001A0100007AFF000037FF000058
:1089200075000000F200000004FF0000B7FD000029
:108930006EFF00009F00000040000000C4FF000028
:10894000E5FE000047000000280200000A000000C9
:10895000ECFD0000A6FF000089010000610000009E
:1089600037FF000096FF00002D00000043000000CC
:10897000DAFF00000E000000FBFF00007CFF00009B
:108980002800000033010000F4000000A8FF0000F0
:108990003FFF00005F0000008700000080FF000034
:1089A0007AFF0000DE0000001901000091FF0000C6
:1089B000DEFE0000A4FF0000840000001F00000095
:1089C00017FF0000D7FF0000F4010000B301000012
:1089D00054FF00001D000000670200006F0100004E
:1089E0004FFF0000FAFE00001801000032020000F4
:1089F0008DFF00000CFE0000AF000000EA01000047
:108A00006DFF000021FE000078000000570200000A
:108A10007A000000A3FE0000720000009C0200002B
:108A20000B0100001DFF00009B000000470200003A
:108A300089000000C4FE000059000000B9010000D8
:108A4000AC00000004FF000001000000350200003F
:108A50000B010000E5FE000054000000B201000020
:108A600022000000F5FE000098FF00001601000043
:108A70000F0000007CFE000065000000EB0100001C
:108A80000F000000C9FE00006400000001020000A9
:108A90000301000097FE000046FF00009D0100005A
:108AA000D2000000F5FE000052FF00000E010000A1
:108AB00056010000F2FE00004AFE0000E300000044
:108AC000080100008CFE000087FE00004E00000040
:108AD0007B0000003CFF0000DAFE00007E0000008A
:108AE0003201000052FF000006FF0000C700000036
:108AF000F9000000A5FF00001EFF00000F000000AD
:108B0000B0000000120000002DFF0000CEFF0000AA
:108B1000060100007D00000069FF0000F0FF00007A
:108B2000B3000000490000005FFF000021FF0000CB
:108B3000550000006200000035FF0000CAFF000081
:108B4000ED0000004800000075FF00001500000067
:108B500015010000CE00000043FF000075FF00007B
:108B6000FE0000009200000079FF0000ACFF000052
:108B7000AF000000E800000058FF0000CCFE00003D
:108B800099000000B6000000D0FE0000ECFE0000DE
:108B900030000000F6FF000019FF000019FF000080
:108BA0005F0000009E000000E7FE000026FF0000BE
:108BB000C60000005D00000052FF000058FF0000EA
:108BC000E3FF00001B000000BBFF00004BFF0000A4
:108BD000A5FF0000340000001B000000CEFF0000D5
:108BE00096FF0000E2FF000078000000BCFF0000DC
:108BF000A5FE000092FF0000CB000000FDFF00007A
:108C0000FEFE0000B6FF0000A80000005D000000AE
:108C100090FF0000A1FF0000960000007900000016
:108C2000C1FF0000D8FF00003F000000AC000000C2
:108C300054000000BAFF000022000000CB0000003A
:108C40000F0000007EFF00006100000082000000B5
:108C5000FBFF0000D5FF0000EAFF00003B00000022
:108C6000F3FF000081FF00003C000000AF000000A7
:108C70002B0000000C000000530000007D000000ED
:108C800018000000B7FF00001500000054000000AD
:108C9000D0FF0000A0FF00004400000075000000AD
:108CA00016000000DBFF00003D000000BE000000D9
:108CB0005D000000CEFF0000CEFF00005A00000063
:108CC00091000000F0FF000075FF0000DFFF0000D2
:108CD0005B000000070000009BFF0000DAFF0000BF
:108CE0005A00000037000000D3FF0000F3FF00002F
:108CF0001D0000002C0000000C000000D9FF000047
:108D000005000000450000005100000003000000C5
:108D1000100000006A000000610000001F00000059
:108D2000DEFF00001B00000051000000EFFF00000C
:108D3000D1FF00003E0000005C000000FDFF0000CD
:108D4000D5FF0000380000006D000000200000008A
:108D5000DBFF00000900000007000000CFFF00005B
:108D6000E9FF0000FEFF000012000000FFFF00000E
:108D7000DEFF0000080000001A000000ECFF000009
:108D8000FBFF00005400000047000000E6FF000069
:108D9000E1FF00004A00000059000000E6FF00006B
:108DA000CAFF00004E00000080000000F9FF000034
:108DB000E1FF000043000000560000000200000038
:108DC000BFFF00000F0000003E000000F9FF0000A0
:108DD000CAFF0000F3FF00002C00000004000000A8
:108DE000D5FF0000E8FF0000150000002000000093
:108DF000E5FF0000D2FF00000500000011000000A8
:108E0000DFFF0000C7FF0000EFFF00000C000000C4
:108E1000E1FF0000C3FF0000EEFF000004000000BF
:108E2000D8FF0000C9FF0000E5FF0000FEFF0000C2
:108E3000E5FF0000C5FF0000DCFF0000EEFF0000C2
:108E4000DEFF0000D0FF0000D8FF0000E8FF0000B8
:108E500002000000EDFF0000DAFF0000D8FF000074
:108E6000A4FF000095FF0000B4FF0000B3FF000066
:108E7000C1FF000093FF0000CFFF000063FF000070
:108E800065FF000032000000B50100005E01000037
:108E900034FC000051FB000024040000E302000049
:108EA00002F9000019030000D0F6000010FA0000DB
:108EB00083120000E9FB0000B8FA00006D05000015
:108EC00000F50000D201000046170000470A00002C
:108ED00008DD0000D4F50000151F000086EF00003B
:108EE00092F80000B00D00002CF60000F90300001D
:108EF0007804000040090000B1F80000B3E9000068
:108F000094140000C207000081EB0000690100001A
:108F100066130000A8FC0000E8F700004B07000003
:108F200016F400000DFA0000C30C00002AFA00003D
:108F3000FDFD00005C0200004D0300005A0100002E
:108F400059F90000CA000000C4FF00002A00000018
:108F5000990100007E050000E6FE00001F160000DB
:108F6000DA0A0000FED10000E80900006D180000D8
:108F70006FE100009FFE0000990E0000FAFD000066
:108F8000890500008DF3000038EF0000111E00007D
:108F9000990800009DF40000860C0000240A0000DF
:108FA000170D000064FA00003DEE000012F2000010
:108FB00036030000600B00002BF60000D703000012
:108FC000B90A00000F010000CFFE000051FC0000B4
:108FD000BCFE00000BFA0000F5010000A007000035
:108FE000C4F30000990500005A0C0000CDF7000002
:108FF00081120000800000000AE00000DE00000096
:109000004909000054F90000C3FF00004CFF0000B4
:10901000690A0000A20C00002DF2000089FB00008C
:10902000600A0000420100006EFB000072020000B6
:10903000BA2000001E1B0000C2CC0000C5E20000E8
:1090400023200000A4EF0000BBF40000BA0D0000D4
:10905000A6010000BBF9000057F400006307000000
:10906000AF0E0000E70700007CFB0000FD050000DC
:10907000C213000027090000D3FE00003EEB0000F1
:1090800036F00000B80400000500000044FA0000BB
:10909000210100007F010000A4FC000005F2000097
:1090A00084010000671D000074020000C8F1000088
:1090B000BF010000AAFD0000C7FB00000A0100007C
:1090C00027060000B10A0000F4F7000076F2000065
:1090D0004BFF000028F90000DFFA000019FD000036
:1090E000FBFE0000CA04000024FA00007004000027
:1090F00089060000F201000008110000E0F5000000
:10910000B5FF00000E1B0000F0FC000023F900007A
:10911000CDF700006DEC00008DFC00005003000056
:10912000DBF90000E5FD0000FA04000036F900005C
:1091300080010000850A0000FDFC0000FB08000023
:109140000A07000066F5000061FF0000B1010000A1
:109150006EFB00005D0A000033020000D8F2000040
:109160008E000000F0F8000083F40000DD04000031
:10917000CC000000A2F700006004000054040000CE
:10918000F2F70000B6030000B60900009FFD0000E2
:10919000F1FD0000B70D00004C0E0000B40C000003
:1091A0004EF400001ADF00009AFC0000E7FD00000A
:1091B00031F80000F20A00009B02000038EB0000CA
:1091C000A90000008B0F0000C4FD0000310E00005C
:1091D000CD1D0000E0FE0000AF0300006A0D00009E
:1091E00079E50000E9EE00005104000040F30000C2
:1091F00052F900007309000047FC00002CF9000040
:1092000035F80000110D00003113000022FD0000B0
:1092100024080000C3FB000056FA000054050000BB
:109220007A010000120000006FFB0000D2FC000079
:109230005DF70000CDF800002CFF0000F5FE0000F7
:109240008BFB000042FC0000C9FB00007F0B00000C
:109250009E12000031FA00006DFF0000DF0A0000DE
:10926000AD000000470400008E0F0000BFF20000B8
:1092700024EF00004EFD000057ED000068040000E0
:1092800084070000A8FA00009E1000005F0500009F
:1092900031F20000AE0300002E050000B0FB00001C
:1092A000A6FD0000A7010000820D0000120B0000C7
:1092B00018F70000D6F9000027FD0000D7F70000DE
:1092C00075F900003502000074FE000075F400001E
:1092D000BD0D00006F01000010FC0000F90B000044
:1092E0009C03000088170000EDFC00004E110000F8
:1092F000D60400003ED300000206000091EC0000FE
:10930000FBF500007B0C0000E1F60000F503000017
:1093100058F100002E0C0000A327000005FC0000FF
:10932000C5F10000BA1600003107000086F4000005
:10933000610B000084DF0000FFEC00009B0C0000CC
:109340000AFC00003C040000D9020000A8FF000055
:109350008CF50000ED100000E20C0000BDEE0000F6
:1093600017F400008AFE000069060000DA09000018
:1093700044080000180A00002FF5000001E1000079
:10938000D9060000B8FE0000CDF60000E9FE00009E
:10939000FDF9000071090000F8F30000FD14000061
:1093A000991B00005EEE0000080C0000930800000E
:1093B0000FF60000C70100008BF9000020F7000045
:1093C00022FD00006BFB000057F6000003060000C2
:1093D000540D0000B6FA0000A8F80000BFFE00001F
:1093E00078FD000084080000F102000013F900007D
:1093F00099090000C70800007CFD0000DBFE0000AA
:1094000065FB000035F000004BFC00003508000053
:10941000BCF5000012F900007203000004FA00001D
:109420007D130000C80700008F07000043190000EB
:109430005FF700009D06000034EF00007AF00000A6
:10944000880B000039E4000043F90000AF10000071
:1094500067F7000025F300000E0800008D1D0000D6
:10946000FE060000AFF90000F00B0000A0FB0000BA
:10947000470300008401000033EA000001FC000003
:1094800018FD000045FD00009A0C0000C9FF000017
:10949000C0FD000058F900006FFD0000EC0E000058
:1094A0001200000099FE00002FFB0000A0FF00004A
:1094B0006411000028FD00003CF60000BCFD000027
:1094C0003FF800005FFB000046040000E1FB0000E5
:1094D000B4F90000FC0100003EF60000900E000010
:1094E000DC17000074FE0000D1060000830B0000B2
:1094F00056F8000094F8000006FD0000CAFB0000CA
:1095000077FF0000EBEF0000A7FF0000520800000B
:109510005DFE00006D07000061FD0000FBFF000024
:109520006105000006FD0000C0050000E70900001D
:109530001F00000011FB00001EFF0000F2020000EF
:1095400040FB00003AF300001EFD0000B3040000E1
:10955000BEF900001306000047010000EAEF00001A
:109560005B110000C8090000A8FA0000B913000050
:109570006B0E0000B6F1000080F20000B90300009D
:1095800062F600001DF60000BB020000BFFD0000F7
:1095900002FF000088F900005DF30000CA1B000014
:1095A0004D1800006FFD0000D70300009F00000071
:1095B000FF00000092ED0000CD070000FBFE000060
:1095C000CBDD0000B1120000C00B00007EF50000F2
:1095D000880A000087F30000110100004710000016
:1095E000FDF700008A09000035FE000083F7000047
:1095F000CC0B0000B0FF000029000000F7FF0000C6
:1096000071F10000C8F40000C6080000FDFF000072
:109610002CFA00004B070000AAF20000250C000005
:10962000221B00003CF900007FFE0000E0F4000077
:109630002000000008140000BBFE0000BCF7000082
:10964000D4EF000074F80000B005000039030000FA
:10965000400600004F0100003AFD000024FD00001C
:1096600037FE00005EFF000046020000A901000076
:109670009E0100008F0C000044FD000023F5000057
:109680004403000014F70000F5F500004E0500004B
:1096900048010000E2F90000F6060000F1FD0000BC
:1096A0000BF900005B14000053FC000031FF0000C8
:1096B00011160000D3010000EF01000070EE000061
:1096C00089F50000BFFF00005BF600009B0500006D
:1096D0005B00000000FC0000CB000000BCEF0000BD
:1096E00099FD00001E1B0000810700005D0E0000B8
:1096F0005B0400006CF500003CFA000010F500006F
:10970000DA090000A6F6000098EE00005A080000F2
:109710005F040000160200005E010000F0F000008F
:1097200021020000100F000050FF0000B2FE0000F8
:1097300054F90000DEFB0000BA06000056080000E5
:109740009CF90000BDFC0000BD020000C7F1000054
:10975000ACFE0000270200004DF8000023FD0000D1
:10976000E0010000CE000000BBFF00007A10000006
:109770009707000096FB000074030000D4FC000073
:109780004D05000022FF00008DF40000990200004A
:109790006DF90000F0F70000F0FF000085FF000009
:1097A00090FF00006402000019FC000033F8000084
:1097B0000B1100003C0800009BF80000C40F0000E3
:1097C000A404000047F5000014FE00005BFA00004E
:1097D00088FF0000CFFD000050F80000B2FB000041
:1097E000EA01000049010000FDFE000082FC0000CB
:1097F000D1F00000920B00005A110000E1FB0000C4
:10980000A508000093070000B4F9000071FD0000F6
:1098100077FE000061FB00000CFF00007FFB0000F2
:109820001DFA00000FFF0000370200007AFF000061
:109830009FFE0000B80100005EFD0000450500002D
:10984000A30800000DF9000080FF0000EC060000F6
:10985000930000006C0400007DFB0000D9F70000BD
:10986000F3FF000090F80000E40000005F04000037
:10987000BC020000AE060000B6FC000086FD000041
:10988000BDF8000020020000740B0000C3F70000C8
:109890000E020000AD0E00006BFE000098FD0000FF
:1098A000EDFA000081F60000EF0400005F02000006
:1098B00016FC00008301000082FD0000B1FD0000E5
:1098C00084070000A3FA000023F80000EA0E00005D
:1098D00084FE0000F1FA0000020A000011FB000003
:1098E000ADF9000088FE0000A7FF0000A6FD000003
:1098F000730300003B0B000022FF0000D5000000B6
:10990000A500000051FE00007E050000A3F6000047
:109910001AFE0000D10500007DF6000031FC0000B9
:10992000E8FF00001DFF000020010000B40100005E
:1099300064F80000A40000005711000064FD00005E
:1099400051000000A50F0000BCFA000054F900000F
:109950006EFD000017FB0000F500000071FA00002A
:1099600026F9000008FE0000310300000AFF000095
:1099700012000000EDF5000060F700005415000033
:10998000680600003CFE0000670C0000AD0000000F
:109990009DF9000069FF000063FC0000CEFC0000A0
:1099A00092FE0000AFF90000B3FB00003D01000093
:1099B00014010000CCFD00000A01000036FE00008A
:1099C000C3FD00008D0A00008D0400002FF9000087
:1099D0000C0600006F0600006F0100000A03000083
:1099E000F8F5000023FB00004D0000007BFA0000AA
:1099F0002CFE0000FAFE00008F030000680000004B
:109A0000A2FE000085FD000088FB00005D0B000049
:109A1000D4070000F0FC00002A0F00002E0A00000E
:109A2000FDF7000062FB0000C9F900003BFB0000ED
:109A300089FF0000EBFA0000DEFD00007607000061
:109A4000C6FC0000E3FF00000D01000059EB000020
:109A50000B0D0000C91700009BFB00002310000045
:109A6000520800005FF5000073FD00006DFB000070
:109A7000C0FA000065FD0000B0FE000071FD0000AE
:109A8000A101000058030000DCFC0000D60100002A
:109A90006AFB00001AF90000C71400003909000031
:109AA000A8F60000C5FF0000E3FC0000D50100009F
:109AB000D10300006BFF00005900000003FA000012
:109AC000E8FE000081000000EEF6000044FF000008
:109AD0001E030000C60000001AFE00007CFF00000C
:109AE0005D010000F9FA00007B0A0000D3070000C6
:109AF00032FC00002D020000FF010000C50700003D
:109B0000CAFC0000CEFC000081FD000050F5000002
:109B1000B0030000D5FC0000CDF80000D504000023
:109B200080020000FAFB0000B50000007CFE00008F
:109B30007BF00000F1080000301000006E02000011
:109B4000760C00006F00000014FB0000F3FB000027
:109B5000E2FA000008FC00001FFD0000B90300004D
:109B6000E1FD000087FC0000DDFF000002FF0000B7
:109B7000ACFB000058FF00006C04000083FA0000FA
:109B80003D040000E70B000065F600004BFE0000FE
:109B900070020000C5F80000DC030000B600000001
:109BA0006E010000290300007CFA0000BAFA0000F0
:109BB00056FD0000CFFF0000FEFC000081FF00000A
:109BC0004E01000001000000DC000000B8FE0000B3
:109BD00014FB0000BCFF00006E080000B40300008E
:109BE000F604000002FF000023FA0000ED0100006F
:109BF000D4000000E5000000780000005C030000D5
:109C0000CCFF00009BFB000069FD000031FA000062
:109C100093FC00009DFF0000440300004AFE00008A
:109C2000FD000000B2FB0000DAF80000DA0D0000D1
:109C30008006000055010000A60600007C0300001D
:109C40005BFE0000B40300001B0200007FF3000075
:109C50000100000034FF0000C7F80000030200000C
:109C600096FC0000F1010000ED030000CDFA0000B9
:109C700030020000A9FF000047F900008604000040
:109C80003F060000A5FD00001A08000011060000B4
:109C90002BF90000BDFF000003FD000087FE00005F
:109CA0006C030000B8FC0000D4000000310000008C
:109CB0004DFC000030000000BDFF000063FE00000E
:109CC000E5FF000093030000A3FC00002FFC000050
:109CD000CE0500003800000049050000070700001D
:109CE000B5000000740200002E000000B600000065
:109CF00075FB0000BAFF00005B050000E0030000F8
:109D000060FE0000EEFB0000C00000003AFA000018
:109D10004FFE0000A101000066FF00001D040000CE
:109D20000AFF0000FA0000004B000000E6F7000008
:109D3000000400005D090000E9FC0000890000004B
:109D4000F407000062000000C3030000E404000008
:109D50007EF6000042F80000B30100000CFE000097
:109D6000FCFD0000E9010000A9FD0000D003000097
:109D700094020000E9F8000021FE000095FE0000BA
:109D800030FE000069FE00008A0100004309000067
:109D9000BC0200006C0000004806000061000000EA
:109DA000FAFD0000F6FF0000C9FB0000E8FA000021
:109DB000E8000000FE00000009FD0000CCFF0000EC
:109DC000EF00000057FF000086000000CDFE0000FD
:109DD000B0FC00008DFF0000D0FA0000F8FE00008B
:109DE000AE0A0000600300007FFF00004002000098
:109DF000DFFD00007CFD00002C0000006BFC00007B
:109E0000BCFE000066030000940000009BFE000002
:109E10006DFE00002CFF000080FE0000EFFE000041
:109E2000CFFF0000FFFF000085FF0000E5020000FB
:109E3000B6FF0000FEFA0000B500000029FA00009D
:109E400074FF0000830B0000BBFE00004300000015
:109E50004E050000B5FB0000EEFF0000A1FF000072
:109E600084FC00000D010000C0FE000021FE000087
:109E7000BD0100008802000002FF00009AFE000001
:109E8000540000006AFD000024FF0000870100006C
:109E9000B80000003A010000C5FD000001FF00000D
:109EA00029FC0000F4F90000130C00008E0A0000E9
:109EB0004BFB0000B501000036FD000010F900006A
:109EC000B3FF00000BFC0000C2FF0000B60500005D
:109ED00026010000A2FF000024030000F4FF0000A0
:109EE00076FF0000E7020000E2FD0000AEFB00008C
:109EF0007800000075020000140000002EFE000033
:109F00009CFE0000DE00000095FF000007FD000041
:109F100080FF000025020000D20300000D010000B8
:109F2000F0FF0000F0FF0000C1FF0000750000001E
:109F300099FE000072010000C401000094000000BE
:109F4000ED0000006AFF0000C60000006C01000088
:109F50008AFE00006FFD000095FF00007000000009
:109F600068FF0000DA000000D701000032FF0000A7
:109F70008DFF000001000000D8FE000020FF00005F
:109F800090FD00003EFF000083020000140200006C
:109F9000F9FF0000C1FE00008B010000A5000000D9
:109FA000BFFF0000E20100000102000050040000B9
:109FB0009E00000060FB000043FD00000DFF00005C
:109FC00022FE000072FE0000080100002D000000CB
:109FD0009BFF000026000000FAFD0000CFFE0000FD
:109FE000670000008CFE000079FE0000E2FF000028
:109FF00041010000DD0300002F010000740100009A
:10A0000073050000D5FD0000A1FF00001302000051
:10A01000F9FA00008D0000001CFF000023FC000086
:10A020007600000071FF000050FF0000E9FF000013
:10A0300037FF00002CFF000049000000C5FE0000B3
:10A040006EFE000043000000D7FF0000B1FF0000DB
:10A050002F0100005F00000048FF0000B2FF000079
:10A06000B2FF0000B0000000A7FF00007201000076
:10A070001A020000F5FE00007B0100003000000025
:10A0800085FD00004E0100001C000000DFFE000006
:10A09000D3FF0000F4FF000086020000D7FE00009E
:10A0A000CEFD0000080200006800000092FF0000E2
:10A0B0006BFF0000A1000000370100006AFE0000F5
:10A0C000BD0000004300000056FE0000F901000042
:10A0D0007C000000FEFE0000B6000000D100000081
:10A0E000F0FF00003BFE0000F4FD0000C2FF000096
:10A0F0004E0200004C02000027010000CF000000CB
:10A1000043010000C3FF0000AAFE0000C6FE0000DD
:10A110002FFF0000520100009200000070FF0000BD
:10A1200050FF000073FF00000EFF0000F2FE000071
:10A130008C010000A200000050FF00003602000069
:10A1400070000000F1FD000057FF00000D0000004E
:10A1500099000000FCFF0000BDFF0000A700000008
:10A16000EBFF0000F6FE00007FFF0000A1FF0000F3
:10A1700003FF0000FBFF0000280000002EFF00008E
:10A18000F3000000CB00000039000000F2010000E5
:10A190009F0000007BFF000020010000C9010000BB
:10A1A000ACFF000096FF0000E00000001D00000072
:10A1B000F0FF0000030100002101000093FF0000F8
:10A1C00093FF0000C8000000ED000000D0FF000079
:10A1D00066FF0000FCFF00000A010000CE01000045
:10A1E00059FF00004AFF0000620100003C0000002F
:10A1F00047000000BAFF0000D8FE0000C6000000C3
:10A2000097000000ADFE000050FF0000B7FF000007
:10A21000AAFF00000D01000082FF0000670000009F
:10A220006702000019FF000069FF0000EC00000059
:10A230008BFF000097FF0000260000009700000041
:10A24000ACFF00005BFF000038000000C0FE000013
:10A25000BEFF00002B0100008FFF000085FF000003
:10A2600063000000B6000000DEFF0000C0FE00003A
:10A27000CEFE000043010000940100001000000029
:10A28000B9000000C2000000430000009EFF000073
:10A29000E8FE000090FE0000BD000000F800000095
:10A2A00099FF000097FF000030FF00001F00000032
:10A2B0004DFF00005FFF00001B010000BBFF00001E
:10A2C0003900000076010000D7FE000055FE0000B6
:10A2D000BAFF00002000000045000000AEFF0000B3
:10A2E0001C0000009200000087FF00000DFF00002E
:10A2F0009EFF00006BFF00004EFF000055000000B5
:10A3000096FF0000AFFF0000480100002D00000094
:10A31000F1000000C4010000CCFF0000F1FF0000CC
:10A32000C7010000100100002CFF000049000000E0
:10A33000BA000000D6FF00004E00000052010000ED
:10A340008B00000044FF0000140000000801000022
:10A350008F00000072FF00009DFF00004C00000015
:10A36000A20100001B010000A2FE00006E00000020
:10A370002B010000FFFF000059000000BDFE00009F
:10A3800082FF00003901000083FF0000D4FE0000BE
:10A3900095FF00003AFF0000A4000000F500000057
:10A3A00009FF0000A4010000BE010000DCFE000067
:10A3B000100000004600000045FF0000F9FF00000B
:10A3C00076000000E8FF00007CFF0000C3FF0000F3
:10A3D00029FF0000EAFE00005900000044000000D0
:10A3E00087FF00007FFF00006E000000BC0000003F
:10A3F0001600000010FF0000FBFF0000E701000056
:10A4000022FF0000F6FE00000A010000C7FF000066
:10A41000C9FF00004800000035FE0000B7FF000043
:10A42000D20100002AFF0000BAFF00005AFF00001E
:10A43000B5FF0000B801000033FF00007DFE000002
:10A44000FBFF0000200000007AFF000015FF000065
:10A4500065FE0000D1FE0000D0FF00004BFF0000B1
:10A4600072FF0000E6FF00001A0000009C000000E0
:10A47000E6FF0000B6FE000068FF00005300000089
:10A480001B000000B5FF0000CAFF0000E0FF000055
:10A490002B0000004B00000092FF000036FF000080
:10A4A000A4FF000099000000F1FF00005EFF000023
:10A4B000780000007B000000C4FE00009DFF00004B
:10A4C000AC000000DDFF000098FF000093FF0000DB
:10A4D000FF000000F3FF000045FF0000BA0000008D
:10A4E0005AFF000050FF0000C9000000E6FF000016
:10A4F000A2FF0000AE0000004C0000009DFF000025
:10A5000045000000F2FF00002200000039000000BA
:10A51000C9FF0000BE000000FEFF0000FFFF0000BA
:10A52000910000006BFF0000E4FF00002501000027
:10A5300092FF0000ABFE00000701000039000000A0
:10A5400014FF0000FE000000F3FF0000E9FE000021
:10A5500090010000A00000006AFE000081000000E1
:10A56000820100002500000021FF0000A200000081
:10A570009A000000250000009B000000D1FF0000B1
:10A58000DE0000006200000041000000A8000000A2
:10A5900051FF00008F000000B90000001200000011
:10A5A000880000005F0000008F00000050FF0000E6
:10A5B0004E0000006B0000009DFE00006B000000DC
:10A5C000170100003B0000001A0000007D000000A1
:10A5D0000200000038FF00003100000068000000A9
:10A5E000D8FF000065000000BA0000002E00000047
:10A5F000B8FF0000E9FF000011000000DDFF0000CF
:10A6000078000000530000004A00000065000000D0
:10A610009DFF000068000000520000007CFF000069
:10A620002A000000760000007DFF000071FF00009E
:10A63000C10000009F000000A4FF0000D6FF000042
:10A64000ABFF00007DFF00004A0000000600000094
:10A650005BFF00001800000056000000EBFF000048
:10A660001B000000EBFF00002EFF0000A7FF000012
:10A670005C000000E5FF00002600000099FF0000DC
:10A6800077FF0000520000002200000066FF00007B
:10A6900005FF0000F8FF0000570000001E0000004A
:10A6A0007800000091FF00001CFF0000A8000000DF
:10A6B0006800000008FF0000BFFF00001E0000004F
:10A6C00042FF000020000000BCFF0000C0FE0000B0
:10A6D000C7FF000025000000CFFF000090FF000032
:10A6E000BAFF0000B6FF0000BFFF0000C1FF00007E
:10A6F00087FF0000B1FF000050FF0000B4FF000022
:10A70000480000005AFF00008DFF0000FFFF00001E
:10A71000D6FF000080FF0000CFFF0000B9FF00005F
:10A7200037FF00003F0000002300000065FF00002D
:10A73000ADFF0000A4FF00009CFF0000AFFF000081
:10A74000B2FF0000DDFF000013FF0000EEFF00007D
:10A7500060000000D9FE0000B3FF0000F5FF00001C
:10A760003BFF0000DFFF0000F6FF0000C1FF00001C
:10A77000C4FF0000CBFF00004A000000F7FF00000C
:10A7800034FF00000500000039000000D2FF000087
:10A790000D0000003B0000001E000000FCFF000058
:10A7A0004900000030000000F7FF000043000000F7
:10A7B0005E0000006B000000610000002C00000043
:10A7C0005B00000041000000230000007900000051
:10A7D0005F000000F3FF0000600000007A0000004E
:10A7E0000A0000003C000000500000006200000071
:10A7F0005D000000430000008E0000002300000008
:10A80000F7FF0000960000002E000000EEFF0000A1
:10A81000630000006D0000005C00000051000000BB
:10A8200063000000530000007300000050000000AF
:10A83000FFFF00004E0000004E0000001F0000005F
:10A8400063000000600000004900000043000000B9
:10A85000470000003E000000120000002800000039
:10A860003A00000052000000600000005E0000009E
:10A87000430000001B000000200000004700000013
:10A8800017000000020000002A0000002000000065
:10A8900031000000FEFF0000120000001700000061
:10A8A000D6FF00001E00000022000000E0FF0000B4
:10A8B0001A00000024000000090000000D00000044
:10A8C000060000001B000000D8FF0000E4FF0000AD
:10A8D00037000000EDFF0000F3FF0000170000004C
:10A8E000E9FF0000F3FF00000A000000D5FF0000B0
:10A8F000CDFF00000C000000ECFF0000D2FF0000C4
:10A90000E8FF0000DAFF0000F5FF00000100000092
:10A91000BFFF0000CDFF0000E5FF0000CCFF0000FE
:10A92000F7FF0000EEFF00009FFF0000D5FF0000D2
:10A93000F7FF0000AFFF0000BAFF0000FAFF0000C1
:10A94000CEFF0000CFFF000007000000CAFF00009C
:10A95000C2FF0000F5FF0000DBFF0000C0FF0000A9
:10A96000E8FF0000D2FF0000C2FF0000F6FF000079
:10A97000B6FF0000ACFF0000E5FF0000A9FF0000EB
:10A98000C7FF0000F0FF0000AEFF0000B1FF0000B5
:10A99000D7FF0000BBFF0000B2FF0000C9FF0000AE
:10A9A000BFFF0000C4FF0000D7FF0000BFFF000092
:10A9B000C5FF0000D7FF0000CCFF0000D6FF00005D
:10A9C000C9FF0000C4FF0000DEFF0000E2FF00003E
:10A9D000D0FF0000DEFF0000DBFF0000E9FF000009
:10A9E00005000000FDFF000000000000F6FF000071
:10A9F000F0FF0000DEFF0000F2FF0000FDFF00009E
:10AA0000E1FF0000D8FF0000FFFF0000E7FF0000AB
:10AA1000F1FF000005000000FFFF0000250000001E
:10AA2000D6FF00003E000000A0FF000075FE000001
:10AA300015FF0000F00400003000000060F9000085
:10AA40003E070000F502000044F600004902000045
:10AA50001107000099FB000051FC000055050000A3
:10AA600087FE000033FE00005300000018FE0000C7
:10AA7000410200004EFE00000BFD00007FFF0000C1
:10AA800024020000ED0000000E1600001BF700007D
:10AA9000DDE0000030220000FA0200004FDF00007D
:10AAA0001F06000099100000FB040000B0E9000040
:10AAB00028F20000B4320000DEF400004AD20000A8
:10AAC000882500004A0A000095E80000BC0000004C
:10AAD000F30300000E0B0000F90D00003CDB00004A
:10AAE00067010000B21E00003FE90000A4EF000073
:10AAF0004C130000250E00001AE800005902000067
:10AB00007A0B00000FF6000018FC0000E9010000BD
:10AB100057000000ABFF00009E150000BAE80000DF
:10AB200067EF0000EA26000026F20000C0EB0000FC
:10AB30002A0C00008502000051FD0000F0FC00001E
:10AB400013FE0000230800009405000026F6000014
:10AB5000F4FF000025070000CFF80000DDFF000033
:10AB600068020000A2120000E902000011DE0000ED
:10AB7000E71400005F0E000018DF0000F90000007D
:10AB8000A10E0000E6FD000071F800005DF9000074
:10AB90002308000014130000B3FC0000EEF40000D2
:10ABA000610800003A060000F0F7000059FA0000C2
:10ABB0006C0D0000B50700009BFB00002EEE0000AE
:10ABC000620C000064060000EBDD0000DB100000FA
:10ABD000BA0800006EF900000AFF000058FF0000EC
:10ABE0004C0B00008EF200009A030000AF01000041
:10ABF00039FA000085060000860000007606000095
:10AC00003BF30000E3FF0000160B000020F0000003
:10AC1000B8FC000074040000DBFB000004FE000030
:10AC200078010000BAFE00002F0100005200000071
:10AC3000B6FB00004CFC00003EFE00008E09000048
:10AC4000600000001C04000018050000E7F0000090
:10AC500016030000350100000BF1000032FC00007B
:10AC600075070000D7FB000014F40000AD0C0000D5
:10AC7000EDF90000C8060000FD0A000023F5000001
:10AC8000720B00001F000000A0020000E50600009B
:10AC9000CDFA000035F80000B60B000001F7000007
:10ACA000F7E90000E60A0000040300009DF500003B
:10ACB0002CFF000093060000E7FE00008F0000005C
:10ACC00073FE0000FF0900001C070000A0FC00004C
:10ACD0007D020000E600000082FD000075FF00001C
:10ACE00092FF000059F40000170200002B0300003F
:10ACF0008CFB000095FC0000920800003AFF000069
:10AD00000CFE00002CFF0000E7FA00003C0C0000E5
:10AD1000E6F40000EA030000120B00008CEF0000D4
:10AD2000C10D00007101000048F10000670B000038
:10AD300085FA0000C5FB0000BA0300003E020000D7
:10AD40008700000002FD0000CAFF0000DC010000D7
:10AD5000470000000DFA000012050000A3080000E3
:10AD6000D5080000D40200005DF80000E1FD0000FD
:10AD7000D70A0000E8F700006DEF0000C70C0000E4
:10AD8000F6040000FBF4000005FC00000C0D0000C0
:10AD9000CCFA0000AE0500007913000072F5000047
:10ADA00084050000F90B00002800000081FB000072
:10ADB000C5FF0000070A0000FBF7000021EF0000BC
:10ADC000900900008B020000BBF10000E8010000C8
:10ADD0003B050000C8FF00009E090000970200002C
:10ADE000EAFC0000DC0A0000EAFE0000CBF40000F0
:10ADF0009F050000330600004AF7000010FE000027
:10AE000034000000550800003CF400002BF4000062
:10AE10005710000080F40000F5FE0000BC060000A2
:10AE2000D6F900000C0200005D03000038F60000B7
:10AE30001604000010060000AFF200002705000015
:10AE4000B6040000D2F90000D1FB00004503000069
:10AE500027010000FBFC0000CE010000D4FA000036
:10AE6000FE01000050FF000010FC0000040500007F
:10AE700009FF0000DE07000089030000CCF7000096
:10AE80001CF80000090F000081FA000058EF0000D4
:10AE900034090000EB030000FDFB000075F4000026
:10AEA0005C09000045FF0000330200006F0900004C
:10AEB000C10A0000400D0000EAE900005C03000048
:10AEC00018130000D9F10000E5ED0000780400003F
:10AED00004130000B1F5000031E50000641100002A
:10AEE000EC160000EBED0000DCF20000AF140000F7
:10AEF0007907000095EE00001F050000DF0B000041
:10AF000003FA0000ACFE000010FE000052F4000046
:10AF1000C2060000E80300005DF4000076020000B5
:10AF200058070000510200002BFB00000800000041
:10AF3000DC0900006E0100003EFA0000F4FE000093
:10AF4000F8010000030200007DFB000025FC00006A
:10AF50005E03000018020000DFFA0000FFFA0000A4
:10AF60005E0300002200000059010000F9FD00000E
:10AF70002F0C00009BF800003EF70000411100007C
:10AF800072F6000008FC0000490400000502000001
:10AF90001DFE000018F90000760600002E010000DA
:10AFA000F4F600001702000008030000B0FD0000E6
:10AFB0007BFB00001B030000FD0B0000BD02000036
:10AFC0000BEE0000E6FB0000E31B0000A5F3000011
:10AFD000E5E500006515000037080000C2EF00003D
:10AFE000D9F40000010E0000CD06000097F4000027
:10AFF0001A0B000022070000AE050000F0F8000068
:10B0000021FD0000D20A000076FC0000F9F60000E5
:10B0100093F50000030A000016060000CAED0000C8
:10B020009EFD00005B0D00007B0B0000F3FA0000AA
:10B0300071F70000DF1000008F030000E1F2000054
:10B04000590100003D0600002D000000F5F700004A
:10B0500011F80000610B0000F5030000F7F000009C
:10B06000DA03000072080000D2F9000099F700002E
:10B0700015110000450C00003CE9000041FF0000F4
:10B0800071100000A6F80000A6EF0000B606000050
:10B0900020080000A6FD000070F40000FA02000085
:10B0A000F31D00009AE30000BEF5000082200000BE
:10B0B0006DEF000047F2000030090000730500004A
:10B0C0005307000048F1000050FE0000960F0000FA
:10B0D000C7F400004FF10000B00700002B10000083
:10B0E00090ED00009A0200003610000043F40000CA
:10B0F00062FC000084FF00009D0E00004609000075
:10B10000CEE400006B0400007D1C00002FEB00006B
:10B1100077F00000571200002F030000E7F2000054
:10B120006EF90000CB0C000099020000E4F300006F
:10B1300052020000DE09000001FE00008EF800004F
:10B140001F160000BF02000058E10000641200005A
:10B15000DF1200002AD800009B000000941E0000AF
:10B1600057F00000F4F70000F20200004C1000005D
:10B17000AD0100009AFE0000B910000092F000003E
:10B18000CB0400006C0F00003FE50000220400002B
:10B19000B5170000A8E60000E80300006F0E0000ED
:10B1A0005FF700006AF3000025010000360C000084
:10B1B00025FC00002C13000097EC00006FFC000041
:10B1C00053200000EEDE0000E1F40000CC1500008A
:10B1D0006DFC00008DF60000250200009DFF0000C0
:10B1E0000A130000AB0100000EDE0000091E000083
:10B1F000740D000071D7000042060000F51D00002C
:10B20000C5F400000DE3000008130000EA0A000086
:10B21000A0E7000077F50000951100005409000038
:10B22000DCE20000CF05000011100000FAFA000077
:10B230005BFE0000A4000000950C000025F8000053
:10B24000A7FB00002E080000BFFC00001BFF000051
:10B25000EEFF000052FC0000ACFA0000B500000058
:10B26000F5FF000072FB00003D040000D5FB00006C
:10B270005FFE00003204000068F700005D1300006C
:10B28000F8F90000BDE80000D11900004E000000F0
:10B29000BAE80000100600006B0C00003FF7000049
:10B2A00090F40000FE08000066070000C2F30000F2
:10B2B00060FE0000BE060000D4000000BAF80000E6
:10B2C0009B04000063100000CAE8000026FA00009A
:10B2D000D21A0000A3EF0000B8E60000BE1A00007A
:10B2E000070400007AE7000038090000F9080000B0
:10B2F000F9FB00006F050000561800008EEF0000FB
:10B300005DF000001E1F0000A4F9000042E40000F0
:10B3100083100000B4090000A1ED000040FE000011
:10B32000FC0E00002B02000022ED00003909000095
:10B330008A050000DCF60000B4FC0000DF07000016
:10B34000761C0000B8E30000C2EC0000022B0000F5
:10B3500033F300009FD80000FF1D0000051000001F
:10B3600041E20000C005000025070000280A000097
:10B37000B80A0000AEF30000D0FF0000DC100000AF
:10B38000C3F9000011EC0000670F0000B2090000D3
:10B3900029F20000B1F800006A06000051FC00002C
:10B3A000E7F70000EAFF000013030000A806000012
:10B3B00055FA000084FE000038100000BA070000B3
:10B3C000D3ED0000C9010000661300002AF100005F
:10B3D0004BF40000F8100000680100001DF20000AE
:10B3E0001D010000FD060000D6FD00003DF9000033
:10B3F00042010000B803000086FE0000AEFB000022
:10B4000010060000260700008DF5000062FC000019
:10B410004E080000A1FC000010F60000010500002D
:10B42000760400007CFA000062FF0000390300008F
:10B4300073000000B4020000E2010000A2FE000060
:10B440006C0A00007EFF000089F000000704000085
:10B450009A0A0000C0F70000F3F20000EB090000B8
:10B46000E006000081EE0000F9FF0000610B000023
:10B4700068F60000B5F900005115000078080000DA
:10B48000C1E9000004000000CF11000076FB0000BD
:10B49000A0EE0000B8030000B00F000032F500007D
:10B4A0007CF30000D40C00006E05000052F2000096
:10B4B000D5010000050D00009C030000960000006F
:10B4C00013F7000085FC0000AE070000F5FF000048
:10B4D000D3F00000AEFA00007A1800002FF500004B
:10B4E00036EB0000D51400001F02000052E40000FB
:10B4F000CC1500008D2E0000A6D8000010E9000039
:10B50000942C0000B802000095DC000070F70000E9
:10B51000701E0000D5FC00003DDF00000F0A000097
:10B52000FC1D0000E3F2000015EE0000041800000E
:10B530004C000000AAEF0000B30D0000040700005B
:10B54000A9F20000E6FF0000C705000062ED000060
:10B55000DEFE0000760C000041F60000B0F80000AE
:10B56000E6080000B90E000086FC000044FC000064
:10B57000590800007F0100006AF8000086FD000005
:10B58000D5030000A3FF00007AFE00008DF8000044
:10B59000EC010000A906000038F4000077F9000073
:10B5A0005C0B0000A5010000DCFA0000F8000000C0
:10B5B000FDFC000048060000AA01000003F20000A4
:10B5C0000F0500004E0B0000B9F50000FEF800006A
:10B5D0003F0800002E01000059F90000E8FC0000BF
:10B5E0006C030000E302000079F80000DAFE0000BE
:10B5F0003009000015040000EFFD00002EFA0000E5
:10B60000CDFF0000C6030000D5FF000074F8000065
:10B610003E000000FB0A000056F80000D7F70000CB
:10B62000090700001F02000049F800005A0000004E
:10B63000241100001606000021F6000039FE00006B
:10B640004A070000B9FC0000E6FA0000BCFD00005B
:10B6500042FF00001F0800000CF800002CF800005A
:10B66000A50A00004BFF0000AEEC0000C20D000078
:10B67000B1270000DBED0000F4E50000AB13000093
:10B68000500E000090ED000044F00000540D00004A
:10B69000D7090000EEEF000013F400008718000047
:10B6A0008A060000BEEB000073030000400B0000A0
:10B6B0006DFA0000B6FC0000730F000095FF00005B
:10B6C000B7F000001B050000E204000054ED00008C
:10B6D000F6FA0000C40F0000BDF90000E5F3000019
:10B6E0007E090000EA0A00001C080000B7080000FC
:10B6F0002AFD0000CAF60000EEFF00003203000041
:10B700005BFC00002AF80000C4FF0000E70B00000B
:10B7100061FC000098EC000023000000490C0000D0
:10B720004BFB0000FEFA00002E0D0000D2030000CB
:10B73000CFF5000021FF00009B060000ADFF0000D8
:10B7400062F800008D00000039090000F9010000D6
:10B75000F9F8000071FC0000B3050000FD000000D6
:10B76000FCF70000E9FF0000BA0D000038060000F9
:10B77000A5EF000084F900006D0E000097010000A5
:10B78000DFF20000E4FB00007C0C0000B6050000C6
:10B790004FF3000040FC00000409000059000000C5
:10B7A00032FB000087030000CB0C00003D060000C8
:10B7B0002DF6000002FC0000BC0500009D01000009
:10B7C000BBFA00000FF60000190400001D0B00007A
:10B7D00055F7000088F50000900B00003E090000BE
:10B7E0003CFA0000AE010000F60D00001507000055
:10B7F0004EF300004AFA0000BC0A0000B20100004B
:10B80000E9F1000022F60000C10A00000B0600006A
:10B8100018F2000053F90000DA0E0000A908000039
:10B8200000FC0000030200002F0600005901000088
:10B83000A6F800006EFC0000A5050000F7FE000061
:10B84000E6EF000040FB00007E0C000096FE0000CA
:10B850002BF50000320200009A0C000048060000A0
:10B860000EFC0000DDFC0000AF0400001901000028
:10B87000F0F7000087FC0000AC0400003FFD000072
:10B88000CDF20000DF000000360A00007FFA000061
:10B89000AFF50000C4070000770D0000E4F90000D8
:10B8A000C9F50000BD060000060C0000CAFC00003F
:10B8B000B2F40000DB010000B7090000E2FC000068
:10B8C00063F0000002FE0000AD0B00004EFF000020
:10B8D000D2F4000081010000E90E00003F050000E5
:10B8E0002EF700000FFD0000820700001503000086
:10B8F0002CF90000ECF90000980400002505000078
:10B9000056F80000F8F80000CC070000C50500005C
:10B910003EFB0000480100003D0900004CFF000014
:10B9200066F5000064040000BB0E0000FAFC000095
:10B9300052ED000012FB0000D80E0000E4040000ED
:10B9400015F00000C3F70000A90E0000D4080000A5
:10B95000A1F90000EAFE0000470700001502000000
:10B960009BF8000018FD0000690500008EFE000035
:10B970000BF500008B010000560800008BF9000059
:10B98000B4F70000AE040000AC090000460200005D
:10B99000E3FB0000A5FF0000C204000030FE000031
:10B9A000A3F800004E0000008306000039FB0000F1
:10B9B000C8F200001A030000610800005EF80000F1
:10B9C000E4F70000F40A0000E20A000088F6000034
:10B9D000EAF80000DB090000270A0000DBF900009C
:10B9E00038F60000B1040000F8070000CCF80000B1
:10B9F0005DF00000730100000A0C000021FC000053
:10BA000031F30000F8030000940F0000ED02000085
:10BA100041F70000B9FE0000100900000902000013
:10BA200072F80000D6FC0000EA030000E801000004
:10BA30006CF9000063FA00004A05000024040000CD
:10BA40007AFB00008F00000034040000A5F900001C
:10BA50009EFA0000B80D0000851000001FF60000DF
:10BA6000A3EA0000B3010000661200000204000017
:10BA70004AEC0000CEF30000CA0F0000640A000088
:10BA8000F7F2000085FA0000060B00005E040000DB
:10BA900063F80000E9FB0000270500004A040000ED
:10BAA000F70400008D06000092FA000017F4000071
:10BAB000F2FE00004303000070FC0000F1F90000FA
:10BAC0008B000000DA07000087FF000040F800004C
:10BAD00056020000E812000001150000E8FC00001A
:10BAE000AAE9000079F30000420500007C0800008C
:10BAF0009E0000007EF7000092F90000960300000F
:10BB0000360900004604000046F80000E7F4000093
:10BB1000A9FB000058030000FB0600009F0C00007A
:10BB2000CE0A0000D6F9000005EE0000DCF50000AA
:10BB300002060000FE07000012FC00009FF9000052
:10BB40000805000010070000DEFD0000FDFE0000FB
:10BB5000080B00002D0B000090FB000031F20000EC
:10BB600054FC0000F10900004406000094FB0000B2
:10BB7000FFFA000079000000CAFD0000E5F60000B1
:10BB800053FB00001105000060060000DAFE000013
:10BB90006AFA0000EA0200003D11000008130000EC
:10BBA0005501000097EE0000E3EF000022000000C6
:10BBB000010A0000510400006DF900002EF9000098
:10BBC000B40200002E05000054FF000016FD000026
:10BBD000C3FE00007EFB0000CFF80000B4080000A8
:10BBE00053170000980800007CEF000003EB0000F2
:10BBF000C7FC0000C8090000650300009FF90000B1
:10BC000008FC0000E00300000F020000AAFE000094
:10BC1000570700005D0C000083020000D5F400000F
:10BC200044F200009CFE0000CD0A0000D109000093
:10BC300089FE0000B2F6000054FA0000DAFE0000AF
:10BC40003CFD00005AFC000010000000DA04000077
:10BC50001402000013FB0000960000002C0F0000EF
:10BC600094110000A601000066EF000061EE0000E4
:10BC7000D6FD0000300A0000F908000099FE00001F
:10BC80007FF500009CF7000034000000EE04000087
:10BC9000C40100001BFC0000E5F80000DA00000011
:10BCA0002C130000C713000058FE00001AEC00001F
:10BCB000ACED000040FF0000560A0000C303000086
:10BCC000A7F900006BF90000940100005305000083
:10BCD000B2020000DE020000F004000007040000D1
:10BCE0005DFD0000F7F4000029F7000037040000B4
:10BCF000A20C00005B080000BFFD0000A7F60000DA
:10BD00009CF4000040F6000015FD00006C060000E9
:10BD10005A0A000092030000BBF900000AFD00006F
:10BD20006C0C0000E313000086090000FAF5000027
:10BD300093EA000092F0000011010000920C000054
:10BD400002090000B6FD0000B4F7000018FA000078
:10BD5000AD0000007E0300009100000017FC000011
:10BD600066FC00006D070000DA110000DB0D00002A
:10BD7000AEFD0000F7EC00000EEA0000E7F6000060
:10BD8000C1050000490B0000A70700006401000086
:10BD900066FC000007F9000075FC00004607000083
:10BDA000E70E0000500C0000630200004BF800009A
:10BDB00093F300001EF5000092FB00006C040000ED
:10BDC00023080000690300009AFC0000FDF9000050
:10BDD000E3FB000059FE0000B70000003E05000034
:10BDE000760A00009A0C000042090000B900000029
:10BDF000E3F50000A4EE00007EF20000D5FF000095
:10BE000080090000250900009A030000AFFD000032
:10BE1000F0F80000FBF700007CFE0000CC070000FB
:10BE2000D00B00005D0800006501000014FD00005B
:10BE300097FB00000FFB000049FC000040FF0000E2
:10BE400077000000DDFD00006EFB0000CAFC000072
:10BE5000FEFF0000C2010000B601000083020000E6
:10BE600061060000330B0000CB0C0000DE06000072
:10BE700035FA000019EF00002AED0000AEF50000D1
:10BE800048020000380A0000C00A00000505000052
:10BE90003DFC000089F60000CCF80000F400000032
:10BEA000F5070000A90900006C060000A3010000CE
:10BEB000F1FD000000FC0000B0FB0000D1FB000021
:10BEC0002DFB000030FA000093FB0000CEFF0000C5
:10BED0002D040000CE0500001D0300009EFE0000A2
:10BEE0009FFD0000C1020000900A0000A60E0000A5
:10BEF000EB090000BDFC0000CBEE000048E90000AB
:10BF000050EF00005BFC000044090000670F0000D8
:10BF1000570C0000C903000033FB000021F70000AC
:10BF20000EF90000D3FE00008E040000340700006C
:10BF3000CE0600008B0400006401000064FD0000D8
:10BF4000ACF80000C7F4000042F400008FF80000D5
:10BF500047000000D3070000940B00009B0800007E
:10BF60006601000079FE0000B0010000D506000067
:10BF7000BC0800008F0300001FFA0000F4F100006D
:10BF800033EF0000BFF3000075FD00009B070000C9
:10BF9000AD0C0000740A00001704000036FD00001C
:10BFA00086F900007AFA00007FFD00009900000089
:10BFB000980300003B060000F60600007404000031
:10BFC000A3FF000053FA00004FF500006BF20000E1
:10BFD000BCF40000B9FC000063060000E20B0000A6
:10BFE000420A0000DB050000BA040000B9050000A9
:10BFF000EB050000E40300003CFE000045F60000F5
:10C000005DF0000060F0000083F60000DAFF000041
:10C010005B080000C80C0000F00B000035060000B3
:10C02000A3FD000046F70000E1F600000EFB000053
:10C030008F0000007C05000088080000A2080000B6
:10C04000050600008401000005FC000057F6000012
:10C0500012F200003BF20000FBF70000DA000000E3
:10C06000DB0800009A0B0000F6090000B808000089
:10C070002C080000720700003B0500001AFF0000BA
:10C08000B2F600005AF00000CDEE000062F20000AF
:10C0900034FA000040040000CF0C0000A00F0000A4
:10C0A0004A0C0000F9040000BAFB0000EFF40000A5
:10C0B000F7F30000E8F800006B010000250900001C
:10C0C000D20C0000050C000066070000EDFF000028
:10C0D000B5F7000050F100005CEF0000FFF2000037
:10C0E000B0FA0000C6030000370A0000270B00006A
:10C0F0000E0A0000240A0000F90900005E08000092
:10C1000059040000C7FD0000EEF5000028EF000014
:10C1100017ED00001CF10000CBF900003004000016
:10C12000AE0C0000F0100000760F00008107000048
:10C13000ABFC00008AF5000081F4000072F80000FA
:10C14000140000002A080000CE0C0000290C00009A
:10C150003B060000BCFD00000EF6000023F10000CD
:10C1600099F00000FAF40000E0FC0000E604000092
:10C1700046090000A2090000140900004909000056
:10C18000A509000030090000EE05000056FF000080
:10C190000AF7000073EF0000D1EB000017EE00007B
:10C1A00025F60000BC0100002C0C00006F110000FF
:10C1B000B6100000470A00008E000000BDF8000025
:10C1C000C9F5000077F80000A7FF0000E2060000B4
:10C1D0005F0A0000F00800003F030000ADFB000014
:10C1E000CFF400003DF10000E0F20000E4F80000B0
:10C1F000720000002106000073080000C108000062
:10C200005D080000E4070000A7070000BA06000070
:10C21000E6030000CCFE000011F80000E4F100008D
:10C22000DAEE000043F0000005F60000E8FE000032
:10C23000C90700002A0D0000040E0000650A000076
:10C24000B10400009D0000004EFF0000A5000000AA
:10C25000DC020000FD020000E1FF0000A0FA000087
:10C2600075F5000090F20000AAF30000EDF8000060
:10C27000860000005D070000D80A0000630A000085
:10C28000DF06000039020000CEFE00001FFE0000A5
:10C29000E4FF0000570200007F0300004902000095
:10C2A00003FF0000B4FA0000CFF600001BF5000009
:10C2B00091F60000E0FA0000730000005405000051
:10C2C0001008000010080000B0060000530600002F
:10C2D0002F07000095070000FE050000A7010000E1
:10C2E00026FB0000ECF30000C1EE000071EE000040
:10C2F00074F300007DFC0000500600007F0D00007C
:10C30000211000000F0D00002B050000C9FC0000EB
:10C3100037F800006CF800007CFC0000A002000070
:10C32000A4070000EF080000F1050000A0FF0000D6
:10C33000CAF80000F2F3000072F2000006F50000F7
:10C34000FFFA0000270200008D07000049090000E5
:10C35000B00800005C080000B1080000F50800000B
:10C36000D3070000790300003FFC000014F4000034
:10C37000B1ED00001BEC000084F0000028FA000082
:10C38000E1050000C10E0000DB110000030F0000FA
:10C39000E606000048FD00000FF7000016F600005A
:10C3A000B7FA000085020000AB0800006C0A00002C
:10C3B0004C0700009600000000F9000000F30000A8
:10C3C00037F10000ACF400009DFB0000DB02000030
:10C3D0004F070000B2080000A90800002C08000068
:10C3E000CB07000078070000FE05000053020000A4
:10C3F00074FC0000A4F5000058F00000D1EE00002D
:10C40000E0F10000FCF80000540200003B0A0000CC
:10C41000010E00002E0D00005B080000EC02000081
:10C42000CFFF00006BFF00005A0100002103000055
:10C43000430200007DFE00002DF900008AF4000098
:10C44000A5F20000CFF40000B6FA00000C020000D4
:10C45000F20700009E0A0000D0090000CC06000090
:10C460005703000011010000BB000000670100003D
:10C470008D01000030000000FCFC0000DFF800002F
:10C480004EF5000003F4000070F600002EFC0000E2
:10C49000F80200001C080000CD090000FD070000A4
:10C4A000170500009D03000003040000660500005E
:10C4B000E4050000E00300003FFF0000D7F80000A3
:10C4C0008FF200000CEF0000E9EF0000A1F5000082
:10C4D000B2FE0000970700006D0D0000830E000003
:10C4E0001B0B0000A3050000A500000001FE0000DA
:10C4F00050FE00005A000000EB0100001E01000089
:10C50000B9FD000015F90000F0F4000037F3000059
:10C5100070F500007EFB0000210300000009000010
:10C52000B50A0000E20800006D060000E604000005
:10C530003E040000460400001704000057020000FB
:10C5400030FE00002FF800003FF2000009EF00006D
:10C550004EF000001CF60000DCFE00009407000016
:10C56000C70D0000530F00001A0C00001707000051
:10C57000A1020000DEFF000015FF00001AFF00000E
:10C58000DDFE00008CFD00009EFA0000DEF60000DB
:10C5900014F4000020F4000009F800009CFE0000E4
:10C5A00052050000FE090000620B0000F1090000C6
:10C5B0001E0700006F040000DE02000051020000B0
:10C5C000A8010000DDFF00009AFC00006FF80000E9
:10C5D00077F400002DF2000025F30000D3F70000EF
:10C5E000EDFE0000FB050000010B0000A30C0000A5
:10C5F0004D0B0000BD0800001C06000033040000C5
:10C60000DB0200005E0100001DFF000083FB000054
:10C6100023F7000038F300001EF1000093F2000041
:10C62000E6F70000CBFF00009F070000B80C0000F9
:10C63000C50D00007A0B0000F2070000A204000004
:10C6400090020000BC010000FB00000060FF000041
:10C6500059FC000058F8000056F40000C5F1000035
:10C6600047F2000061F6000081FD00007B0500003C
:10C670008C0B0000C40D0000580C00003B090000AA
:10C6800009060000C3030000540200004A01000034
:10C690008AFF000020FC000099F70000FDF2000076
:10C6A00034F00000EFF0000067F50000D2FC00005D
:10C6B00030050000FD0B0000F00E0000A40D00008E
:10C6C000150A0000390600003D0300006701000064
:10C6D00025000000E2FE0000D4FC000081F900000B
:10C6E0006EF50000E8F100003BF1000063F400008B
:10C6F000A0FA00007B0200007E090000760D000019
:10C700005E0D0000A40A00007B0700009F040000EB
:10C710009C02000079010000620000003FFE000062
:10C72000BFFA000085F6000063F200005CF0000034
:10C73000F0F1000030F700001FFF00001B070000B1
:10C74000B90C0000A70E0000240D0000130A000021
:10C75000E3060000630400008E020000D400000025
:10C76000AEFE000049FB00000FF70000E9F20000F8
:10C7700020F00000B6F00000FCF4000032FC0000E5
:10C78000820400003F0B0000A00E0000220E0000FB
:10C79000560B00002108000090050000E303000094
:10C7A000770200009C00000072FD000008F9000004
:10C7B00055F400006CF0000039EF0000B3F1000008
:10C7C00083F7000095FF000095070000310D000081
:10C7D000D70E00003E0D00004A0A0000310700009D
:10C7E000FA0400006B030000DD010000CAFF000036
:10C7F00035FC00006CF70000C5F200009AEF000065
:10C800006FEF0000D3F2000061F900008501000025
:10C81000F6080000A20D00007C0E0000990C00003C
:10C82000AB090000D5060000E90400008A030000FF
:10C830000B020000D8FF000013FC00003BF70000D3
:10C8400063F2000017EF00001FEF00009CF20000F1
:10C8500026F900004D010000C8080000A90D0000E5
:10C86000CE0E00002D0D0000820A0000BE07000061
:10C870009E050000EE030000F401000047FF0000E9
:10C880005FFB0000ADF6000060F2000086EF0000E4
:10C89000A4EF00003CF3000091F900004D010000FE
:10C8A0008C080000320D00003D0E0000BE0C0000A0
:10C8B000490A0000FD0700002F060000B704000031
:10C8C000150300006B0000002CFC0000F5F60000D2
:10C8D00044F2000047EF0000F8EE000012F2000002
:10C8E00046F8000036000000E5070000560D000085
:10C8F000FB0E00005A0D0000B60A000037080000C9
:10C900005A06000023050000B70300007201000072
:10C91000B7FD000090F8000056F300007EEF000025
:10C9200044EE0000B0F0000062F6000042FE00009D
:10C9300065060000510C0000D70E0000C10D00007C
:10C940000C0B000094080000AE06000083050000F8
:10C9500086040000DC020000AAFF0000C7FA000005
:10C9600015F5000050F0000012EE000042EF00004C
:10C97000E5F3000026FB000060030000370A00001A
:10C98000EC0D0000C60D00006C0B0000410900001A
:10C990008D070000A106000034060000FA04000024
:10C9A0003302000056FD00004AF700009FF100002E
:10C9B000F4ED0000AEED0000EBF000001BF700000E
:10C9C0001EFF00009A060000D40B0000090E0000B4
:10C9D0000C0D0000B00A0000DE0800008107000016
:10C9E0004C0600004205000069030000D5FF00006E
:10C9F000D0FA000050F50000AAF0000052EE00004E
:10CA00000CEF0000D3F2000020F9000073000000DA
:10CA100017070000BD0B0000320D0000370C0000AE
:10CA2000A40A0000F8080000940700008B0600002C
:10CA300036050000F1020000E4FE000084F9000069
:10CA400010F40000A3EF0000BDED00001FEF000098
:10CA500075F3000045FA0000A3010000080800007B
:10CA6000300C0000F30C0000C40B00000A0A0000A8
:10CA70006C0800005C07000078060000510500000B
:10CA80001803000015FF0000AFF900001AF40000C1
:10CA9000A1EF00008BED0000F5EE000074F3000044
:10CAA00038FA0000A6010000F8070000240C00007E
:10CAB000E50C0000E20B0000710A0000DA0800003B
:10CAC000FC070000FE060000A80500005C03000053
:10CAD0001BFF0000B5F9000007F4000094EF000010
:10CAE000D6ED000059EF0000C6F300001EFA00006A
:10CAF000160100002D070000410B0000620C000031
:10CB0000570B0000F3090000C708000013080000DD
:10CB1000780700006A0600004B0400005E00000079
:10CB20001BFB000060F5000078F0000007EE00003D
:10CB3000E0EE000066F20000F2F70000ACFE00003C
:10CB400005050000DD090000D50B0000270B0000E3
:10CB5000E7090000D8080000A6070000D80600007A
:10CB60003D060000F90400006A02000023FE0000F8
:10CB7000B7F8000052F300007BEF00004AEE00001F
:10CB80001AF0000060F400005BFA00003D010000B4
:10CB9000F9060000CE0A0000ED0B0000710A00004B
:10CBA0001609000000080000EE060000A8060000BC
:10CBB00033060000B4040000810100007DFC000089
:10CBC000CFF60000A6F10000A8EE0000D6EE0000AF
:10CBD000B9F10000AAF60000FFFC000050030000BD
:10CBE0001B080000EB0A0000B80A0000140900004E
:10CBF00064080000B00700003E0700005B0700006B
:10CC0000B2060000A2040000CB0000007EFB000082
:10CC100000F60000A6F100007DEF0000F6EF000036
:10CC2000C8F200006BF7000004FD0000960200004F
:10CC30007B0700005E0A0000B40A0000E60900005D
:10CC40000909000054080000D70700007907000018
:10CC5000AD060000C20400003701000054FC0000D3
:10CC6000F7F6000064F20000AAEF0000A0EF000059
:10CC700051F2000005F7000024FD00004D03000004
:10CC800076080000420B0000450B0000520A00002D
:10CC9000340900002C08000079070000E0060000BD
:10CCA000E50500008103000077FF000043FA000063
:10CCB000CAF40000B3F0000033EF0000B5F000004C
:10CCC000ACF4000068FA0000AD000000220600008D
:10CCD000D6090000030B0000620A000027090000CB
:10CCE00042080000C40700001D07000029060000DC
:10CCF000FF0300002E00000033FB0000C9F5000018
:10CD000067F1000077EF000071F00000E8F3000029
:10CD100064F90000B9FF00008105000089090000E6
:10CD2000C10A0000330A000065090000560800002F
:10CD300043070000A0060000D20500001F04000009
:10CD4000C6000000CEFB000035F6000050F10000E8
:10CD500097EE0000BBEE0000C6F10000DEF600001A
:10CD600072FD00000C040000F1080000B80B000088
:10CD70006D0B0000B7090000A60800007207000054
:10CD8000B90600008E060000AE0500008203000018
:10CD90006DFF0000F3F9000059F40000F0EF00000F
:10CDA0005AEE0000D9EF0000B9F3000063F900006B
:10CDB000F4FF0000AC050000AD090000360B0000D8
:10CDC000F0090000AD080000220800005F07000025
:10CDD000490700003A070000F80500001E030000A4
:10CDE00076FE0000C5F800008FF300001EF0000082
:10CDF00051EF000042F1000046F50000AEFA0000DD
:10CE00005C0000008805000065090000900A000031
:10CE1000DC090000F808000058080000F2070000D4
:10CE2000BD070000660700002E0600005D0300003D
:10CE3000FDFE0000C6F90000CAF4000049F1000040
:10CE40000DF0000076F10000E2F40000C8F90000E7
:10CE50006FFF0000CE040000F6080000900A0000FA
:10CE60000E0A00003E09000077080000A20700003B
:10CE70004F070000350700005C0600002804000092
:10CE8000650000004EFB0000F8F50000E9F100002D
:10CE90001DF00000DBF00000C2F300006AF80000A3
:10CEA000DFFD00002E0300008E070000BA0900001D
:10CEB000560900003F080000CB0700006A07000089
:10CEC0004C0700008C0700002207000062050000EC
:10CED000F301000032FD0000F3F7000061F30000F1
:10CEE000B3F000009DF00000F5F20000BDF6000078
:10CEF0008CFB00007A000000F904000033080000F9
:10CF0000140900005F0800004B070000F006000055
:10CF100005070000FA060000FC0600005E0600009F
:10CF200054040000D00000004DFC00008AF700000F
:10CF3000C1F30000F3F1000037F2000067F40000D5
:10CF4000FBF7000056FC0000DF0000002005000099
:10CF5000C10700001B080000AF0700000207000027
:10CF6000800600009E060000CE060000D6060000E7
:10CF70003406000032040000E7000000B9FC0000A5
:10CF80005BF80000D6F400000EF300003FF3000051
:10CF900017F5000014F80000F4FB0000E4FF0000A7
:10CFA000890300008E060000A4070000340700007B
:10CFB0007D0600001B0600000C060000270600008E
:10CFC000620600002A060000D90400004C0200009E
:10CFD000BAFE000082FA0000A5F600002DF4000061
:10CFE0006EF3000063F40000B2F600000EFA0000D9
:10CFF000EFFD00009F01000024050000160700005F
:10D0000076060000B305000094050000440500000A
:10D01000A905000064060000990600002F06000024
:10D020006A0400003201000032FD0000F7F8000041
:10D030008CF50000EBF30000EBF3000063F500005B
:10D0400038F80000C4FB000058FF00009002000008
:10D050000E050000C1050000F2040000A30400005A
:10D0600025050000910500005E0600004007000055
:10D070003F0700004B060000EF0300005A000000CD
:10D0800052FC00007EF80000B0F5000088F40000BB
:10D09000F6F4000097F6000033F900005AFC000097
:10D0A0006CFF0000170200002D04000023050000A3
:10D0B000100500001105000081050000FA050000C0
:10D0C00080060000F1060000D5060000DD05000026
:10D0D000D5030000E400000069FD0000FDF9000038
:10D0E0004AF70000C1F5000079F5000070F6000075
:10D0F00068F8000013FB000011FE0000FF000000B4
:10D10000D2030000A7050000A705000014050000D9
:10D1100015050000360500008905000046060000E0
:10D12000CA0600008A06000045050000C60200008D
:10D1300046FF00006DFB0000EFF700009BF50000CC
:10D14000DAF400007BF5000051F70000FEF9000062
:10D1500003FD0000F8FF0000AC0200009E04000088
:10D1600012050000890400009C0400002B0500004B
:10D170009F0500007406000000070000CA060000BA
:10D18000B20500004F030000F0FF000032FC000079
:10D19000BCF8000038F6000032F5000089F5000008
:10D1A00001F700006AF9000051FC000034FF0000A4
:10D1B000C7010000F9030000F8040000E6040000C5
:10D1C000E70400004D050000DC05000058060000E3
:10D1D000C4060000B3060000AD0500009D0300007A
:10D1E000A200000029FD0000D4F900003FF7000074
:10D1F000D7F50000BFF50000E0F60000F3F80000EE
:10D20000B2FB0000A3FE0000830100003404000014
:10D210008D05000042050000E40400000605000042
:10D2200037050000C205000088060000DE06000089
:10D230004B06000093040000B10100000AFE00004C
:10D240004FFA000044F7000094F500005BF5000081
:10D250006FF6000080F800001CFB0000D9FD000004
:10D2600080000000DB02000066040000AC04000047
:10D2700054040000AE04000034050000B9050000AD
:10D2800078060000B50600005D06000021050000DC
:10D29000D1020000B3FF000055FC000044F900007B
:10D2A000F7F60000F3F5000007F600002CF7000089
:10D2B0002AF90000AEFB00004CFE0000DF00000079
:10D2C00079030000B0040000930400005304000040
:10D2D000BC0400005E050000AA0500005F06000017
:10D2E000B70600001F0600009A04000004020000B8
:10D2F000DDFE00009BFB0000B7F80000F1F6000027
:10D300005EF60000B4F60000E6F70000C6F9000083
:10D3100008FC000057FE0000D3000000440300009A
:10D32000C5040000EB0400008E040000CD040000E2
:10D330003C0500009C050000110600003A060000B4
:10D34000C30500004C040000F001000004FF0000D1
:10D35000E4FB000028F900006CF70000C0F60000B4
:10D36000FCF6000019F80000DAF90000F4FB0000F8
:10D3700049FE0000A300000027030000A3040000F2
:10D380009E0400005C04000049040000BD0400008D
:10D39000400500009C050000F5050000AE050000FA
:10D3A0007A0400005402000082FF000084FC0000A8
:10D3B000DCF9000015F8000062F7000081F70000BA
:10D3C00045F80000AAF9000099FB000096FD000056
:10D3D000A1FF0000C8010000B503000075040000B3
:10D3E000ED030000F30300002B0400007B040000A9
:10D3F00042050000A5050000B80500003A05000040
:10D40000BB03000062010000A6FE0000E3FB000079
:10D41000A6F900005BF80000F0F7000030F800000B
:10D4200014F9000085FA000052FC000021FE000003
:10D430001D0000006E020000D9030000E703000099
:10D440008D030000B003000065040000E304000049
:10D45000830500002C0600001006000050050000A7
:10D46000900300000B01000058FE0000C2FB00000A
:10D47000D8F90000C8F8000072F80000B4F8000005
:10D480006FF900009DFA000015FC0000BEFD0000D1
:10D49000BEFF0000C701000048030000BA030000FF
:10D4A00098030000CE03000048040000D5040000EB
:10D4B0009C0500004B06000071060000BE05000040
:10D4C00025040000DA01000027FF000082FC0000B4
:10D4D0004BFA0000D0F800002DF8000036F80000EC
:10D4E000D4F80000F8F900007DFB00004CFD0000BE
:10D4F00061FF0000A5010000830300001B04000081
:10D50000C9030000B8030000F9030000650400002F
:10D510000B050000CC05000043060000F2050000EA
:10D52000D3040000D60200004A000000ADFD000058
:10D5300053FB000098F900009FF8000088F80000F5
:10D5400019F9000005FA000038FB0000B0FC0000EB
:10D5500060FE00004C00000039020000660300007D
:10D56000850300001D0300000A03000057030000AC
:10D57000C40300009F04000080050000D9050000DE
:10D58000A10500009A040000AE0200004400000063
:10D59000BAFD000070FB0000C5F90000E1F80000D2
:10D5A000D2F8000046F9000027FA00005EFB0000F8
:10D5B000B8FC000057FE0000330000000D02000020
:10D5C0000E030000EA0200008B020000A50200002A
:10D5D000FF020000A3030000A1040000A205000058
:10D5E00051060000340600002E0500004B03000029
:10D5F000E30000005AFE0000F9FB000027FA0000DB
:10D600000EF90000C2F8000029F90000EDF9000051
:10D61000EDFA00003AFC0000B5FD000074FF0000C8
:10D6200066010000CE0200003F030000D9020000A6
:10D6300099020000AA020000DC020000B40300000E
:10D64000BE0400008C050000DA050000550500004E
:10D65000FA030000E001000063FF0000F3FC00009B
:10D66000EEFA00009CF9000010F9000034F9000007
:10D67000D0F90000C0FA0000E3FB00003CFD000010
:10D68000D7FE0000B00000004D020000E7020000DD
:10D690009B02000052020000640200009902000098
:10D6A000570300007504000078050000060600001E
:10D6B000BD05000089040000840200001D00000078
:10D6C000A7FD00007BFB0000F4F900002BF900002F
:10D6D0002AF90000AFF900007BFA000093FB00007C
:10D6E000EDFC000072FE0000540000000302000088
:10D6F000F0020000D90200006A020000650200008A
:10D7000056020000EA0200000904000003050000C0
:10D71000C7050000BE050000E10400003E03000054
:10D72000F400000081FE00003EFC000093FA0000BF
:10D7300097F900004EF90000ABF9000053FA000021
:10D7400029FB000039FC000072FD0000FBFE000018
:10D75000CE0000004A020000B30200002C020000CC
:10D76000BD010000530100003A0100002202000048
:10D77000530300009304000095050000E405000039
:10D7800039050000A00300008C01000038FF0000F4
:10D790000BFD00004AFB000038FA0000C2F900004F
:10D7A000D3F900005DFA000017FB0000FAFB00004F
:10D7B00008FD000062FE000015000000C501000029
:10D7C0005202000008020000CA0100006D010000C2
:10D7D000300100005F0100005F020000AE030000A6
:10D7E000B7040000840500007C0500009B040000D5
:10D7F000210300004E0100004CFF00005BFD000013
:10D80000C3FB00009FFA000018FA000000FA0000B5
:10D8100068FA00002AFB000029FC000065FD0000FA
:10D82000D7FE0000B3000000FE0100002A02000045
:10D83000DD0100003F010000A80000006B000000B7
:10D840009B0000005C010000A9020000050400002C
:10D850000705000064050000F7040000F203000063
:10D8600060020000880000009DFE0000DEFC000059
:10D870008FFB0000B3FA00005FFA00007BFA0000A3
:10D8800009FB0000D7FB0000DEFC00000DFE0000DD
:10D890007FFF0000D9000000760100006101000058
:10D8A00013010000B60000003F000000240000004B
:10D8B000720000002E010000580200007A030000F0
:10D8C0004C040000D3040000D90400002904000027
:10D8D0000303000087010000CCFF000016FE0000DB
:10D8E00092FC000054FB000093FA000066FA00006E
:10D8F000AAFA00006AFB00006DFC000086FD000033
:10D90000E0FE00003E000000320100006A0100005D
:10D910002B010000CB000000680000001D0000008B
:10D92000FFFF0000490000001F010000200200006E
:10D930003203000041040000F40400002B05000045
:10D94000C1040000D30300005E020000A700000035
:10D95000F6FE000061FD00001DFC000037FB00002A
:10D96000DDFA0000F3FA00005FFB000039FC000064
:10D970004DFD000081FE0000ECFF0000E50000000E
:10D980002B01000021010000EA00000097000000C8
:10D990003E00000020000000260000004B000000B8
:10D9A000E7000000A10100004C0200000703000096
:10D9B0008F030000E2030000D40300003D030000D9
:10D9C000480200000A010000A2FF000038FE00002B
:10D9D000F3FC0000F9FB000063FB00003DFB0000CE
:10D9E00072FB0000EDFB0000C3FC0000D1FD000055
:10D9F00005FF00002D000000BE000000DB0000005D
:10DA0000D200000091000000470000000600000066
:10DA1000DAFF00001D0000004D0000006D00000056
:10DA2000F00000007D010000DF0100006E02000038
:10DA3000F10200002C0300004E030000F802000079
:10DA4000520200005A01000017000000DDFE000035
:10DA5000B3FD0000BDFC00001DFC0000DAFB00006F
:10DA6000F3FB000071FC000034FD000043FE0000E9
:10DA700083FF00007B000000F4000000FF000000B6
:10DA8000F3000000B000000041000000250000008D
:10DA90001A000000100000003B00000061000000C0
:10DAA0007F000000B5000000EE0000004C01000007
:10DAB000B40100001202000085020000DA0200003A
:10DAC000CA02000075020000E8010000FF0000002B
:10DAD000F7FF0000EBFE0000F7FD000030FD000046
:10DAE000B0FC000083FC0000A0FC000017FD00005B
:10DAF000D5FD0000CDFE0000C1FF00005D0000006C
:10DB0000AA000000A90000007700000051000000FA
:10DB10001B000000070000001F0000003B00000089
:10DB2000600000007A00000083000000A0000000F8
:10DB3000BE000000ED0000003C0100009501000067
:10DB40000A0200006F02000086020000720200005C
:10DB50002802000076010000A4000000B6FF0000CB
:10DB6000CBFE0000FFFD000069FD000016FD000077
:10DB70000DFD000053FD0000DEFD0000A9FE0000C9
:10DB80007AFF000007000000520000006200000061
:10DB9000390000001900000001000000F7FF00003C
:10DBA0001A0000004E0000007B0000009000000002
:10DBB0009200000099000000A2000000A7000000F1
:10DBC000CE0000001901000082010000ED010000FC
:10DBD00028020000610200006C0200000E0200003A
:10DBE0007F010000C5000000E9FF000019FF0000F0
:10DBF00062FE0000D4FD000085FD00007AFD0000FB
:10DC0000A6FD00000BFE0000A5FE000046FF000080
:10DC1000BFFF0000F8FF0000150000000D0000002D
:10DC2000F0FF0000F7FF0000140000003C000000BF
:10DC30007A000000AA000000B5000000BD0000004E
:10DC4000BD000000A8000000A30000009C00000030
:10DC500091000000A2000000CA000000F0000000D7
:10DC60002F0100005A0100004D0100003C0100009E
:10DC7000EF000000820000000A00000072FF0000B8
:10DC8000F6FE00008BFE000033FE0000FDFD0000EC
:10DC9000FEFD000037FE00008DFE0000E7FE0000E4
:10DCA00054FF0000A7FF0000CCFF0000E2FF0000CF
:10DCB000E1FF0000E2FF0000D7FF0000D6FF0000F8
:10DCC000E0FF0000F2FF0000180000002B00000041
:10DCD00028000000270000003A0000004900000072
:10DCE00049000000480000005100000054000000FE
:10DCF0004C000000500000005900000069000000C6
:10DD0000800000009A000000D1000000ED0000003B
:10DD1000ED000000CC0000009D0000007500000038
:10DD200018000000D4FF0000A7FF00005FFF000004
:10DD300046FF000042FF000045FF00005EFF0000BC
:10DD40007FFF000096FF0000ACFF0000CDFF000049
:10DD5000D6FF0000D2FF0000EBFF00000B00000028
:10DD60000D000000300000004C00000043000000E7
:10DD700060000000660000005F000000440000003A
:10DD800036000000410000001C00000018000000E8
:10DD90001A0000001600000027000000220000000A
:10DDA0001500000013000000210000002500000005
:10DDB0001E0000002A00000012000000E9FF000021
:10DDC000D9FF0000C9FF0000C4FF0000C1FF000030
:10DDD000B9FF0000BDFF0000BFFF0000BCFF000056
:10DDE000C3FF0000C4FF0000C6FF0000C8FF000022
:10DDF000C6FF0000C5FF0000C3FF0000BAFF00001F
:10DE0000C8FF0000E1FF0000E6FF0000EDFF00009A
:10DE1000FCFF0000F8FF0000ECFF0000E3FF000043
:10DE2000F4FF0000F0FF0000EDFF00000200000022
:10DE300003000000FCFF0000F4FF0000F6FF0000FC
:10DE4000F4FF0000FEFF00001000000014000000BE
:10DE5000260000003100000028000000260000001D
:10DE600026000000220000001B000000120000003D
:10DE700023000000410000004F0000005A00000095
:10DE80005E0000004F0000003B0000003300000077
:10DE90003A0000004800000041000000430000007C
:10DEA0005D000000660000007300000065000000D7
:10DEB00070000000870000005500000073000000A3
:10DEC00048000000200000005D0000001F0000006E
:10DED0004600000061000000300000005E0000000D
:10DEE0004400000033000000300000000D0000007E
:10DEF0003000000026000000260000003000000076
:10DF00000C0000001C00000002000000F6FF0000F2
:10DF1000150000000F0000002A0000001B00000098
:10DF20000D0000000C000000E0FF0000DAFF000020
:10DF3000CFFF0000D6FF0000F4FF0000EFFF00005D
:10DF4000F7FF0000F7FF0000D8FF0000E0FF00002F
:10DF5000DAFF0000DAFF0000E7FF0000E9FF000041
:10DF6000F4FF0000F6FF0000F5FF0000F8FF0000DE
:10DF7000010000000A0000000A0000000E0000007E
:10DF8000080000000A00000013000000100000005C
:10DF900012000000140000001D0000001A00000024
:10DFA00017000000120000001C0000002700000005
:10DFB0002400000034000000400000004200000087
:10DFC00050000000480000004A0000005D00000012
:10DFD000550000005C000000550000005B000000E0
:10DFE000550000004F000000570000003C000000FA
:10DFF00031000000360000003F0000002600000055
:10E00000520000005400000050000000E8FF000033
:10E010001400000086000000F9FF0000240000004A
:10E020001B00000028000000FAFF0000D6FF0000DF
:10E03000200000009DFF0000A3FF0000B2FF0000D1
:10E0400085FF000066FF000063FF00005FFF000027
:10E0500051FF000063FF00005CFF0000CDFF0000E7
:10E060001700000052000000FD000000C00000008A
:10E070001B000000490000005800000014000000D0
:10E08000B9FF0000A8FF00006FFF000081FF000043
:10E0900065FF00002CFF00005FFF000030FF000064
:10E0A00033FF000040FF000057FF00002EFF00007C
:10E0B00048FF000037FF000042FF0000B9FF0000EA
:10E0C0001B00000087000000D70000005E01000078
:10E0D0001E010000510000006D000000AD000000B6
:10E0E0003E000000DAFF0000C7FF0000B2FF0000A2
:10E0F0009BFF000075FF000064FF00005FFF000051
:10E1000047FF00004BFF00003DFF00002CFF000018
:10E110002CFF000024FF000035FF000095FF0000E9
:10E120000400000079000000E10000006C01000024
:10E1300094010000E0000000A4000000BB0000000B
:10E140008100000020000000F7FF0000D3FF000066
:10E15000C3FF0000A4FF00009DFF0000A2FF00001D
:10E160007EFF00008BFF00006CFF00005EFF0000E0
:10E1700067FF00006FFF000078FF0000D6FF00007F
:10E180008B0000001E010000B40100002702000007
:10E190005902000097010000E10000003701000073
:10E1A000F6000000580000001B0000000A000000FC
:10E1B000F3FF0000F4FF0000FAFF0000EEFF000094
:10E1C000F6FF0000CFFF000099FF000088FF00006D
:10E1D00074FF000079FF000082FF0000EEFF0000E6
:10E1E000930000001B010000F60100005202000035
:10E1F000D401000092010000A50100004B010000C5
:10E200009B0000003900000001000000C7FF000073
:10E21000ADFF000093FF00008FFF000090FF0000A3
:10E220007EFF00007EFF000037FF000023FF00009C
:10E230002FFF00002AFF00007DFF0000ADFF00005F
:10E2400025000000B90000004D010000110200008F
:10E25000190200009C0100009A010000A8010000C2
:10E2600027010000830000002C000000E6FF0000F2
:10E27000B2FF000088FF00006FFF000093FF000066
:10E2800030FF000030FF0000FEFE0000B5FE000081
:10E2900009FF0000ECFE000010FF000082FF0000FC
:10E2A000F7FF00005C000000E1000000A00100009A
:10E2B00009020000D0010000CD010000880100002B
:10E2C000C90000001B00000082FF00006DFF00007D
:10E2D00012FF00009AFE0000D4FE0000AFFE000016
:10E2E00045FE000092FE0000DFFE00005BFE000025
:10E2F0009EFE000069FF00003DFF000063FF00007C
:10E300009DFF000002000000440000006E000000BD
:10E31000940000007100000052000000FEFE0000AA
:10E3200067FE000050FE0000F2FD0000FAFE000053
:10E3300068FF0000B8FF00009C0000001C00000007
:10E3400084000000DB00000095FF0000A7FF000034
:10E3500024FF000001FF0000D2FE0000C4FE000008
:10E3600040FF000010FE000078FE000000FE0000EC
:10E37000E0FD000086FE000066FE00004AFF00008F
:10E3800084FF0000B400000051010000A60100005D
:10E39000120200009D010000250100008300000022
:10E3A000C5FF0000F9FE0000B9FD000089FD000076
:10E3B000D9FC0000E0FC00004CFD0000F4FD000072
:10E3C0004DFE000010FF0000E6FF00006C000000A2
:10E3D00069010000D1000000C60000004F000000ED
:10E3E000C8FF00006AFF0000D2FE0000D4FD00005C
:10E3F00057FD00004AFD000008FD000079FD000007
:10E400006BFE000075FF000036000000AA0200004D
:10E410005B030000E40200003E0300008D010000E9
:10E4200096000000C8FE000075FD0000F6FB00002D
:10E43000D7FA00005CFB000085FB0000AFFD000088
:10E4400080FF00002001000062030000A302000022
:10E4500050050000DB02000017020000D50000009C
:10E4600082FE00007FFD000016FC000077FB00002C
:10E4700081FA000040FC000078FC00005000000021
:10E48000C8020000800500002D070000F40700000E
:10E49000130600007D0400005301000013FD00007E
:10E4A000F0FB00002CF900006FF9000090F900006B
:10E4B0000AFB000012FD0000AFFF00006203000035
:10E4C000C0040000C209000003090000C60A0000E1
:10E4D000180800002404000076000000B4FA0000D0
:10E4E0008EF8000084F40000AEF6000001F7000092
:10E4F00048FD0000B7020000DD080000260E000005
:10E50000C40D0000E80D00006D040000EE010000E5
:10E51000F1F90000CCF2000042F8000078F10000B0
:10E5200019FF00009DFD0000C00500008D060000E1
:10E530008F0700002B080000D4030000A406000091
:10E54000A9FF00009DFF000071060000E2FA000034
:10E550006C040000FAFD000016FD000077FF0000CB
:10E56000AEFA0000B000000001F900004602000011
:10E570002EFD0000110300004B0400004C0B0000B6
:10E58000C8070000590A0000EB050000AFF90000C1
:10E590009D0500009CF20000D9FB000045FE000034
:10E5A00055F700003808000092F700002D06000023
:10E5B00058FF00001C05000036090000600500003F
:10E5C0001D090000D90000002FFF00005F040000BB
:10E5D00060F2000036FF000070FA0000CFF8000083
:10E5E0009308000087FD0000D107000031FC000007
:10E5F000D0FF0000BCF900006AF90000D506000059
:10E60000CE0D0000C90C0000731500007901000058
:10E61000E1F7000006020000B8E000001F02000061
:10E620001FF80000F0FE00003512000072F6000036
:10E63000A510000060F80000CF030000FB030000FD
:10E640004EFA0000A909000095F8000053080000E8
:10E650003D08000012F20000880800001FF10000D1
:10E66000AEF500000F080000BEF40000280900000D
:10E670000EFD000008FF000087FC000092FA000079
:10E68000D012000073050000920F0000FD0700008B
:10E690006CE90000A2FA00003BFA00000EEE000058
:10E6A0001414000059FD000037FC00002A06000089
:10E6B00013E60000730A00002500000010070000A8
:10E6C000A20C000026F4000091000000B4EB000052
:10E6D000E40B000089020000B4F40000F41700000D
:10E6E0008BDD0000470500002000000051EB00001A
:10E6F00015150000D3F400003CFC000013020000DC
:10E70000D40C00002E1400006E060000EDFE000088
:10E7100090E1000018F00000B0130000C2F6000005
:10E720004F1900005200000007D90000210400002A
:10E7300083F20000F4120000381C00004A020000BE
:10E7400082F300002EE300009DF30000AD080000FE
:10E75000901B0000C30F00002BF4000058E70000DE
:10E76000FDEB000049020000671B0000900A00005A
:10E7700034F000001EF1000043E90000C80300006F
:10E7800029230000BF180000DE080000B2EF0000DF
:10E79000AADF000046FA00005E180000270900000A
:10E7A000630200005CF2000032E10000F4FD0000B2
:10E7B000210C00000B1B0000F20F000034F10000E0
:10E7C00097F3000002F40000CFFF00005310000098
:10E7D0009B02000010FC0000A9FC0000CEEE00002F
:10E7E000BB090000870E0000B0F700003E040000E7
:10E7F00074EE000094EE0000B30F0000F409000076
:10E8000018030000EA050000ABF60000E5FB00007D
:10E81000FF25000002080000C4E100001AFB000010
:10E82000F8EE0000DB0200009213000020F500006B
:10E8300047F90000100100005D0700008B04000094
:10E8400040030000920100005E0B00006112000016
:10E850007AF50000B4F20000E2FB0000B0FF000017
:10E86000CD0B0000160300000FF000003CFA000082
:10E870006809000091000000E4050000FAF80000BB
:10E88000D4FE0000DB0D00006BF000000C02000065
:10E89000B10800001FF80000960700003F030000C9
:10E8A00063EC0000DFF900007D150000940B000010
:10E8B00016FC0000B6FE0000E0F10000B901000007
:10E8C000A20C000044FB00004B1A00006FE50000A2
:10E8D0000EE400000E25000011FF00004EF10000C4
:10E8E0002D0D0000D50D0000A0E4000072FD000019
:10E8F000B4160000B5ED0000B8FD00007A1200006B
:10E900002DF800009BF600007806000088FF00004C
:10E9100078F90000880200001204000044FA0000A8
:10E920005BFF0000D0030000C2FA000064FF00009B
:10E930006EFA0000D3020000DB0000007712000036
:10E94000780B000045CB0000420300003A1F000096
:10E9500030F800008EF6000065FE00001202000094
:10E9600068F400001D0E0000E310000022E8000023
:10E9700040FF00008A15000066FE00001101000043
:10E980005DF200008DF10000E5080000E9090000DB
:10E9900021FE00006EF0000001050000D209000019
:10E9A000AAF80000D6FA0000F4FA0000D500000032
:10E9B00085040000F0110000B0F600006ADD0000E0
:10E9C000880E000007110000BDF90000FEF50000F0
:10E9D000AFF90000F80000006F000000830D000098
:10E9E0007B05000009EB00005705000056100000F1
:10E9F0001D0600004602000066DE000015F700005C
:10EA0000D61600007709000038F20000D6ED0000AD
:10EA1000560F0000D60A00009BF5000040F90000E8
:10EA200060FA000059010000E3090000CD02000077
:10EA30004CF60000FFF300005E060000340B0000FF
:10EA400003FB000090F6000050FA0000970400005D
:10EA5000D503000065FC000059FF000098FC000091
:10EA600083FF0000FC03000020110000E0FC000018
:10EA7000F4DC00006E060000EF1B00004201000005
:10EA800051E8000074F20000F60C000024050000BC
:10EA90009F050000050100007BFB00004F03000004
:10EAA000C3130000DE0B0000E7DC000084E9000077
:10EAB000231400003614000084F700004AF100001F
:10EAC000F10100002C02000047060000A50700002D
:10EAD0009DF70000ADF000002E000000FA0E0000CF
:10EAE000E70400001CF40000E2F7000099070000B2
:10EAF000F50700001DFD0000C1F90000C3FC000087
:10EB0000E4FF0000F30100003C0300005AFF000096
:10EB1000F2FB000070FF0000F90A0000440400004E
:10EB200035F00000A0FA00009A0D0000B00A0000C5
:10EB3000B1F800002DED0000C0FE0000BF0A00008B
:10EB40006D020000AE01000066FE0000A41300008C
:10EB500024110000E0EE0000A5EC0000D4F9000054
:10EB6000B8100000B00700003CED0000CCF200003F
:10EB7000FE0A0000A9190000130700004BF2000074
:10EB800041F800001001000072070000730400004B
:10EB900095F80000C5FA000013FF000049040000CA
:10EBA000490700009FFD000031F90000C9FD000089
:10EBB0007A0500004C05000042FB000032FD000019
:10EBC000A902000067FD000063FD0000470200008D
:10EBD000BF05000061010000E8F80000C6FB00006E
:10EBE000D0020000BA020000C4FE00004DFC00008C
:10EBF000D201000030010000D8020000580C0000D3
:10EC000076FA000088EF0000E4FB0000F50C00003D
:10EC1000FC0F0000EAF6000081EB000033FB00006F
:10EC2000D90F00009E1000001EFD0000E0F700005C
:10EC3000F0080000BF0A000065F70000DDEC0000EE
:10EC4000A1FB0000FC1000002A0800001AF30000DD
:10EC500033F80000930D000022140000CFF70000ED
:10EC60007EE400000AFE000076160000990F000006
:10EC700030F200007FEB00008E040000361400002C
:10EC80000909000064EF000007ED0000AD0400007A
:10EC9000301300006B0800003EF6000097F70000FC
:10ECA000540400000405000064FC0000F0F90000BA
:10ECB0004B0100003A080000470300002AFA000058
:10ECC00001F8000061FF0000780600009E020000CD
:10ECD00000FE0000A2FB0000C5080000300D00008F
:10ECE0001CFA0000F3EF000043F600009909000051
:10ECF0006E0F00009E01000064F300003DF500006F
:10ED0000AD0600005C0E00004A070000B1FA0000EA
:10ED100071F600008C020000CA070000ACFE000083
:10ED2000EFF6000021FA000071060000280700003D
:10ED30005AFB000060F6000078FE00002F0B000078
:10ED40007C0A000042030000C6FD00004CFA0000EF
:10ED500022FD00004EFD000069FD0000460200009B
:10ED600072060000440600009DFE000023F700002C
:10ED70002DF9000045000000A8040000AE040000CA
:10ED80000102000008FE000023FB0000CCFC000094
:10ED9000F0020000210600009802000053FC000071
:10EDA000DCFB0000550000008E020000F6010000B0
:10EDB00055FE0000D4000000B10500000C02000068
:10EDC0005BFB0000B8F70000BBFE0000DD070000A1
:10EDD0006E060000B1FD00005FF700008DFC000032
:10EDE000CE050000130A0000C6050000FAFC000072
:10EDF00075FB0000A9FF0000C60200001CFF000018
:10EE00003FFA000013FC0000BB0200000C060000EB
:10EE10006902000075FE0000ECFD00002902000000
:10EE2000D80400002C0300007A0200001E0100003C
:10EE300008FE00006AF80000CCF900002C05000074
:10EE4000D80A0000AB03000041F6000055F50000B1
:10EE5000670100000E0B0000C5070000CCFA00009F
:10EE600059F6000044FE00008F060000B0050000C7
:10EE700046FF00007FFD0000C4FF0000DBFF000034
:10EE80000BFF00002501000075040000980300003E
:10EE9000BDFC0000A4F80000A6FB0000B8030000C1
:10EEA0002D0700005601000029FC00005EFA00005A
:10EEB000CB040000F6080000F2FD000039F7000066
:10EEC00017FA000066060000EA0900000E010000C3
:10EED000E6F70000C1F9000080050000ED08000021
:10EEE000ED0200008DFA0000C1F900005D04000091
:10EEF0005C060000FEFC0000CBF600006FFB00008B
:10EF000026070000A406000065FB000024F70000AF
:10EF100079FF00003B0B0000AD090000D6020000A5
:10EF200049FD00005EFA000065FD00002FFD0000B5
:10EF3000B3FD0000B8020000A3060000E4050000D5
:10EF4000C5FD0000E9F60000B5F90000D40000009E
:10EF5000D204000087040000AC010000B5FD0000F1
:10EF600011FB000038FD00007103000012060000D4
:10EF70000C020000F2FB00002FFC0000A5000000C6
:10EF8000A2020000B601000029FE00006601000098
:10EF9000B80500007D010000D0FA0000DBF700009A
:10EFA000B4FF000035080000DC050000DDFC0000B7
:10EFB00057F7000060FD00006F0600000E0A000019
:10EFC000E1040000BFFC00005DFC00001D0000002B
:10EFD000A90100003DFD000019FA0000D5FC000069
:10EFE0003B0200009D050000430400004F010000AB
:10EFF000BDFD000037FF0000F90400007E0700009F
:10F000005204000044FC00003CF7000037FA000006
:10F01000EA010000FF06000069050000B5FE0000DF
:10F02000E7F80000BAF9000047FF00007A06000088
:10F030000208000007020000E3FA0000B1F8000037
:10F0400035FE00006E050000DA060000DC0000005E
:10F05000E5FA000011FC0000D60200005A0800008A
:10F060007B06000062FD0000C3F50000E6F700002B
:10F07000F3000000D0080000A707000063FF0000B5
:10F0800070F90000A0F70000B7FB0000DA030000F1
:10F09000C10800005F060000F9FE000059FB0000F7
:10F0A0001DFE0000DC030000CB0600007103000021
:10F0B0009FFC000003F6000095F60000B7FE00007C
:10F0C00072060000840700003300000018F80000FA
:10F0D000CDF700002EFF0000BD0600005209000021
:10F0E000CF0400001BFE000036FC00000100000001
:10F0F00028050000F7040000D6FE000007F7000016
:10F10000C0F400001CFB000082040000880800001E
:10F110004304000036FC0000D7F9000084FD000025
:10F1200087020000C6040000DBFF0000B7FA000001
:10F13000E7F90000D2FD0000AD0300001905000052
:10F140000D03000007FF000009FC000053FD000054
:10F1500035010000AA050000C6050000B800000047
:10F16000E5F9000062F60000DDF80000D2FE0000C4
:10F170001805000017050000430000008BFC00008C
:10F180004EFA000047FC00006C0100004A06000037
:10F190003209000031070000EC020000B2FE00005E
:10F1A0008CFA00004BF80000A4F8000023FB0000DC
:10F1B000D7FE0000730300003C060000420400007C
:10F1C00046FF00007DF90000ABF9000087FF00005A
:10F1D0006B0400003D0600004103000008FD000034
:10F1E00054F7000071F600002FFC00004C040000F2
:10F1F0009A090000AF0900000104000037FD00007B
:10F20000EDF8000091F900004AFF00003204000010
:10F210007F060000F50300006FFC00005BF60000B5
:10F220003FF50000F1F90000C9000000EC06000005
:10F2300032080000A803000001000000B7FD000034
:10F2400059FF00006F04000034070000570500005C
:10F2500064FE00000EF70000F4F2000080F40000ED
:10F260001EFC00003E050000A70B00001A0C000069
:10F27000060600004DFC000053F500001EF60000DD
:10F2800087FC0000F8030000D40700008F05000091
:10F2900058FF000034F9000062F6000037F8000063
:10F2A00012FE0000DF060000840C0000DE0B0000F0
:10F2B0006106000095FE0000E6F9000025F9000057
:10F2C00017FB00008DFD000029FF000022FF000059
:10F2D0000BFE00005AFE00001FFF0000A20000000D
:10F2E000D90100009F0200007E0200005A010000C8
:10F2F00052010000CC0000009EFF0000EDFD000068
:10F3000000FC000043FB0000A0FC00007CFE0000AD
:10F31000610000000A030000B1040000A70400001F
:10F3200048030000F7010000AC0000002AFF0000C5
:10F330002EFE000099FD0000EDFD00008CFE000097
:10F34000EFFE0000CAFF00001A000000C5FF000029
:10F35000FAFE000088FE000054FF00004201000099
:10F36000FE0300007B050000BC040000B3010000A8
:10F370007DFD000026FA000090F80000FAF9000078
:10F3800031FE0000BF0200009E050000CE05000017
:10F390008F030000F6FF00000CFD00008BFB000057
:10F3A00049FC0000F6FE0000740200006A0600003E
:10F3B0001A0900006109000081060000E400000055
:10F3C0000AFA000049F40000FAF10000E1F300003D
:10F3D00019FA000041030000760C0000D81100006B
:10F3E000A910000076090000F5FE000078F5000085
:10F3F00005F000004BF1000051F800004A01000048
:10F4000010080000A90A00006E080000E2010000D8
:10F410006DFC00003BF8000032F70000E0FB00004C
:10F42000A6030000810C000049120000F411000046
:10F43000B30A000039FE00006FF100009CE80000F4
:10F4400018E700008DED000083F900006707000059
:10F45000D81200001A180000C1140000A80A000009
:10F46000CCFD0000C5F200004FED00008FEE000063
:10F47000A0F5000066FE00006E05000070080000A8
:10F480002F0700003203000045FF00002FFD0000A1
:10F4900035FC000020FE0000100200009306000072
:10F4A000F5090000930900005F06000097000000C6
:10F4B0005AF90000B6F2000091EE000087EF00005C
:10F4C0006CF500006EFE0000EC070000860E0000E8
:10F4D000D6100000570E000059070000DAFD0000AA
:10F4E000B9F50000ADF20000B5F4000061F90000CC
:10F4F0007AFE0000AB010000330200000F010000A3
:10F50000FCFF0000FBFF000046000000610200005D
:10F51000460600007B090000F60A000021090000F1
:10F52000900400001BFE0000C7F60000C8F00000B9
:10F53000E7ED00004DF00000E2F60000D3FF000010
:10F5400047090000F60F000086120000CF0F0000F0
:10F550006C080000F0FE0000D0F60000EEF20000A3
:10F560008DF30000A1F700003EFD0000DF01000068
:10F57000FC0300006903000079010000570000004F
:10F58000D9FF0000E5000000010400006E07000044
:10F59000560A00009D0A00004607000030010000E6
:10F5A0001AFA0000F8F30000EBEF000074EF00001F
:10F5B000F5F200002CFA000077030000610B000058
:10F5C0000D100000871000000D0D00006406000003
:10F5D000BDFD0000D7F60000D5F30000A5F4000043
:10F5E00005F8000028FC0000A0FF00001501000045
:10F5F000680100007C010000A90100003202000047
:10F60000BF030000A30600005A0900006B0A0000B7
:10F610008F080000EA03000058FD00006AF60000B1
:10F6200034F10000FBEE000071F0000090F50000E6
:10F63000C7FD0000960600008A0D0000681100005A
:10F64000F8100000520C000087040000EFFB0000DF
:10F65000B6F500004DF3000096F400004BF80000F2
:10F66000CEFC00007B0000001E02000037020000FC
:10F670002A0200007C020000CD0200001C040000F1
:10F680009A060000C50800007E090000E707000098
:10F69000F5030000D9FD00003CF7000043F2000034
:10F6A00001F000001BF100007AF50000CFFC000023
:10F6B000410500009C0C000012110000FB1000002E
:10F6C000E50C0000D7050000B0FD000037F7000092
:10F6D000F6F3000036F400002CF7000080FB000079
:10F6E000BAFE0000230000009B000000870100001C
:10F6F000C20200001303000076040000D0060000E0
:10F700001F090000390A00001F0800008F030000D5
:10F710003AFD000061F600000AF100007CEE0000F6
:10F7200090EF000011F40000CAFB0000B9040000D3
:10F73000E80B00002910000071100000070D000008
:10F74000820600009CFE000034F80000AAF40000CD
:10F7500040F400001FF6000073F90000B7FC000041
:10F7600097FE000096FF00005F000000E00100002F
:10F770004C03000092040000CF060000B80800000F
:10F780007A090000110800002704000095FE00001F
:10F7900021F80000CEF2000004F0000027F0000085
:10F7A00035F3000018F900001A0100007F0800007E
:10F7B000990D0000860F0000ED0D00008709000084
:10F7C0001703000066FC000070F700005BF5000006
:10F7D000A1F50000A6F7000094FA0000CEFC00009E
:10F7E0006AFE0000BAFF000053010000070300009A
:10F7F00083040000F30600009F0900002F0B0000A7
:10F80000860A00000A0700007E010000A9FA000035
:10F810001CF40000C5EF0000ACEE000024F1000075
:10F82000A0F6000091FE0000D5060000020D0000C9
:10F8300051100000F60F0000450C0000D705000035
:10F8400089FE0000C7F800008EF50000FAF4000001
:10F8500074F6000067F900003DFC000003FE0000A4
:10F860004BFF0000AA0000008F0200002A040000E5
:10F87000E90500004A080000060A00002D0A000001
:10F88000D40700001E030000EBFC00005CF6000043
:10F8900084F100007BEF00007EF0000061F40000C6
:10F8A00009FB000029030000020A0000560E0000B8
:10F8B0005D0F0000170D000035080000A6010000D4
:10F8C00055FB000011F700008CF5000004F6000065
:10F8D0000EF80000A5FA00009DFC00004CFE0000A0
:10F8E000D2FF0000A10100007C03000077050000AA
:10F8F00058080000F30A0000CB0B0000140A0000B7
:10F90000C305000096FF00008BF8000070F20000B5
:10F9100015EF00002DEF0000BDF20000F7F8000029
:10F92000FA00000092080000DE0D000064100000E4
:10F93000770F0000900B000058050000AAFE0000A1
:10F940007BF9000066F6000077F500006DF6000018
:10F95000E9F8000062FB000036FD000013FF000024
:10F960003C0100008D030000BE0500001B080000E4
:10F97000B10A00003E0C00006C0B0000DC07000028
:10F98000E8010000B7FA0000FAF30000A7EF00005A
:10F99000A5EE0000D7F000000FF6000089FD000082
:10F9A000650500007A0B0000F20E0000880F0000D1
:10F9B0003F0D000052080000DA01000013FC0000B7
:10F9C0000FF80000CCF500007AF50000BDF600004D
:10F9D000C2F80000FBFA000077FD000046000000BE
:10F9E000D60200003D050000FA070000D80A00001A
:10F9F000D40C0000650C000062090000190400002E
:10FA000045FD000083F600004BF1000029EF0000E7
:10FA100043F0000031F400008CFA0000C501000042
:10FA2000610800003F0D00008C0F0000070F000070
:10FA30009A0B0000110600003900000040FB000096
:10FA40007CF700006BF500005CF50000D5F60000C7
:10FA5000EFF8000087FB0000AAFE0000B2010000E2
:10FA600098040000960700008A0A0000010D0000BB
:10FA7000820D0000410B000074060000EBFF000047
:10FA800026F9000057F30000C0EF000054EF00001B
:10FA9000D7F10000E3F6000081FD0000250400001E
:10FAA000C30900007D0D0000030F0000E70D0000FA
:10FAB000190A0000EE0400008DFF0000AEFA0000FD
:10FAC000E1F60000ACF4000085F40000F8F5000059
:10FAD00034F8000025FB00008CFE0000F10100005E
:10FAE00065050000F8080000400C0000340E00001E
:10FAF000B30D0000720A0000F404000005FE0000CF
:10FB000020F70000B8F10000E5EE000012EF000061
:10FB10001DF200009DF7000069FE000007050000CF
:10FB20002B0A0000850D0000CD0E0000640D0000C2
:10FB3000910900008E04000066FF0000BDFA00007D
:10FB400018F70000FAF4000081F400003DF5000011
:10FB50000AF70000D5F9000054FD00002B01000059
:10FB600047050000C5090000AB0D00006B0F000049
:10FB7000630E0000710A00006A04000077FD0000B7
:10FB80008DF6000034F1000092EE0000DDEE000082
:10FB9000FCF1000068F7000004FE00007F04000094
:10FBA000D1090000AE0D0000420F0000C20D0000A0
:10FBB000250A000087050000740000009CFB00007F
:10FBC000ACF7000034F5000053F400008CF40000A2
:10FBD000EFF500008AF8000015FC00004B00000063
:10FBE000A6040000BE090000810E00009C10000069
:10FBF0009B0F0000B60B00007C0500001BFE000000
:10FC000015F7000094F10000E5EE000041EF000060
:10FC10001DF200003AF700007BFD0000A803000081
:10FC2000BE080000950C0000930E0000D70D0000E8
:10FC30003B0B0000960700003F030000ADFE0000F4
:10FC400048FA0000FCF600000CF5000038F4000053
:10FC5000D0F40000D8F600000EFA00004DFE0000BF
:10FC60001D030000E6080000710E00002A110000CC
:10FC7000B4100000780D0000F0070000E70000005D
:10FC8000DFF90000F6F3000037F0000060EF00003D
:10FC900008F1000013F50000AAFA0000B20000000D
:10FCA0001B060000910A0000D60D0000590E00004E
:10FCB000650C0000350900002C050000C60000009E
:10FCC0003CFC00005AF80000A6F5000025F40000F6
:10FCD000ECF3000039F50000D0F700008EFB0000C7
:10FCE00025000000780500006A0B00005E0F000090
:10FCF00078100000F70E0000980A00006D04000064
:10FD000062FD0000BFF60000C2F1000075EF0000C8
:10FD1000E0EF0000ABF2000090F7000062FD000091
:10FD20001103000007080000F40B0000F00D0000B4
:10FD30004C0D0000140B0000D8070000B0030000B9
:10FD400039FF0000D7FA000062F7000025F5000037
:10FD500007F4000071F400005BF6000088F9000071
:10FD6000D0FD0000BD020000BE080000600E0000D3
:10FD7000DE100000621000004C0D0000D5070000EE
:10FD8000FD0000000EFA00002BF4000081F00000DE
:10FD9000ADEF000053F1000058F50000DEFA00005E
:10FDA000CC000000170600008C0A0000C20D000005
:10FDB000150E0000140C0000ED080000FB0400000C
:10FDC000AC00000034FC000066F80000B0F5000054
:10FDD0000CF40000BAF300000BF50000AAF70000D5
:10FDE00083FB000044000000160600005F0C0000CA
:10FDF000C70F000056100000800E0000CE09000062
:10FE0000A8030000CAFC000069F60000D8F1000059
:10FE1000E3EF000066F0000025F30000E1F70000CA
:10FE200043FD000072020000490700003F0B000084
:10FE3000310D0000B40C0000040B00004D08000060
:10FE40006E0400002D000000D0FB000017F8000039
:10FE500055F50000A3F300009CF3000031F500000D
:10FE600016F800005CFC00006E010000CE070000E8
:10FE7000C40D0000EE0F0000BA0F0000610D00007D
:10FE8000710800008002000009FC000051F600002B
:10FE900098F20000F1F0000088F1000039F4000051
:10FEA00056F800004EFD000032020000240700005A
:10FEB000670B00002C0D0000D70C0000140B000095
:10FEC0002A08000054040000C1FF00002EFB0000BF
:10FED00049F7000075F40000FBF2000028F3000071
:10FEE000E0F4000021F80000ABFC0000110200006B
:10FEF00096080000820D0000080F0000910E00001F
:10FF0000A50B0000D5060000480100004FFB0000D3
:10FF10004DF600001CF30000B1F100004CF20000AF
:10FF2000BAF4000086F8000018FD0000B3010000DC
:10FF3000BF060000240B0000D40C0000CF0C000012
:10FF4000A60B0000A008000069040000C1FF00002B
:10FF500003FB0000F8F600005CF4000014F300005E
:10FF600076F3000068F5000090F80000E8FC00005F
:10FF7000F901000039080000220D0000B90E000050
:10FF8000810E0000E00B0000700700004902000035
:10FF900088FC0000A9F7000054F40000BBF2000048
:10FFA000FDF20000C9F4000001F800002BFC000085
:10FFB0006B00000071050000770A0000DC0C0000F7
:10FFC000AA0D0000DF0C0000BB090000980500002E
:10FFD000B0000000C9FB0000A6F70000CEF400004E
:10FFE00084F30000C8F30000A3F500007AF80000D5
:10FFF0006BFC0000C50000005A060000E30B000087
:020000040001F9
:10000000F90D0000940E0000DC0C0000B8080000A0
:1000100036040000D9FE0000D0F9000022F60000EE
:10002000D7F3000058F3000078F40000ECF600006D
:1000300068FA000038FE0000C50200004808000011
:10004000930C0000DC0D0000620D0000520B00005C
:100050006B070000BF0200009CFD00000DF90000CE
:10006000B7F50000D5F30000B1F30000DEF40000A6
:100070003CF7000092FA00006FFE0000FD02000055
:10008000C70800009D0C0000B20D0000CD0D00005F
:10009000540B00001D07000025020000B1FC000009
:1000A000F2F70000B3F4000011F300004BF300007E
:1000B0000EF50000DCF700008BFB00006EFF000077
:1000C000C9030000EC080000A40C00009D0D000016
:1000D000200D0000890A00003E0600009301000088
:1000E00061FC0000DAF70000E6F400006CF30000A9
:1000F0009CF3000044F5000014F800005FFB0000D2
:1001000009FF00005C030000500800007E0C0000A6
:10011000FA0D0000B50D00005F0B0000F0060000B6
:10012000EB0100007CFC0000BEF7000073F400004F
:10013000F1F2000064F3000064F5000088F80000AC
:1001400010FC0000B9FF0000CC030000F207000023
:10015000880B00008D0D0000650D0000510B0000A4
:10016000AA070000DC02000099FD0000D2F80000A0
:100170003DF5000063F300007CF3000014F500007F
:10018000B6F7000020FB0000A3FE000059020000AB
:10019000A3060000DC0A00008B0D0000FC0D00002F
:1001A000860C0000180900005C040000DAFE000064
:1001B00076F9000069F50000F5F200008DF200000C
:1001C00028F40000EFF6000093FA00005EFE000045
:1001D00007020000F7050000C5090000940C0000AC
:1001E000770D00005C0C00008E0900005705000030
:1001F0004100000011FB0000C8F60000F1F3000010
:10020000FDF20000F0F300002BF600005FF90000A3
:1002100006FD00008C000000490400007108000089
:10022000190C0000E80D0000830D00001C0B0000FD
:1002300010070000DD01000024FC000035F700007D
:10024000C8F300002BF20000D7F2000032F50000E6
:100250008EF8000092FC00004E000000E903000050
:10026000AD070000030B0000EA0C0000E40C0000E6
:10027000180B0000A707000016030000DEFD0000B9
:10028000F9F8000041F500001FF3000003F300003F
:100290009DF400006BF7000005FB0000B3FE0000BA
:1002A00015020000B1050000BF090000E30C0000CA
:1002B000FA0D0000C70C0000B10900002B0500007A
:1002C00090FF000005FA000075F500008BF20000B9
:1002D000C6F1000024F3000013F60000ECF9000062
:1002E00003FE000099010000F1040000590800001D
:1002F0000F0B0000740C0000320C0000150A000007
:10030000A60600003702000037FD00009DF800003F
:1003100010F5000026F3000011F30000BEF4000009
:10032000B2F700004EFB00000DFF00007B02000052
:1003300004060000EF090000EC0C0000A70D00000F
:10034000620C00006909000002050000ACFF00001B
:100350002AFA0000B7F50000F2F2000032F20000C5
:1003600080F300006CF6000040FA000049FE000037
:10037000C0010000E404000006080000BE0A0000FE
:10038000560C0000F30B0000160A000014070000D2
:100390001603000054FE0000B2F900002AF6000027
:1003A000F5F30000A9F30000EFF4000068F7000087
:1003B000E2FA000073FE0000C90100001E05000003
:1003C000F8080000470C00003F0D0000660C00001C
:1003D000D4090000DF05000039010000FAFB00002D
:1003E00089F70000ADF4000076F30000F8F3000098
:1003F00004F6000017F90000BCFC000040000000FB
:10040000420300006E0600009F090000E60B00009A
:10041000790C00003B0B000085080000C2040000BE
:1004200046000000B0FB0000D2F7000039F50000E4
:100430002DF400009CF4000072F600006BF900003F
:10044000D9FC00000C00000034030000CB060000C3
:10045000540A0000660C0000BE0C0000490B0000AE
:100460001D0800001904000044FF00007DFA000090
:10047000D6F6000086F40000D2F30000D2F40000AB
:1004800023F7000063FA0000CCFD0000F600000036
:100490001204000060070000A60A0000100C000013
:1004A000E40B00006B0A000041070000710300002C
:1004B00000FF000096FA00002EF7000019F500007A
:1004C0004FF4000018F500003FF7000032FA00007A
:1004D00092FD0000CB0000001F040000CE070000CA
:1004E000400B0000A80C0000360C00006E0A000053
:1004F0001C0700003A030000BAFE000074FA000076
:1005000052F7000047F50000B5F40000A6F5000022
:10051000FBF70000EDFA000019FE000034010000B6
:10052000490400001C080000190B0000550C0000D5
:100530001D0C00000C0A0000DA060000EE020000AC
:100540006AFE000043FA00001EF7000025F50000D7
:10055000A6F40000A8F50000F1F70000DEFA0000A4
:10056000F3FD0000000100004E0400002908000017
:10057000EE0A0000FD0B0000650B000046090000BC
:1005800069060000910200003BFE000052FA0000E4
:1005900039F7000035F500009CF4000090F50000EC
:1005A000C1F7000082FA000091FD0000AA000000DF
:1005B000320400002A080000C70A0000F10B000006
:1005C0002B0B0000F108000032060000560200006C
:1005D0002FFE000045FA00001EF700002FF5000076
:1005E0008EF4000074F5000081F7000027FA000087
:1005F0002CFD000046000000F5030000FF0700008E
:10060000980A0000970B0000F20A0000C2080000E0
:10061000E20500002D0200000DFE00003DFA000082
:1006200023F700002CF500008EF400004BF50000CD
:1006300044F70000E4F90000CDFC0000E6FF0000F4
:10064000CF030000D6070000490A0000740B000029
:10065000A00A0000DD08000075060000B0020000DE
:100660009CFE000093FA000044F700001CF5000017
:100670005AF4000019F5000010F70000CEF9000050
:10068000EEFC000014000000C2030000AC070000F4
:100690006C0A0000AB0B00001C0B00007809000086
:1006A000D0060000FD020000CFFE00009EFA000010
:1006B0003FF7000021F500004FF4000019F500009D
:1006C0000FF70000D0F9000006FD00002D0000002B
:1006D000E1030000DD070000E30A00000F0C00004A
:1006E000820B0000B3090000B2060000F202000015
:1006F000A1FE00008BFA000063F700004FF5000038
:10070000A5F4000083F50000B4F700007DFA0000B6
:1007100096FD0000B00000000B040000FE07000082
:10072000BC0A0000FA0B0000D60B0000C60900004E
:10073000B1060000D40200005AFE000045FA000095
:1007400018F700001DF50000A7F40000ABF500004D
:10075000F7F70000E0FA0000F4FD000008010000D7
:10076000790400005D080000030B0000EF0B00009F
:10077000380B0000100900001C06000023020000D6
:10078000CAFD0000F7F90000F9F6000010F50000BE
:10079000A6F40000C0F5000003F80000CFFA000046
:1007A000E5FD0000FE0000009D040000850800003B
:1007B000FD0A0000F90B0000F50A0000B308000074
:1007C000DA050000E2010000BFFD0000E6F90000CC
:1007D000DEF600000DF5000093F40000A2F5000025
:1007E000C0F7000072FA00007DFD00009D000000CF
:1007F0006504000058080000C70A00009F0B0000B5
:10080000C30A00007C0800008C050000BF01000046
:100810009EFD0000DEF90000E1F600000AF5000090
:1008200090F4000076F5000084F700002DFA000037
:100830001DFD00003E000000460400002A080000E4
:10084000760A0000700B0000530A000084080000C4
:10085000060600003002000028FE00003FFA0000FB
:1008600017F7000015F5000072F4000043F50000D2
:100870003EF70000E1F90000F3FC00001700000063
:1008800008040000FE070000710A00008C0B000045
:10089000B10A0000FF0800006F060000930200008C
:1008A00083FE00006EFA000026F7000011F500003C
:1008B0004EF400001EF50000FFF600009DF9000058
:1008C000AEFC0000C8FF0000D9030000EF070000E5
:1008D000820A00007D0B0000C70A00000209000028
:1008E00055060000B7020000B1FE0000C2FA000089
:1008F0008EF7000061F5000078F4000024F5000098
:10090000FAF600006DF9000052FC00006BFF0000D9
:1009100034030000350700009A0900001D0B000099
:100920005E0B0000870900000E0700009C0300001A
:100930004FFF000040FB0000BDF7000066F500001F
:1009400065F40000DCF40000BAF600002AF90000AB
:10095000FEFB00001CFF0000E40200001007000086
:10096000BF090000F60A0000250B0000D9090000AD
:1009700076070000450400003D00000033FC000045
:10098000B9F8000027F60000F9F4000032F5000085
:10099000D3F600003EF90000FDFB0000D8FE000089
:1009A000490200005406000045090000FA0A000050
:1009B0008E0B0000700A000077080000BE050000E2
:1009C000D7010000C9FD00001CFA000029F7000053
:1009D0007BF5000029F500005AF6000072F80000CF
:1009E00008FB0000F4FD0000260100002F050000B8
:1009F00073080000730A00007A0B0000840A0000EC
:100A0000E808000093060000F5020000F8FE000070
:100A10001AFB0000EEF70000E4F5000016F50000F8
:100A2000D1F5000093F70000E6F90000BAFC0000E1
:100A300096FF000044030000E30600001C090000CC
:100A4000C30A0000AE0A0000040900003E070000CF
:100A50005704000080000000C3FC000059F90000AA
:100A6000D4F600006CF5000067F50000AFF600005A
:100A7000CEF800006CFB000026FE00007F010000A5
:100A80002005000032080000EE090000810A000085
:100A9000EF0900004308000027060000D80200000C
:100AA000EFFE00004BFB00002BF800001DF60000DD
:100AB00044F50000F6F50000B9F7000026FA000042
:100AC000C9FC0000BCFF00005503000069060000DF
:100AD00076080000B10900002D0A00004909000055
:100AE000D107000059050000AC01000005FE000020
:100AF0004EFA000073F70000BCF5000053F500004B
:100B000097F60000A1F800002AFB0000E8FD0000B5
:100B1000F400000066040000E50600008208000002
:100B20009E09000091090000CF0800003607000070
:100B3000860400001701000029FD0000BEF9000036
:100B400010F7000091F50000A4F50000D9F60000B0
:100B5000DDF8000076FB000007FE00001901000030
:100B60004604000066060000410800003409000049
:100B700064090000C4080000180700009604000083
:100B8000FC0000003AFD0000D4F900001EF7000050
:100B90009CF500009FF50000DFF60000F4F800006F
:100BA00081FB000012FE00002E0100003B0400004B
:100BB00038060000E107000032090000500900007B
:100BC000840800001B0700009A04000030010000A8
:100BD00062FD0000E9F9000027F7000094F500002D
:100BE00097F50000D9F60000D7F8000074FB00006C
:100BF00012FE00003201000033040000D2050000A4
:100C0000A8070000D408000004090000A1080000A3
:100C100014070000BD0400004D01000078FD000035
:100C200016FA000044F70000A3F50000B3F5000039
:100C3000E6F60000EBF8000084FB0000FFFD00007A
:100C40002C010000180400008F050000230700009D
:100C5000A60800000A090000480800000507000077
:100C6000C204000062010000CDFD00004BFA00004C
:100C70006EF70000B7F500007FF50000AAF600004F
:100C80008FF800001BFB0000C2FD0000F500000013
:100C9000AD030000A60400006C060000260800005A
:100CA000B00800009408000089070000FB05000060
:100CB0000D03000068FF0000F2FB000099F800003F
:100CC00060F6000098F5000038F60000CBF7000051
:100CD00026FA0000BFFC0000DEFF00003203000027
:100CE00004040000EF040000ED060000FB07000014
:100CF000A8080000730800007D07000087050000B9
:100D000072020000C4FE000010FB000022F8000088
:100D100025F60000CAF50000B2F6000061F80000F8
:100D2000F0FA0000AFFD000083010000B3030000F3
:100D3000F70300003605000098060000BC0700001D
:100D4000660800007208000092070000AD05000070
:100D500076020000ABFE000014FB000016F8000055
:100D600047F6000004F60000CAF6000080F8000014
:100D700022FB0000F0FD0000DA010000AD030000DE
:100D80007C030000B8040000BD050000FA06000066
:100D900017080000480800001D0800006806000051
:100DA00079030000FCFF00001BFC00000AF90000B2
:100DB000C8F60000F3F5000055F60000ABF70000A0
:100DC00029FA000002FD0000130100009903000051
:100DD000CD030000B3030000C5040000400600007E
:100DE000190700007E080000790800009207000043
:100DF000BD0500003E0200007BFE0000D9FA0000A5
:100E0000E8F700002BF60000C1F500006CF60000CA
:100E100067F800000EFB000099FE0000B70200001A
:100E200007040000C3030000380400008B04000026
:100E30008F050000FA060000C90700002A0800001C
:100E400068070000540500004302000071FE000026
:100E5000D6FA0000F4F700002FF60000BFF50000FE
:100E600070F6000066F800003DFB000003FF000084
:100E70003A03000050040000160400002E04000095
:100E8000710300005704000082050000980600006E
:100E90006B070000E2060000D505000060030000BB
:100EA000DCFF00005DFC000046F900000EF70000CA
:100EB000FFF5000008F6000065F70000CEF900001D
:100EC0002CFD0000E50100002204000003040000E6
:100ED0009A030000B0020000610200008F020000CF
:100EE0002F040000A8050000920600003C07000047
:100EF000ED05000056030000050000006AFC00003C
:100F000070F900001FF7000004F6000018F600005A
:100F100053F70000ACF9000040FD0000BE010000E6
:100F2000580300003D03000019030000E901000020
:100F30001701000018010000BF0200008E0400002D
:100F40002106000061070000D7060000210500000F
:100F50005D020000F2FE0000BBFB0000DEF80000B6
:100F6000EEF6000040F6000086F600002FF80000C4
:100F7000BBFA000038FF0000C8020000E2020000D7
:100F80002703000078020000860000004F000000E8
:100F9000060100004B02000013050000AC06000033
:100FA0001F0700004C07000095050000E302000049
:100FB000C3FF00005AFC000074F9000080F7000035
:100FC00077F6000045F600008CF7000015FA0000E7
:100FD00075FE0000100200009102000017030000DF
:100FE000F102000051010000710000004C000000FF
:100FF000A8000000AF02000025050000B1060000B7
:10100000AC0700006A070000D90500006E0300006D
:101010006200000014FD000013FA0000DCF700007D
:1010200090F6000055F600005DF70000EDF90000B5
:1010300011FE00008901000020030000820300006F
:10104000C5020000E201000068000000ABFF0000E4
:101050005C00000047010000060400004606000096
:10106000E8060000AF0700008F06000059040000EA
:10107000DA01000083FE00008CFB000017F900007D
:1010800078F70000A7F6000030F7000024F9000010
:10109000D5FC00003B01000063020000BF0200001D
:1010A000120300006C01000064000000ECFF00006F
:1010B000BCFF00002001000019030000050500002E
:1010C0009D0600001D070000AE0600001A05000086
:1010D000A3020000A7FF00009AFC000012FA000023
:1010E00040F800004FF700007DF700000EF9000007
:1010F0006DFC000005000000F3010000F502000097
:10110000A7020000D6010000C2000000B6FF0000E8
:1011100006000000920000009F0200003B05000056
:101120002206000042070000FD0600003305000013
:10113000540300004F00000046FD00008CFA000040
:1011400063F800002AF7000007F7000078F80000B5
:1011500065FB000010000000360200005C02000089
:101160001B0300009801000050000000BBFF0000BE
:10117000D3FE00009DFF0000BB0000006B020000DA
:10118000D6040000070600001C0700003E07000010
:101190000C0600002B0400009401000010FF00006A
:1011A0008EFC000072FA0000E2F8000010F8000067
:1011B0007BF80000F7F90000DDFC0000CEFF000026
:1011C000FE0000009E0100008B010000E400000012
:1011D0005D00000099FF000079FF0000CDFF0000D6
:1011E000B60000003E0200006B030000AF040000E8
:1011F000A905000000060000F5050000D604000067
:1012000002030000230100000CFF0000D1FC0000DD
:10121000E5FA000092F900001EF90000AAF90000AA
:101220005DFB0000CDFD000091FF00007D0000008F
:101230001D010000E9000000860000000F00000012
:10124000A8FF0000C7FF0000D5FF000076000000E7
:101250007E010000C701000092020000D8030000D8
:101260002F040000BF040000EC0400004004000054
:1012700067030000C6010000A2FF0000BCFD0000E3
:10128000DEFB00004AFA00008EF9000096F900002B
:10129000ABFA00002FFC0000CBFD0000E5FE0000D3
:1012A0007AFF00005500000088000000A200000046
:1012B000770000004C0000003800000099FF00009B
:1012C000E5FF00002A00000058000000FD000000BB
:1012D0005E0100000B020000E40200004F0300006A
:1012E0006B0300002B0300007802000034010000B3
:1012F000A8FF000040FE000007FD0000EFFB00001B
:101300004DFB000053FB0000EEFB0000C0FC0000A2
:1013100090FD0000B9FE000056FF0000BCFF000079
:10132000D3FF0000C8FF0000ECFF0000B2FF000088
:101330003C000000F0FF0000D7FF00009F0000000D
:1013400076000000B30000002F010000C101000082
:101350000D02000010020000BB020000400300006C
:101360000D0300009D0200000602000018010000AD
:10137000F7FF000004FF00000CFE0000BCFC0000B2
:1013800058FC00007DFC00005AFC0000EEFC000050
:10139000D5FD000094FE000061FF0000DAFF0000B0
:1013A000EBFF000033000000820000008A00000014
:1013B0008C000000AD000000C5000000C50000006A
:1013C00097000000920000007E0000007300000003
:1013D000B9000000BE000000E8000000600100004D
:1013E0008D0100009501000014020000570200006A
:1013F000CC0100006A0100001E010000470000004F
:1014000097FF0000BFFE00000AFE0000FFFD000085
:101410008DFD0000BFFD0000C0FE000015FF0000B4
:1014200059FF00001D00000051000000B000000046
:10143000270100002C0000009D0000000E010000AC
:101440009900000018010000C10000003A000000EF
:10145000470000005F00000081000000CC00000099
:10146000C8000000BA000000D0000000D600000054
:10147000230100002C010000E90000009C01000095
:10148000880100000901000009010000C1000000FE
:1014900081000000F9FF000061FF0000ECFE000089
:1014A00010FF0000F3FE00000FFF000010FF00001F
:1014B000BEFE00001EFF000074FF000080FF000061
:1014C000EFFF0000FCFF000028000000A10000006A
:1014D000280000005200000038000000B4FF0000A7
:1014E000E5FF0000070000000200000030000000DF
:1014F0008400000028000000DAFF00005F00000008
:101500004E000000030000000C000000F1FF00008E
:101510004800000071000000D2FF0000D7FF00006B
:10152000AEFF000030FF0000B1FF0000CFFF000061
:1015300098FF0000B3FF0000F9FF00006D000000FD
:101540005D000000270000000E0000008EFF00007C
:1015500066FF0000CFFF0000FFFF00003100000029
:10156000750000006E0000003A000000F1FF00006E
:1015700014000000750000005E0000005400000030
:10158000D1000000CC000000A1000000AD00000070
:101590006200000005000000EFFF0000A2FF000055
:1015A0001DFF00006FFF00004AFF000035FF000034
:1015B0006CFF000056FF000094FF0000B4FF000025
:1015C00098FF0000C9FF0000CDFF000010000000E0
:1015D000760000002C000000510000001E000000FA
:1015E000CDFF0000EEFF0000F1FF00000000000052
:1015F000100000005C00000009000000BDFF0000BA
:101600004A0000003B0000000B0000003800000012
:1016100042000000BD000000030100003C0000008B
:1016200019000000C8FF000022FF000092FF000028
:10163000A2FF00002FFF000034FF0000F5FF0000B4
:101640004E0000000E000000ECFF000085FF0000CF
:10165000E8FE0000F5FE00008BFF0000C8FF000060
:10166000FFFF00003B0000002E000000D0FF000044
:101670003AFF000076FF0000D6FF00009FFF000049
:10168000C6FF0000FBFF00000F0000002F0000005D
:1016900044000000E6FF000067FF0000F6FF0000C6
:1016A000090000006AFF000012000000D6FF0000E1
:1016B00075FF000030000000840000007E00000084
:1016C00037000000C7FF000058FF000058FF00006F
:1016D000A7FF0000050000004400000033000000E8
:1016E000D6FF00003800000001000000AEFF00003F
:1016F0003E000000C7FF00001C0000004200000088
:10170000D2FF0000E1FF00009EFF0000A6FF0000E6
:10171000A6FF00000E00000068000000E0FF0000CF
:10172000B7FF0000D7FF0000CFFF0000F5FF00006B
:101730001D000000600000008B000000560000004B
:101740006200000043000000ECFF00001D000000EC
:10175000070000000B000000400000002B0000000C
:101760006700000039000000140000002D00000098
:10177000E6FF0000E3FF0000FFFF0000E4FF0000C1
:10178000050000003A000000230000001F000000D8
:101790002600000013000000390000006E00000069
:1017A000720000005C000000EBFF0000E8FF00009A
:1017B000E0FF0000CBFF00002A0000000C0000004A
:1017C0001000000026000000FCFF0000DAFF00000F
:1017D0000600000039000000730000005D000000FA
:1017E000C9FF0000D0FF0000AAFF0000A5FF000015
:1017F000F6FF00000D00000019000000E9FF0000E6
:10180000C2FF0000070000002200000004000000EA
:1018100015000000FEFF0000F9FF0000D7FF0000E8
:10182000C5FF0000DAFF0000EFFF0000F3FF00003B
:10183000E1FF0000F1FF0000E1FF0000DAFF00001F
:10184000B0FF000088FF0000B7FF0000CAFF0000E3
:10185000070000002D0000001A000000200000001A
:10186000D6FF0000C9FF0000E4FF0000DEFF00001B
:10187000FDFF00002D0000001A000000D8FF00004E
:10188000D2FF0000C2FF0000BCFF0000D0FF00003C
:10189000F4FF00000C00000015000000E7FF00004E
:1018A000C8FF0000E2FF0000E6FF00002800000083
:1018B0002A000000FBFF0000F8FF00000900000004
:1018C0001F0000000700000006000000E3FF00000A
:1018D000CBFF0000E0FF0000E0FF0000F7FF00008A
:1018E000EEFF0000CAFF0000D0FF0000BEFF0000B6
:1018F000CDFF0000F4FF0000D5FF0000B7FF00009F
:10190000A4FF0000BAFF0000CCFF0000B6FF0000FB
:10191000BCFF0000ABFF0000AAFF00008BFF00002F
:101920007AFF000093FF0000A0FF0000A9FF000065
:1019300090FF00008DFF00008DFF0000A5FF00005C
:10194000B0FF0000A6FF0000B2FF0000B0FF0000E3
:10195000A3FF000082FF000075FF00007CFF000075
:1019600095FF0000BFFF0000DAFF0000DAFF000073
:10197000B3FF0000BDFF0000B6FF0000B7FF00008E
:10198000F0FF0000F1FF0000F1FF0000E5FF0000A4
:10199000D2FF0000DDFF0000EDFF0000FBFF0000B4
:1019A000B8FF000078FE0000C2FD00005AFD0000F4
:1019B00063FD0000C8FE00004CFF00007CFF00003B
:1019C00065FF000080FF0000CB000000DF0000008A
:1019D000670000005AFE000030FC00006EFE0000B0
:1019E0007E0000004E020000930200002101000072
:1019F00097020000C2020000C2030000540400006D
:101A00004102000060010000B5FF0000100000006E
:101A1000F5000000BF000000E0000000030000002F
:101A2000940000006A000000FDFE000030FE00008F
:101A3000AAFC0000F0FC000054FE0000C1FE000003
:101A40004AFF0000BCFD000054FD00006CFC0000DB
:101A5000CAFA000054FE0000C90000006102000044
:101A60000E02000047000000B7020000DD03000086
:101A70008905000042060000CF030000C0020000FC
:101A8000AE0000000C000000A0FF000056FE0000A9
:101A9000F1FE000037FE00002AFE0000BDFE00003F
:101AA0009BFD000060FD0000C6FC00008FFC0000F4
:101AB000C1FC000061FC0000E1FC0000F0FC000043
:101AC00005FB0000CBFB00007000000023030000BA
:101AD00013040000B4010000ED00000054020000F7
:101AE00090020000460500000F0500007903000089
:101AF00039020000700000007600000095FF000031
:101B0000CDFE00002FFE00000BFD000035FD0000A3
:101B1000A0FD00007FFC000083FB00006CFA0000C9
:101B200008FA00006DF9000064F70000ECF900000D
:101B300070FE0000B70100007A0300006A02000096
:101B40005B0300009304000059050000E10600005B
:101B50001505000008030000840100004A00000091
:101B6000B6FF000081FE000080FD0000B9FC00000F
:101B700068FC000011FD00000AFD000036FB0000BB
:101B800082F9000012F900000EFA000001F80000CE
:101B900067F90000A9FF0000600300002B050000AA
:101BA000A40300006A030000D00300001D0300002E
:101BB0002A0500006D04000023020000FD00000063
:101BC000F9FF00002B00000065FE000070FC000023
:101BD000B3FB00001FFA000080FA0000FEFB0000CB
:101BE000A2FC000074FC000043FA0000C3F60000F1
:101BF0001BF80000040000001C0500004005000068
